:020000040800F2
:10000000F0FF022009D4060851D406086909020845
:1000100051D4060851D4060851D406080000000047
:1000200000000000000000000000000051D406089D
:1000300051D406080000000051D40608399A00087F
:1000400051D4060851D4060851D4060851D40608E4
:1000500051D4060851D4060805B900080DB90008A6
:1000600015B900081DB9000825B9000851D40608C3
:1000700051D4060851D4060851D4060851D40608B4
:1000800051D4060851D4060851D4060851D40608A4
:1000900051D4060851D4060851D406082DB90008D9
:1000A0008DE600089DE60008C5E600080DE600089C
:1000B0001DE600082DE600083DE6000841F40008B2
:1000C00041A9000849F400084DA9000851D40608C8
:1000D00051D40608C12A06088D2B0608792C06087B
:1000E00035B9000851D4060851D40608D5E60008F1
:1000F000E5E60008F5E600087DE6000851D40608AC
:1001000051D4060851D406084DE6000851D406081B
:10011000652D0608512E06085DE600086DE600080C
:10012000A1B10008B5B10008C9B10008DDB10008EF
:10013000F1B1000851D4060851D4060851D406087C
:1001400051D4060851D4060851D40608F9D5000840
:1001500005B2000819B20008000000003D2F060893
:1001600051F4000859A90008000000000000000038
:1001700051D4060851D4060851D4060800000000E6
:100180000000000051D40608293006081531060881
:1001900051D406080000000000000000000000002C
:1001A00000000000000000000000000051D406081C
:1001B00051D406080000000051D4060800000000D9
:1001C000000000000000000000000000000000002F
:1001D000000000000000000051D4060851D40608B9
:1001E00051D406080DD5000851D4060805E70008CB
:1001F0002DB2000841B2000855B2000869B20008EB
:0C0200007DB2000891B20008A5B2000811
:1080000010B40C4B4FF0E02C1A68DCF8180019681B
:108010008A42F9D159688842F6D89C684FF47A713F
:1080200001FB04F31B1AB3FBF4F35DF8044B01FBF3
:1080300002307047A01A002070B40D4A0D4E0E4C4D
:108040000E4D4FF0010C36F8020F002340FA03F1F9
:10805000C90704D50CFA03F114609180083201338A
:10806000102BF3D104F58064AC42ECD170BC7047A6
:10807000AC1A00204AFD0608000002400020024021
:10808000002A4FEA014C30B503460ABFE6468E4649
:108090008C4600F1C005002419689A6841EA0C0179
:1080A00042EA0E029A60C3E900140C33AB42F3D1EA
:1080B000D0F8C030C0F8C44043EA0E03C0F8C03066
:1080C000C0F8C84030BD00BF30B4436919690A68C0
:1080D00022F001020A609A68B3F80CC01468E268E2
:1080E00022EA0C02E260046890F810C020680822BE
:1080F00002FA0CF202403AD1224890F88C52022047
:1081000000FA0CF06060002D2FD0187E01282FD0CF
:10811000D3F8A0100131C3F8A010EFF31180502163
:1081200081F312885C68DD6B216821EA05011D6C12
:108130002943C0B2216080F3118898681969DC6A0C
:1081400000680C601C6B4C605C6B8C609C6BCC6042
:108150004262B3F87C20C2620A68012422430A60AA
:108160001C76C2689B891343C36030BC7047FEE72E
:10817000D3F8A4000130C3F8A4000B6862F3000335
:108180000B60F2E7A01A002010B40D4CD4F8903226
:10819000002B12DD002004F5257C0146DCF874304C
:1081A00003F1C00259600C339342FBD1D4F89032F2
:1081B000013083420CF1AC0CF0DC5DF8044B7047ED
:1081C000A01A002070B5484C04EB401393F86025CA
:1081D00002B970BD072800F283804C2202FB0042E6
:1081E00094F8A45894F8A5E892F8466683F8466592
:1081F00075454FF000034FEA401C82F846360CD01C
:108200000EEB4E0304EBC30393F8A828561E012E71
:108210004FEA4E0356D9032A4ED004EB0C00A0F8C7
:108220004415EFF31182902383F3128890F84635BA
:10823000B0F8441543EA41030021D2B29BB280F862
:10824000461582F3118894F88C12D0F85C451A090F
:1082500082EA13225A40B9B1D0F84815646FD2436C
:108260001B019BB202F00F0201208840134304F16E
:10827000C0011D0402D46268024362600C345B00DA
:10828000A1429BB2F5D170BDD0F84815646F1B01B7
:1082900010319BB202F00F0201208840134304F119
:1082A000C0011A0402D46268024362600C345B00AD
:1082B000A1429BB2F5D170BD0EF1010202F00302A2
:1082C000AA42AAD0734404EBC303034493F8B5183D
:1082D0000029A2D004EB0C03012283F846259CE779
:1082E00000239B78FFDE00BFA01A0020704700BF6C
:1082F000704700BF024B03EB401393F861057047D2
:10830000A01A00204368826C10B49A61EFF31182C6
:10831000502383F312884168C46B0B6823EA04037B
:10832000446C2343D2B20B6082F31188D0E9074139
:108330008268036912681C605960D0E909419C6039
:10834000D960B0F85C10D16200235DF8044B03766D
:10835000704700BF026890F810C01168022303FA4A
:108360000CF3194200D1704710B4074C41684FF02C
:10837000000C84F808C908686CF3000008605DF818
:10838000044B5360704700BFA01A00200B4890F8C0
:10839000091989B101EB4101002310B4490000F62D
:1083A0000C101C4650F82320063302B114608B4297
:1083B000F8D15DF8044B7047704700BFA01A002049
:1083C0000B4890F8091989B101EB4101002310B461
:1083D000490000F60C101C4650F82320063302B169
:1083E00014608B42F8D15DF8044B7047704700BFB2
:1083F000A01A0020204B1B78002B3CD12DE9F04126
:108400001E4C94F80929A2B31D4E04F60C125027F5
:108410004FF02C0E1D4607E094F8091952F8180B7E
:1084200001338B42056024DA117C0029F4D05168B5
:10843000880AA0F5801006EB000853284FF0FE0CC8
:1084400098BF98F810C0EFF3118087F31288D1F825
:1084500024800EFB0C4C08F10108CCF8F489D1F80B
:1084600014C04CF0010CC0B2C1F814C080F31188E4
:10847000D2E7BDE8F081704700000020A01A00207C
:108480004CFD060800EE100AB8EE400A704700BF27
:10849000BCEEC00A10EE103A98B27047704700BFA9
:1084A000704700BF704700BF704700BF0120704792
:1084B000094A0A4BD2F8682CD3F83C05526AD3F823
:1084C000401592F85330012B08BFB2F85030A0EBA2
:1084D000010008BFC0187047A01A0020982B002088
:1084E000012380F85130704710B4EFF311818023DD
:1084F00083F312880C4AC9B2D2F84435D2F8484501
:10850000D2F84405D2F8482581F31188904203F14E
:10851000FF33A3EB04038CBF0020012003EBC0203A
:108520005DF8044B704700BF982B0020074BD0F834
:1085300094105B68D0F8A0205B1A9A42B8BFC0F8CC
:10854000A030012380F8CC3000207047001000E0FC
:10855000072809D8054B4C2202FB0033B3F8440628
:10856000B0FA80F04009704700207047A01A002040
:10857000072806D8034B4C2202FB0033012283F864
:1085800046267047A01A0020384A38B54C2303FB12
:10859000002393F8533603B938BD92F8A4C892F873
:1085A000A5389C450ED003EB430402EBC40494F8B9
:1085B000A8E80EF1FF35012D4FEA430446D9BEF17C
:1085C000030F3ED04FF04C0C0CFB002CACF84416C3
:1085D000EFF31181902383F31288BCF844469CF892
:1085E000463643EA44030024C9B29BB28CF846469F
:1085F00081F31188190A92F88C4281EA13115940CB
:1086000004B1C9434C2404FB00241B0118489BB24D
:1086100001F00F021A43D0F84C55D4F88C06012112
:10862000A847D4F88816B4F850C6CA88D4F8843657
:1086300042EA0C02CA8058601A6842F001021A60CD
:1086400038BD5D1C05F003056545BBD01C4402EB3D
:10865000C404044494F8B5180029B3D04C2303FB98
:108660000023012483F84646ACE700BFA01A00208F
:10867000982B002010B584464FEA810E102312F487
:10868000004F14BF0E2407245200013BCCF80040D9
:1086900092B2F444F3D100EB81128C01035142F801
:1086A0002130122010BD00BF10B584464FEA810E64
:1086B0000424130B03EB430318331201013CCCF8E1
:1086C000003092B2F444F4D100EB01130A0184505B
:1086D00043F82140062010BD704700BF704700BF1F
:1086E000034B00EB400003EBC00393F81D097047F8
:1086F000A01A0020074B93F85035834207D9064B48
:1087000000EB400003EBC003D3F8200970470020C2
:10871000704700BF982B0020A01A002034E700BF4C
:10872000072808D8044B03EB401393F8602512B1D7
:10873000012283F846257047A01A0020072808D890
:10874000054B03EB4013B3F84405B0FA80F0400941
:1087500070470020704700BFA01A0020054B93F817
:108760005035834283BF044B03EB4013D3F85005CD
:1087700000207047982B0020A01A002003689A69F7
:10878000D10508D54FF4807213218177DA611A6818
:1087900022F080021A609A69920508D54FF400729F
:1087A00013218177DA611A6822F080021A609A69CF
:1087B000510508D54FF4806213218177DA611A6878
:1087C00022F080021A609A69120508D54FF40062FF
:1087D00013218177DA611A6822F080021A609A699F
:1087E000D10408D54FF4805213218177DA611A68D9
:1087F00022F080021A609A69920408D54FF4005260
:1088000013218177DA611A6822F080021A607047BA
:10881000194B1A4A1968D2F85435CB1A322B05DC99
:10882000D2F86835CB1A002B11DC7047D2F85815F6
:1088300049B192F864358888096803F001031B0187
:1088400000FA03F38B610023C2F868357047D2F851
:1088500058356BB118689B8810B44469234218BF1F
:108860001B0432315DF8044B8361C2F86815704710
:108870003231C2F868157047A01A0020982B0020EA
:10888000D0E90920131A58425841704790F84F38E0
:1088900030B53BB990F84D1890F84E380124DAB253
:1088A000914200D830BDB0F8565804FA03F22A437A
:1088B000A0F856280133F2E70379024613F00100CD
:1088C00006D0D2E90731D2685B1A013A03EA020006
:1088D000704710B5037913F0010304460ED0FFF77B
:1088E000EBFF034650B1226A6369E1689B5C013289
:1088F000B2FBF1F001FB1022DBB22262184610BD80
:1089000003799B070AD5436A8269D154436A026995
:108910000133B3FBF2F102FB11334362704770473E
:10892000017170470379014613F0020007D00B690B
:10893000D1E90921013B521A1A40D2B2981A704764
:10894000074AD2F858354BB192F8642599881868CF
:1089500002F00102130101FA03F383610020704762
:10896000982B00204FF40070034B1060D3F878353B
:108970000B600020704700BF982B0020002070473C
:1089800001207047012070470020704710B41C6917
:1089900094420CD394460A4661448C42996938BF8C
:1089A000A4EB0C0261445DF8044B66F03BBF5DF83C
:1089B000044B7047012343770020704708B50346F6
:1089C0008269006BD96A02449A6101B1884700202C
:1089D00008BD00BF436A1B681B6A5B685B78024680
:1089E00013F0010008BF5077704700BFF0B5214C6D
:1089F000214A224B95B0054604F10C00CDE9000256
:108A0000049304F110000023CDE90503CDE90E33F2
:108A10001B4A09920B93221D1093139311936B6AB7
:108A20002F7F0A921868012302228DF80C300793D9
:108A30008DF820308DF834308DF848303B1D02928F
:108A40000E460C9362F084FC8FB1330E63710634D2
:108A5000320C330A22706370A670686A694657F058
:108A60007FFA6B6A186862F073FC15B0F0BD0534CC
:108A7000EEE700BF0000002040310020D58900084B
:108A8000B589000810B5044694B0502206496846DE
:108A900066F0C8FE606A694657F062FA636A186851
:108AA00062F056FC14B010BDB0FD0608C2628161D0
:108AB000704700BF2DE9F0410446406A00681E4639
:108AC0000F46904662F044FC237FA069002B35D00E
:108AD000234D030E6B75052205F116039870EA64A9
:108AE000020C000A58701A703B68AB650020D8F879
:108AF00000302B66012E2363286724D0022E1BD161
:108B0000D8F80420A866796885F86400E9661344FB
:108B100014496A670120236385F87800E967124BDE
:108B2000627F606AA3F11401002A08BF194657F05A
:108B300017FAE36A73B1206BBDE8F0810B4B042296
:108B4000A3F11505CAE7074B85F86460C5E91A303B
:108B50006867E4E7636A186862F0FAFBEBE700BF56
:108B600000000020BD890008300000201500002012
:108B700000B583B081610192049A0093C26201231F
:108B80006A4601A9FFF796FF03B05DF804FB00BF3A
:108B9000043070470D4B93F8B025D3F8AC15024460
:108BA000D2B283F8B02593F8B02501441206C3F879
:108BB000AC1505D593F8B02582F0800283F8B02576
:108BC000034B012283F89420704700BF982B0020AC
:108BD000000000202DE9F047154FD7F8B455ED0AF5
:108BE00020D00026B14607F2EC587419D7F8B835F2
:108BF0001048D3F828A0C7F8E49504EBD4746410A7
:108C000010234246E102D0470F280BDD0A4B03F147
:108C1000100153F8042B013207D18B42F9D12546BC
:108C2000B542E2DCE802BDE8F087661CF8E700BF69
:108C3000982B0020503100208431002030B585B0C1
:108C400068465AF001FE1048104AD0F8FC10009B0C
:108C50000F4D4FF0604441F08071C0F8FC100021CE
:108C600000F1C840C4F8B05FA0F56500516011681C
:108C7000084CA0F67D60A0FB030341F001019B0CB2
:108C8000A360116005B030BD00ED00E0001000E011
:108C900055CEACC5A01A00202DE9F04F01308E4C06
:108CA0008E4D8F4E83B001F1FF385FFA80FA1027A6
:108CB00060F064FA4FF4FA7B4FF0E0224FF47A7CD4
:108CC000C1466B68C3F30803002B40F0CB80EFF381
:108CD0001183002B40F0C68023689169206883428D
:108CE000FAD160688142F7D8D4F808800CFB08F00C
:108CF000A0EB010EBEFBF8FE0CFB03EE4FF00108EB
:108D0000CDF804906B68C3F30803002B40F08E800D
:108D1000EFF31183002B40F089802368916920686C
:108D20008342FAD160688142F7D8D4F808900CFBEE
:108D300009F0411AB1FBF9F10CFB0313A3EB0E038D
:108D4000B3F57A7FDED3BBF1010BDDF80490B8D127
:108D500050464FF47A7B60F0C9FE4FF0E022DC46CB
:108D60006B68C3F30803002B40F09980EFF3118385
:108D7000002B40F094802368916920688342FAD1E7
:108D800060688142F7D8D4F808800CFB08F0A0EBAB
:108D9000010EBEFBF8FE0CFB03EE4FF00108CDF810
:108DA00004906B68C3F3080323BBEFF311830BBB81
:108DB0002368916920688342FAD160688142F7D8BC
:108DC000D4F808900CFB09F0411AB1FBF9F10CFB47
:108DD0000313A3EB0E03B3F57A7FE2D3BBF1010BD0
:108DE000DDF80490BCD1B9F10108BFF461AF03B064
:108DF000BDE8F08FEFF3118387F312889069116952
:108E0000C90344BFC6F8FC8590692168D6F8FC9573
:108E1000DBB283F311884944D4F808900CFB09F3C2
:108E20001B1AB3FBF9F30CFB0133D2E7EFF3118309
:108E300087F3128890691169C90344BFC6F8FC859D
:108E400090692168D6F8FC95DBB283F31188494418
:108E5000D4F808900CFB09F31B1AB3FBF9F30CFBD5
:108E600001336BE7EFF3118087F31288916913697F
:108E7000DB0303D50123C6F8FC3591692368D6F8D6
:108E8000FCE5C0B280F31188A06873440CFB00FEBF
:108E9000AEEB010EBEFBF0FE0CFB03EE2EE7EFF394
:108EA000118087F3128891691369DB0303D50123CD
:108EB000C6F8FC3591692368D6F8FCE5C0B280F3AA
:108EC0001188A06873440CFB00FEAEEB010EBEFBE4
:108ED000F0FE0CFB03EE60E7A01A002000ED00E0BE
:108EE000982B00202DE9F043144CDFF8549083B008
:108EF00004F520764FF0020802E00834B4421AD09C
:108F000094F90650002DF8D1276807F13F4303F587
:108F10007E0309EB9323083493F8B40061F0F8F86A
:108F200034F8041C0123CDE900582A46384662F083
:108F3000C9F9B442E4D103B0BDE8F083AC1A002013
:108F40004CFD06082DE9F0411348144D4FF42572ED
:108F5000002166F0BFFC4FF00008A5F1BC0705F644
:108F6000EC3440F2FB2655F82810002354F8332047
:108F700091420BD001330F2BF8D1002008F10708E4
:108F800061F0C6F8B045EED1BDE8F08107EBC30350
:108F900093F8AC0CF2E700BF6C24002008FE060832
:108FA00010B5084C08485AF0BFFC4022002104F5D7
:108FB000C06066F08FFC4FF0FF33C4F84036C4F851
:108FC000433610BD982B00200E00440010B54FF41E
:108FD0004010104C82B05AF0A7FC0023012102225D
:108FE000CDE9002120461A464FF4C05162F06AF9DB
:108FF000636A23F470236362636A43F42023636229
:10900000636A23F470436362636A43F420436362D8
:1090100002B010BD0000024010B5044665F0A6FB8A
:1090200081B22046BDE81040FFF7CCB838B50B4DF3
:1090300000EB400005F60C1303EBC00393ED027A3E
:10904000D3ED037AE7EE007AC4002544B0EE670A58
:1090500065F08CFBD5F80C39186038BDA01A0020DB
:1090600010B5044665F082FB81B22046BDE8104091
:10907000FFF78ABA38B5194B93F8A42893F8A538A6
:109080009A4226D1164A92F847560DB34FF0000C7B
:1090900002F5C9626146136859621868083261F3C3
:1090A000C710186032F8040CD862186840F08000CD
:1090B0001860186861F341001860DC6832F8020C2F
:1090C0000CF1010C20436545D86022F8021CE2DC5B
:1090D00038BD62F0E1FC0028D4D138BDA01A0020D0
:1090E000982B0020F8B50C4B1D685A6915400540B7
:1090F0005D617DB1094F0126B5FA85F4C4F11F0405
:1091000007EB840306FA04F4D3F8000603689847D3
:10911000A543F1D1F8BD00BF003C0140982B0020D1
:109120002DE9F8430269C36812EA030828D005460E
:109130000E464FF00047B8FA88F327FA03F2D243FD
:109140001B3B2A6108EA0208042B16D8DFE803F06B
:10915000332A221A0300B36A002B35D003F1FF39FA
:1091600000231FFA89F9B362746A34B12368204678
:10917000494698476468002CF8D1B8F1000FDAD15D
:10918000BDE8F8837068A98E03689847B8F1000FAE
:10919000D1D1F5E7B068298F03689847B8F1000F7F
:1091A000C9D1EDE7F068E96B036889B29847B8F177
:1091B000000FC0D1E4E73069296C036889B2984791
:1091C000B8F1000FB7D1DBE7EB6A1FFA83F9CBE701
:1091D00038B51E4CD4F83C3573B1D4F84025D4F8DA
:1091E0003C359A4208D0D4F84035E218013392F861
:1091F0008806C4F8403538BD154AD2F8682C0023DB
:10920000526AC4F8403592F8531001F0FF05B1B12D
:10921000B2F8505082F853305DB10E49D01C10F8AE
:1092200001CF01F801CB0133B2F850C09BB29C458D
:10923000F5D809484023043201215BF039FCC4F819
:109240003C55D4F83C050028CDD1D4E7982B00201C
:10925000A01A0020203200200427002090F850306F
:109260005A1C0344D2B280F8502083F83C1090F886
:1092700051300BB1132A01D963F08ABB704700BF8C
:10928000002280F8512063F083BBF8B5A0F6680493
:109290002379DB0727D5657994F84C3805F0010769
:1092A0003D460BB3D4F848341A68D36A5B0853625E
:1092B00094F8503823B1B4F85A380133A4F85A3826
:1092C000636C85F001025979186861F0EBFA0123AB
:1092D00084F84F38002384F84D3884F84E38A4F8C9
:1092E000563884F84C38F8BD94F84F68012E04BF06
:1092F00094F84D3884F84E382046FFF7C7FA636C6F
:109300004EB9012284F84F287A4059791868BDE88F
:10931000F84061F0C7BA002284F84F283A46F4E7D3
:1093200070B5A0F66804A1F12903666C334D30686E
:109330000022302B426231D895F8883E95F8891E7C
:109340000133DBB2012B85F8883E09D9B4F85638D1
:1093500085F8882E5B08A4F856384B1C85F8893EA2
:1093600095F8892E0023082AA4F8583815D185F8D5
:10937000893EB5F88A3E01339BB2032BA5F88A3E9D
:1093800008D92379DB0705D5E36A94F856084BB36F
:10939000216B98470023A4F8563870BD5B396C29BF
:1093A0000CD8B4F8563885F8882E5B0843F0800353
:1093B000A4F8563895F8893E0133CFE794F8513830
:1093C000002BCDD1012285F8883EA5F88A3E802366
:1093D00084F85128A4F85638717985F8892E61F0FF
:1093E00061FABDE7E3696269D054E369E268013379
:1093F000B3FBF2F102FB1133E361CBE7982B0020C2
:1094000070B5094C05460926013E00D170BD94F99E
:1094100000001BF0A7F9031E04DBEA186178117243
:10942000A278EA540434EFE76C0A07082DE9F84300
:10943000DDF820800F4615460021202204461E46F6
:1094400066F048FAB8F1000F0CD0D8F80030E3818C
:109450001B0C2382D8F80430B8F80A20E3821B0CD6
:1094600062822383384663F0E7FAEB0619D4431E81
:10947000B8B107EB000C01E0013B12D31CF801ED81
:10948000BEF12E0FF8D1C01A421E032AA8BF032234
:10949000082B03F10109A8BF08239046B9441A46D6
:1094A00006E008280246B946A8BF08224FF0000887
:1094B0004FF02033394623606360204666F0B2F9EE
:1094C00004F10800154B238142464946837066F03B
:1094D000A9F9611EE21D11F801CFACF16103192B4E
:1094E0009CBFACF1200C81F800C09142F3D104F193
:1094F0000A0011F8013FA3F16102192A9CBF203B29
:109500000B708142F5D118232373330CA382E572CB
:10951000099B6683E361BDE8F88300BF202020003B
:109520002DE9F04FD848DFF890B3006887B0CBF84A
:109530005405002B60D09C18A046154601F5FE7618
:109540000C461FE0002D64D0DBF88435AB4200F000
:10955000C780DBF88035AB4200F0F980DBF8883556
:10956000DBF88C15AB424BD8A94200F27481691A22
:1095700020465EF01BFF0135454504F5007406F5F5
:10958000007639D0DBF89035AB42DBD8DBF8A0753C
:10959000EB1A396BDA0802328A4203F0070A02D367
:1095A000BB6B9A420BD93946104603925EF0CEFE51
:1095B000039A0746002800F08881CBF8A0053B7984
:1095C000002B40F01F81D7F82890B9F1000F00F070
:1095D00075813B6BD21AFB680AEBC20203EB422295
:1095E00020463B464FF400710135C847454504F518
:1095F000007406F50076C5D1002007B0BDE8F08FF5
:10960000A942B4D94FF400720021204666F062F9F5
:10961000B1E74FF400722946204666F05BF98023DB
:1096200084F8BE310C2384F8C231DBF88015974AE8
:10963000DBF87835C4F8C6119142C4F8CA3100F39A
:109640000F81934A934F82FB010287FB01070A4473
:10965000C817C0EB6212C0EB27308F4F84F8C101EE
:1096600087FB02C7C2EB821C8010A1EB0C01013109
:1096700020F03F0017440843D117C1EBE7110A441B
:1096800084F8BF21814A84F8C001013B934200F372
:10969000F3807F4A7F4882FB031280FB03101A4449
:1096A000D917C1EB6212C1EB20317B4884F8C51198
:1096B00080FB0270C2EB82178910DB1B013321F0A3
:1096C0003F0110441943D317C3EBE0131A4484F845
:1096D000C41184F8C3214AF65523A4F8FE314AE7A1
:1096E0004FF0FF3384F8EC3184F8ED3184F8EE313B
:1096F00084F8EF315223237063706123A37084F8E0
:10970000E7314123E37084F8E6317223002784F8BF
:10971000E43184F8E531DBF89835C4F8E8314FF4EA
:10972000F0723946201D66F0D5F8552384F8FE31D5
:109730006FF05503C4F8F071C4F8F471C4F8F8710F
:1097400084F8FC7184F8FD7184F8FF3113E74FF45D
:1097500000720021204666F0BDF8504B03CB45F661
:10976000EB0323809023C4F80710A3700222082182
:10977000F823C4F80300617322746375DBF878354D
:109780002273A27384F82C20DBF880259B1A2362B5
:10979000DBF88825DBF88C359B1A63620023E372C3
:1097A000E3736377A377E37784F82D3084F82E3062
:1097B00084F82F3084F83130394BA361394BC4F829
:1097C00042303E232377012384F83030364A802309
:1097D00084F8403084F846104AF65521A4F8FE116A
:1097E00003CA324BC4F84700C4F84B1003CB1388AC
:1097F000A4F84F309378C4F85200C4F8561084F897
:109800005130B8E64FF400720021204666F062F84D
:10981000BAF1000F60D13B6C04F12009002B00F07D
:1098200097803B6B22491122CDE900AA2046FFF721
:10983000FDFD3B6C1A6C002A00F099801B6B1D49E2
:10984000CDE900AA48461122FFF7F0FD04F14009D6
:109850004FF4E07387E0E91A20465EF0A7FD8AE640
:10986000FF2284F8C1214FF6FF72A4F8BF21074AF6
:10987000013B93427FF70DAFFF2384F8C5314FF6CC
:10988000FF73A4F8C33126E7A01A0020FF03FB00F2
:10989000832008829755454181808080209D07085C
:1098A0003F00FF0029940E0D2C9D0708389D0708E6
:1098B000189D07081C9D0708982B002049464FF467
:1098C0000072204666F006F855E62D4A231F43F83D
:1098D000042F9E42FBD14EE6D7E910274FEA0A1328
:1098E000002A42D0023B002F3FF445AE013BBF6C43
:1098F000F9D1A1464FF40073002F3FF43CAECDE9FF
:10990000035609EB030A059408E00024CDE900643E
:10991000FFF78CFDBF6CBFB1D14515D03C793968DC
:109920003B6B484607F11C06112209F12009002C67
:10993000EBD17A793C6942F02102CDE90064FFF76E
:1099400075FDBF6C002FE7D1DDE90356059C12E6DB
:10995000CDE900AA5346DBF87C1508222046FFF724
:1099600065FD4FF4F0737F6CC6E7013BBBE7CDE9C3
:1099700000AA0449534648461122FFF757FD65E700
:10998000DEADBEEF1C9D070838B590F82830012BDE
:10999000044606D0407F08B9012038BD0023637714
:1099A00038BD406A03681A7B92B9637F002BF3D0FD
:1099B0000A4D0B49022305F68C6256F08BFA95F896
:1099C0008D3ED84303F0010300F001006377E7E721
:1099D0001B6A002BE9D0002038BD00BF982B002067
:1099E0009800002038B5044694F82830012B07D0A1
:1099F000637F0BB100236377012038BD1B6A23B15D
:109A0000606A03681A7B002AF8D1637F002BF3D0C9
:109A1000074D0849022305F68C6256F05BFA95F86B
:109A20008D3E03F00102DB076277E5D5DCE700BF7E
:109A3000982B00209800002010B4EFF3118310221F
:109A400082F31288094A0A4C11684FF0E020013174
:109A50001160816951600022C4F8FC250269DBB203
:109A600083F311885DF8044B704700BFA01A0020F3
:109A7000982B002030B4EFF31183102282F3128868
:109A80004FF0E0220E4894691169C90344BF0121D7
:109A9000C0F8FC150B4948BF94690D68D0F8FC2547
:109AA000DBB283F3118889684FF47A702A4400FB93
:109AB00001F31B1B30BCB3FBF1F300FB023070471A
:109AC000982B0020A01A0020224B5B68C3F30803E8
:109AD00030B4D3B9EFF31183BBB91F4B4FF0E02C77
:109AE0001A68DCF8180019688A42F9D15968884266
:109AF000F6D89C684FF47A7101FB04F3181AB0FB96
:109B0000F4F030BC01FB02007047EFF31182102328
:109B100083F312884FF0E02310489C691969C90348
:109B200044BF0121C0F8FC150B4948BF9C690D6872
:109B3000D0F8FC35D2B282F3118889684FF47A727A
:109B40002B4402FB01F0001B30BCB0FBF1F002FB28
:109B50000300704700ED00E0A01A0020982B0020C1
:109B60002DE9F047FFF7B0FF224D234FD5F8904283
:109B700006464FF000094FF0AC08002C2DDD002305
:109B80001A4608FB0351013391F831139C4242EA13
:109B90000102F6D142EA090A5FFA8AFA91467B6825
:109BA000C3F30803B3B9EFF311839BB9FEF728FAA7
:109BB000801BB0F5FA6F02DCB9F1000FDDD1BAF10C
:109BC000000F04D00D4B93F88E2E542A09D0504626
:109BD000BDE8F087FFF74EFFEAE7CA464FF00009FD
:109BE000DDE7B3F8942E0132A3F8942E5046BDE879
:109BF000F08700BFA01A002000ED00E0982B0020A5
:109C0000AF4B93F88C320BB901207047AC48AD498B
:109C10000268AD4B2DE9F04FA1FB02125209A3FBE4
:109C20000213DB0803EB830387B0A2EB4303DAB232
:109C30000592A64A92F850150491A54902F56A6466
:109C400004EB83070022A1F1880300F2445A019338
:109C500090468946049B984500F00E81DAF818205A
:109C6000DAF80460D2F89430D2F898500293FFF7F3
:109C70002BFF029B0390B00000F1085000EB431053
:109C8000019B93F890C1914B93F88E2E05F180665D
:109C9000393E542A00EB861600EB8C1302D18B4917
:109CA000A1F896CE9E4240F280811968002900F00A
:109CB0007581196C002900F08A81D3F88010002981
:109CC00000F08781D3F8C01003F580730029E9D133
:109CD000181A9E424FEAA01040F26781291A4529BE
:109CE0004FF0000628BF45213546B64603EB8111EB
:109CF0009B4616460DE01A6C002A40F0EF80D3F820
:109D00008020002A40F01A81D3F8C02003F5807328
:109D10002AB9994206D91A68002AECD040339942F0
:109D200000F2E08032467646112E40F24681DEF1A6
:109D3000150100F14281674BD3F89C3098423CBF3B
:109D4000644BC3F89C00019B0398D3F89431C01A6C
:109D500000281CDB039803F5F42303F59073984265
:109D600088BF0346019888BF0533C0F89431594B2A
:109D70000198D3F89C30052B86BF053BDBB200234E
:109D800080F8903153484FF0FF33C0F89C3031B128
:109D900005FA01F1C6F114060125B5400D434E4EFA
:109DA000C5F3C43306EB8303D3F8400D05F01F035E
:109DB00006EB8303D3F8401D41EA0031C5F344109C
:109DC00006EB8000C5F3842306EB8303D0F8400D37
:109DD000D3F8403D41EA001141EA032181EA112311
:109DE00083EA131303F00F00019BD3F890300F2880
:109DF00003F1010340F0BF80B1F5803F80F0BB80EC
:109E0000542A4FEA11113FD0019AB1F5606FC2F8A0
:109E1000903045D0A9F80C1094F85830059883423A
:109E20000CD0BA6823689B1A23603A6B63689B1A4C
:109E300063600023BB603B6384F8580023680133F0
:109E40002360BB680133BB604FF6FF73994205D1B5
:109E50006368013363603B6B01333B6308F10108C6
:109E6000B8F1080F04F15C0407F15C0709F114096B
:109E70000AF1200A7FF4EEAE019A0123012082F854
:109E80008C3107B0BDE8F08F1048B0F8902E013249
:109E9000A0F8902E019AB1F5606FC2F89030B9D158
:109EA000074A92F8A53803EB430302EBC30343448C
:109EB00093F8B5380D2BADD1802389F81E30ABE770
:109EC000A01A00201F85EB51CDCCCCCC982B0020C4
:109ED000183D0020000000204CFD06088033994208
:109EE0007FF620AFA3EB0B0C3E4A4FEAAC1C0CF103
:109EF000010C82FB0CB2A2EBEC72012AB8BF01226A
:109F000095404FF0010C9644013A0CFA02F21543C9
:109F10009C46DCF800209AB1DCF84020002A5AD098
:109F2000DCF88020002A59D0DCF8C0200CF5807CB9
:109F300042B16145EDD89B466346EAE6C033EEE6A2
:109F40000CF1400C6145F6D9ACEB03029211254BA4
:109F5000013283FB02B3A3EBE273012BB8BF0123F1
:109F60009D409E440122013B02FA03F31D436346D8
:109F70009B466346CDE6542A05D11B49B1F8902E85
:109F80000132A1F8902E019AC2F89030D2F88C30AC
:109F90000133C2F88C304FF6FF713DE74033181A99
:109FA0009E424FEAA0103FF699AEBCF1000F04D0DC
:109FB000019B0CF1FF3C83F890C1542A7FF44EAF13
:109FC000094AB2F8923E0133A2F8923E46E7803346
:109FD0007EE6C0337CE60CF1800CB3E70CF1C00CDC
:109FE000B0E700BF56555555982B002070B51F4C53
:109FF00094F8A42894F8A5389A4232D1D4F8905213
:10A00000002D11DD1A4894F88C62002406B3037EFB
:10A01000012B20D002691368013443F00103A542EB
:10A0200000F1AC001360F1D1FFF74EFD114BD3F8F6
:10A030009841002C0BDD03F5CE7303EBC4041968C3
:10A040009A88C86808330243A342CA60F7D170BD3A
:10A05000FEF758F9DEE7002380F89C30FEF752F94E
:10A06000D8E761F019FD0028C8D170BDA01A002002
:10A07000341D0020903C00202DE9F04FD0F80090D6
:10A08000057CD9F800304FF0020A0AFA05F52B4298
:10A0900083B002D103B0BDE8F08F4169DFF888B228
:10A0A0009F4B4FF04C0808FB01B804465868D8F89D
:10A0B0004C36B8F850261F68D8F88466FB6823EA47
:10A0C0000203984AFB60C2F8BC01336823F0010325
:10A0D00033609BF88C3223B9C9F8045003B0BDE853
:10A0E000F08F3046019159F02DFC8E4A01990123E1
:10A0F00088F87036D2F8C431002B00F005813B6837
:10A1000023F080033B604C2303FB01B34FF0FF308F
:10A1100093F88036F862062B2FD8DFE813F0CD00D5
:10A120002E00A5002E0007002E0083003B6A23F4BA
:10A1300080733B624C2303FB01B33C6A93F88106B6
:10A1400060F349243C623C6AC0F3400060F3CB24D6
:10A150003C62F86993F8824664F30100F86193F871
:10A160008306FB6960F30713FB61FB6923F00C03B3
:10A17000FB613B6A43F480733B624C2303FB01B3F6
:10A1800031684BF6EF7421400024A3F86446316037
:10A190003068B3F8641601433160316893F86D0696
:10A1A00060F30D313160316893F86B0660F38B21F9
:10A1B0003160316893F86A0660F3092131603168D3
:10A1C00093F8690660F3C7113160316893F8680647
:10A1D00060F38611316093F86C06316860F34511C5
:10A1E0003160B3F86606716860F30F017160D3F8EF
:10A1F0005C06D3F88416B060D3F86006F0601620D1
:10A200004860086840F001000860D3F84C16B3F8C5
:10A21000503609684248CC682343CB604368C2F893
:10A22000C03159E73B6A23F480533B624C2303FB64
:10A2300001B3386A93F8814664F34D303862F869A7
:10A2400093F8824664F30920F86193F88306FB696A
:10A2500060F30F33FB61FB6923F44063FB613B6AEE
:10A2600043F480533B6288E73B6A23F010033B6270
:10A270004C2303FB01B33C6A93F8810660F3451459
:10A280003C623C6AC0F3400060F3C7143C62B869AA
:10A2900093F8824664F30920B86193F88306BB699A
:10A2A00060F30F33BB61BB6923F44063BB613B6A5E
:10A2B00043F010033B6260E73B6A23F001033B621B
:10A2C0004C2303FB01B33C6A93F8810660F341041D
:10A2D0003C623C6AC0F3400060F3C3043C62B8696E
:10A2E00093F8824664F30100B86193F88306BB6972
:10A2F00060F30713BB61BB6923F00C03BB613B6ACE
:10A3000043F001033B6238E7FFF7DEFB054A257C9B
:10A31000D4F800900199C2F8C4010AFA05F5EEE6F6
:10A32000001000E0903C0020A01A0020464B5B6823
:10A33000C3F308032DE9F0470546002B5FD1EFF387
:10A340001183002B5BD1414B4FF0E0241A68A069C8
:10A3500019688A42FAD159688842F7D89E684FF442
:10A360007A7101FB06F4241AB4FBF6F401FB0244F3
:10A37000354E374F4FF010084FF0E02C4FF47A7EF7
:10A380004FF001097268C2F30802CAB9EFF31182F3
:10A39000B2B91A68DCF8180019688A42F9D159680C
:10A3A0008842F6D8D3F808A00EFB0AF1091AB1FBCF
:10A3B000FAF10EFB0212121BAA42E3D3BDE8F087AA
:10A3C000EFF3118288F31288DCF81800DCF8101023
:10A3D000C90344BFC7F8FC95DCF818001968D7F822
:10A3E000FCA5D2B282F311885144D3F808A00EFB29
:10A3F0000AF2121AB2FBFAF20EFB0122DBE7EFF3CC
:10A400001181102383F312884FF0E023C9B29E69B3
:10A410001A6912F4803F0E4A1EBF0120C2F8FC05E3
:10A420009E690A4B1868D2F8FC2581F31188024412
:10A4300098684FF47A7101FB00F4A41BB4FBF0F4AC
:10A4400001FB024494E700BF00ED00E0A01A0020E9
:10A45000982B00202DE9F0473C4B3D4D3D4E00F13F
:10A46000FF3810274FF0E0204FF47A7C6A68C2F37F
:10A470000802002A54D1EFF31182002A50D11A6841
:10A48000846919688A42FAD159688C42F7D8996868
:10A490000CFB01FEAEEB040E4FF00109BEFBF1FE1A
:10A4A0000CFB02EE6A68C2F30802EAB9EFF311820C
:10A4B000D2B91A68846919688A42FAD159688C42FB
:10A4C000F7D8D3F808A00CFB0AF1091BB1FBFAF18D
:10A4D0000CFB0212A2EB0E02B2F57A7FE2D3B8F1C6
:10A4E0000108C3D2BDE8F087EFF3118287F3128829
:10A4F00084690169C90344BFC6F8FC958469196879
:10A50000D6F8FCA5D2B282F311885144D3F808A042
:10A510000CFB0AF2121BB2FBFAF20CFB0122D9E788
:10A52000EFF3118187F3128884690269D20303D59E
:10A530000122C6F8FC258469D3F800E0D6F8FC2592
:10A54000C9B281F311887244A1E700BFA01A0020AC
:10A5500000ED00E0982B002030B50C4683B0054696
:10A56000D8B1036803F13F4303F57E039B0A0C4A0D
:10A57000134493F8B4005FF0CBFDC4F3810204F000
:10A580000303CDE90032C4F34113A9882868C4F35A
:10A59000001260F097FE03B030BD4FF0FF33E6E7E6
:10A5A0004CFD060800B1D7E7704700BF70B50E4BF1
:10A5B00093F85065AEB10D4C002504E00135B5426D
:10A5C00004F120040DD0237F002BF7D0E068002891
:10A5D000F4D0217D0135FFF7BFFFB54204F120041F
:10A5E000F1D1012070BD00BF982B0020E41F002096
:10A5F00038B50409013C072C18D80E4D00F00F03A4
:10A6000035F8140040FA03F212F0010210D00122D2
:10A6100002FA03F3013B1840254465F0EFF995F881
:10A62000C03D054A034402EBC30038BD002038BDDD
:10A63000104638BD4CFD0608AC1A002008B51D2098
:10A64000FFF7D6FF10B190F9063053B11E20FFF787
:10A65000CFFF10B190F9063003B108BD5523C38078
:10A6600008BD5523C380F1E7F8B50268017C0446B4
:10A67000022310688B40184206D1106808238B40D3
:10A68000184218BF5360F8BD6569536004238B40BE
:10A690005360EFF31183502282F312882A6C116801
:10A6A000C9070BD5DBB283F3118895F86C3013B171
:10A6B00095F87D60FEB12268217CDEE7506880B2AB
:10A6C00088B9D5E909618E422BD0AF690F44D760B4
:10A6D00089B222D806462869401A80B2506000210B
:10A6E000AE6285F86C10116841F00101DBB21160B7
:10A6F00083F31188D9E795F87A00FFF779FFAB6EFD
:10A70000DA68012166F3C302DA6085F87D1000285B
:10A71000D1D02821FFF720FFCDE7711A89B251600F
:10A72000DDE7012285F86C20BCE700BF70B51B2077
:10A73000FFF75EFF08B12923C3801C20FFF758FFF5
:10A7400008B12923C380FEF741FC2D482D4E2E4C25
:10A7500059F0EAF85EF0A6FA00220221432059F0EF
:10A76000B7FB5BF0BFFB294901F580534FF0A040D8
:10A770000122C1F8600C83F8242683F83126826B0D
:10A7800042F400128263224AC3F828264FF48172F1
:10A79000A3F82C264FF401620025A3F8262606F123
:10A7A000C80106F1A00283F82F565FF07FFFD6F8AC
:10A7B000F030184AA2FB03239B090421013BE1620C
:10A7C000A362636943F001036361236865F30923AE
:10A7D0002360236865F306132360236843F0800336
:10A7E0002360E36843F00103E3602A460221692005
:10A7F00059F06EFB236843F00103236070BD00BF76
:10A800000700340000000020004C0140A01A002086
:10A8100040004001D34D621038B55BF063FB1B2054
:10A82000FFF7E6FE08B12923C3801C20FFF7E0FEF6
:10A8300008B12923C380204B93F8CD41012C01D0CE
:10A84000012038BD1D4DC3F8D051FEF7BFFB1C4899
:10A8500059F06AF85EF026FA00220221432059F0EE
:10A8600037FB184A02F580534FF0A04083F8244686
:10A8700083F83146C2F8600C816B134C41F400112F
:10A880008163C3F828464FF48174A3F82C4605F180
:10A890002002002405F148014FF4016583F82F469A
:10A8A000A3F826565FF002FF224621464FF0FF3004
:10A8B00059F00EFB204638BD903C0020F4000020EB
:10A8C00007003400A01A002040004001174A184930
:10A8D000D2F8883030B443F47003C2F888300B6883
:10A8E00043F001030B600B689B07FCD58B68104A93
:10A8F00023F003038B60936813F00C0FC3F3810103
:10A90000F9D19160136809480A4D23F0867323F446
:10A91000803313604FF41F044FF000635560C2F89A
:10A92000A010D46030BC8360704700BF00ED00E031
:10A930000038024002300300704700BF002070471B
:10A940000148FDF71BBF00BF7C3E00200148FDF71A
:10A9500015BF00BFD03E00200148FDF70FBF00BF6C
:10A96000243F002030B1036882881B691A4214BF5B
:10A9700001200020704700BF10B1036882889A62EE
:10A98000704700BF10B1036882889A61704700BFAA
:10A990002DE9F04F076889B07D680790D7E904601A
:10A9A0007168AA6812F08002FBD1BB69347C93F80D
:10A9B0000EE006920EF0030ECDF814E093F80DE0D1
:10A9C000326893F8119093F80F8001920EF0010A0B
:10A9D00093F80CE05A8903920EF0010E4FF0020C2E
:10A9E000CDF810E093F810E01A6802920CFA04F423
:10A9F0000EF0010B44F00C04B3F808E05B6809F0BA
:10AA0000030908F00308002800F08680019A079ED9
:10AA1000466146685460047C0068069A0CFA04F4A7
:10AA200044F00C044460086862F300000860306879
:10AA300062F300003060326842EA0C0232600A6859
:10AA40004BF6EF7002400A600A684EEA02020A60A2
:10AA50000A6869F30D320A600A6868F38B220A609B
:10AA60000A68059C64F309220A600A686AF3C7123F
:10AA70000A600A68049C64F386120A600A686BF331
:10AA800045120A604A68039C64F30F024A60029A06
:10AA90008A60CB603268FB690240326030681A8994
:10AAA000024332603268587C60F30D3232603268A3
:10AAB000D87B60F38B2232603268987B60F3092286
:10AAC00032603268587B60F3C71232603268187B9C
:10AAD00060F386123260187C326860F3451232608F
:10AAE0005889726860F30F027260D3E90023B26084
:10AAF000F360336843F0010333600B6843F00103F4
:10AB00000B606B6843F001036B606B6843EA0C03F6
:10AB10006B6009B0BDE8F08F079A7261019A5460CA
:10AB20000A6860F300020A600A684BF6EF700240A0
:10AB30000A600A684EEA02020A600A6869F30D3286
:10AB40000A600A6868F38B220A600A68059860F355
:10AB500009220A600A686AF3C7120A600A68049840
:10AB600060F386120A600A686BF345120A604A684D
:10AB7000039860F30F024A60029A8A60CB600B6808
:10AB800043F001030B600B6843F002030B606B683A
:10AB900043F002036B6009B0BDE8F08F70B4046845
:10ABA00090F838506368012284F824201A6822F053
:10ABB00040021A60B0F804C02289624516D0BCF584
:10ABC000807F6146A8BF4FF480710229B8BF02217F
:10ABD0001A6891FAA1F1B1FA81F122F03802013933
:10ABE00042EAC10292B21A60A4F808C0027BA17ABC
:10ABF000914209D0196872B321F0020119601968F5
:10AC000021F001011960A2721A6842F040021A6034
:10AC1000226A267B9368C3B100218C4614329C447F
:10AC200093680131002BF9D196B18DB1012909D872
:10AC3000BCF1070F06D801EB81018B00226A134497
:10AC40001B7B2BB970BC57F0A9BE0EB1002DF5D1FE
:10AC500070BC57F0D3BE41F002011960196841F091
:10AC600001011960A272CFE738B52C4AD0F89030B4
:10AC70005268D0F88810044673B1501A83420BDC36
:10AC800094F88030C4F88820012B10D0D4F8843098
:10AC90000133C4F8843038BDD4F89430C4F8882027
:10ACA0000B44C4F88C3094F88030012BEED16168ED
:10ACB000201D04F19805EFF3118C102383F3128803
:10ACC00063681B6A0BB3D4F8A0302A461BB1D36962
:10ACD0001432002BFBD10B6A6BB1996839B99342DE
:10ACE00009D0196829B15B6899680029F7D0143335
:10ACF000F3E7C3E900055FFA8CFC8CF31188D4F804
:10AD000084300133C4F8843038BD0D625FFA8CFCA6
:10AD10008CF31188FFF742FFB8E700BF001000E096
:10AD20002DE9F041826992F88C30012B8AB00546FA
:10AD300049D0023B012B50D892F8FC30D26C2D4CFC
:10AD400063F07F03137087693B6DD7F8108003F1C0
:10AD5000010E0FCCEC46ACE80F00FB6CCDE9003ED9
:10AD60000FCCACE80F0094E8030007F110068CE864
:10AD70000300EFF31180102383F312883B691B6AF1
:10AD8000002B2ED0029B6A461BB1D3691432002BD4
:10AD9000FBD1D8F8203073B1996839B99A420AD0FA
:10ADA000196829B15B6899680029F7D01433F3E773
:10ADB0001E60C3F804D0C0B280F31188AA6911697B
:10ADC0000B6A002BFCD1136D5A8852BAEA819A881B
:10ADD00052BA2A82DB885BBA6B8201200AB0BDE8D6
:10ADE000F081C8F820D0C0B280F311883046FFF758
:10ADF000D5FEE3E7140B07082DE9F04190F88C30FD
:10AE0000056D012B8AB004466FD03ED9023B012B61
:10AE100067D890F8FD30C26C5A4E63F07F03137010
:10AE2000036DD0F8108003F1010E00F110070FCE72
:10AE3000EC46ACE80F00E36CCDE9003E0FCEACE889
:10AE40000F0096E803008CE80300EFF31180102355
:10AE500083F3128823691B6A002B00F08A80029B0F
:10AE60006A461BB1D3691432002BFBD1D8F82030CD
:10AE700023B3996839B9934220D01968D9B15B6876
:10AE800099680029F7D01433F3E7C36C4FF0FF3211
:10AE90001A605A609A60DA60D0F890300522B3F5F3
:10AEA0007A7FC0F8A0203BD8032380F88C300120A3
:10AEB0000AB0BDE8F0811F60C3F804D0C0B280F3CF
:10AEC00011882269136A002BFCD16B885BBAA4F845
:10AED0008030AB885BBAA4F88230EB885BBAA4F808
:10AEE000843001200AB0BDE8F08190F8FC2090F891
:10AEF000FD309B1A5B100133DBB205EB430235F8E2
:10AF000013305BBAA0F8803053885BBAA0F8823067
:10AF100093885BBAA0F8843001200AB0BDE8F081C4
:10AF200003691A7B0AB35B69FBB190F84830E3B15F
:10AF300090F8FC30C26C606563F07F03137090F88A
:10AF4000FC1090F8FD30026D0F48C4F8B4005B1A95
:10AF500007330121C4F8AC30E36C84F8B0100A4424
:10AF6000C4E9293284F88C10BBE7022384F88C30C2
:10AF7000B7E7C8F820D0C0B280F311883846FFF791
:10AF80000DFE9EE7140B07082D850008F8B54569EE
:10AF9000002D70D02C68236A1B7B002B77D1D4E95D
:10AFA0000467317C6368022202FA01F1D6E900608D
:10AFB00041F00C01002F35D0D0F800C0D7F804E0E4
:10AFC0002CF0010CC0F800C0DEF8000020F00100F9
:10AFD000CEF800007160397C8A40396842F00C027A
:10AFE0004A605A6822F002025A605A6822F001024E
:10AFF0005A60236A1B6943B1236A686C1B699847CE
:10B00000012800F08D80022837D0236ADA69FAB966
:10B010005869002842D099692162C3E90522BDE838
:10B02000F840BBE59A681706FCD49A68D2070DD49D
:10B03000026822F00102026071605A6822F0020286
:10B040005A60236A1B69002BD6D1DEE7DA68ECE789
:10B05000226A94F82410127B1433D2B2236200299E
:10B0600037D1002A55D12846FFF792FC2B681A6A7F
:10B07000D169002914DCF8BD2362236ADA6914332C
:10B08000002AF9D1236ADA69002AE1D1C0E7AB6866
:10B09000002B84D01A689B88936180E72062F8BDFA
:10B0A000D06951699C69002965D00125657361608B
:10B0B000596980B260810029DDD092693649DB6927
:10B0C000002A0ABF0A460121002159735A6058819B
:10B0D000F8BD276A2E68B9683B68B069002B52D06A
:10B0E0004FF0010C80F80DC043608BB27169438151
:10B0F00051B1F06979684381274B00290ABF19468D
:10B100000123002341604373002384F82430002A84
:10B11000A9D0AB68002BA6D01A689B889362A2E7DF
:10B12000236A2A68143B2362136AD96900297FF7CE
:10B130006CAFDE6959699769A1B1844687F80DC083
:10B140007960B1B256697981002E3FF45EAFD26961
:10B150009B6951811049002B04BF00200B4650739E
:10B16000536052E78C460D494FF0FF0E81F864E1C1
:10B1700001F5B271E2E70D460849FF2681F86461E6
:10B1800001F5B27192E79C46044B4FF0FF0E83F835
:10B1900064E103F5B273A5E7B43F0020000000208E
:10B1A0000348D0F8743113B100F5B47018477047F4
:10B1B000000000200348D0F8983113B100F5C670A4
:10B1C00018477047000000200348D0F8BC3113B185
:10B1D00000F5D87018477047000000200348D0F8E9
:10B1E000E03113B100F5EA70184770470000002005
:10B1F0000348D0F8043213B100F5FC7018477047CB
:10B20000000000200348D0F8283213B100F5077081
:10B2100018477047000000200348D0F84C3213B1A3
:10B2200000F5107018477047000000200348D0F860
:10B23000703213B100F519701847704700000020F4
:10B240000348D0F8943213B100F5227018477047C4
:10B25000000000200348D0F8B83213B100F52B707D
:10B2600018477047000000200348D0F8DC3213B1C3
:10B2700000F5347018477047000000200348D0F8EC
:10B28000003313B100F53D701847704700000020EF
:10B290000348D0F8243313B100F5467018477047BF
:10B2A000000000200348D0F8483313B100F54F7078
:10B2B00018477047000000200F4B1049013800EB81
:10B2C000C00003EB8003086BD3F868210C4B9A4253
:10B2D00014BF4FF080734FF48003184382B00863AB
:10B2E000096B0B400193019BD2F8003143F001033D
:10B2F000C2F8003102B07047000000200038024060
:10B30000006402402DE9F0410138124C00EBC0000E
:10B3100004EB80041048D4F86881804514BF3820BD
:10B3200036200F4615461E465EF0F2FED8F8003174
:10B3300043F00103C8F8003194F97901C4F874713D
:10B34000C5F30112A909C4F87C61BDE8F04158F0C9
:10B35000BFBD00BF00000020006402402DE9F04F97
:10B36000BA4BBB4F85B007F1A00A4FF001094FF06F
:10B37000000BA3F55876B8460BE00BF1010BBBF1BF
:10B38000040F09F1010908F128080AF1050A00F083
:10B39000F78098F80030022BEFD19AF903305A1C4D
:10B3A00018BFDBB2A94A08BF002303EB430002EB3E
:10B3B000800014BF9E464FF00D0E5FFA8BF20D2BEE
:10B3C0005CD8A449002404E00134202C01F10301DD
:10B3D00054D00F78002FF7D14D789542F4D19E4983
:10B3E000D6F86C5104EB44040C44416894F8F24DD7
:10B3F0008460A942047000F03581D6F89051A942CA
:10B4000000F05781D6F8B451A94200F05681D6F821
:10B41000D851A94200F05981D6F8FC51A94200F058
:10B420005881D6F82052A94200F05F81D6F84452E4
:10B43000A94200F05681D6F86852A94200F0618115
:10B44000D6F88C52A94200F06C81D6F8B052A942CD
:10B4500000F06B81D6F8D452A94200F06A81D6F888
:10B46000F852A94200F06981D6F81C53A94200F0B5
:10B470007081D6F84053A94200F06F810133DBB2EE
:10B48000734500F10C009AD9002300939AF9042027
:10B49000531C18BFD2B26D4B08BF002202EB42040E
:10B4A00014BF94464FF00D0C03EB84045FFA8BF14C
:10B4B0000D2A5BD8674B002004E00130202803F1FF
:10B4C000030353D01F78012FF7D15D788D42F4D15B
:10B4D000614B00EB40001844636890F8F25DD6F8C9
:10B4E0006C01A560834225704DD0D6F8900183424F
:10B4F00000F0DC80D6F8B401984200F0D380D6F892
:10B50000D801834200F0DD80D6F8FC01834200F0D0
:10B51000E480D6F82002834200F0EB80D6F84402A3
:10B52000834200F0EA80D6F86802834200F0ED80A2
:10B53000D6F88C02834200F0F080D6F8B002834245
:10B5400000F0E780D6F8D402834200F0FE80D6F8FF
:10B55000F802834200F0F580D6F81C03834200F025
:10B560000481D6F84003834200F0FB800132D2B25E
:10B57000624504F10C049BD90023C8E90433FCE6BE
:10B5800005B0BDE8F08F4FF0000E774607EBC7031C
:10B5900006EB8303781C93F98071002FE6D12F4AC4
:10B5A00083F88191132183F8801102937346D41894
:10B5B000C8F814400190CDF80CE0FFF77DFE029B27
:10B5C000264AD3F88831196865F306011960DDE968
:10B5D0000030002BD0D061680D6867F300050D6066
:10B5E00003995158227C022303FA02F242F00C0222
:10B5F0004A60D8F810205568D5F800C067F3000CF1
:10B60000C5F800C0157C1268AB4043F00C035360D2
:10B61000D8F818301024C3E902471F82D8F8042054
:10B620005F600C321A60D8F81C304FF480711A60D9
:10B630001982C3E90177DF6009493B463A46FFF7C3
:10B6400061FE012388F80C3097E600BF60030020FC
:10B65000B83F00203C0B07084CFD0608680100209D
:10B660008DAF0008BC46394601EBC10706EB8707E2
:10B67000013197F98051002D7FF400AF3D4B0091CF
:10B680006344C8F810300846142387F8803187F8DF
:10B690008191FFF711FED7F888311A6864F306022A
:10B6A0001A60F3E64FF0480E02276FE74FF0240EC2
:10B6B0006CE74FF0240C0121D6E74FF0480C022133
:10B6C000D2E74FF06C0E032760E74FF06C0C0321BC
:10B6D000CAE74FF0900C0421C6E74FF0900E042704
:10B6E00054E74FF0D80C0621BEE74FF0B40C05210B
:10B6F000BAE74FF0B40E052748E74FF0D80E0627FB
:10B7000044E74FF0FC0C0721AEE74FF0FC0E072793
:10B710003CE74FF4A27E092738E74FF4907E0827D4
:10B7200034E74FF4907C08219EE74FF4A27C092176
:10B730009AE74FF4B47C0A2196E74FF4C67C0B21BC
:10B7400092E74FF4C67E0B2720E74FF4B47E0A271A
:10B750001CE74FF4D87C0C2186E74FF4EA7C0D21DE
:10B7600082E74FF4EA7E0D2710E74FF4D87E0C27CE
:10B770000CE700BF68010020D3B20D2B2BD800B519
:10B78000164B4FF0000C06E00CF1010CBCF1200F41
:10B7900003F103031CD093F800E08645F4D193F83D
:10B7A00001E08E45F0D10E4B0E480CEB4C0C02EB39
:10B7B0004202634400EB820193F8F23DC1F8683322
:10B7C00000F5587000EB820081F860335DF804FBEF
:10B7D00000205DF804FB0020704700BF3C0B070809
:10B7E0004CFD06080000002010B40C4C002304F5AA
:10B7F000777C01E0152B0CD003EB430201331CF8DE
:10B8000002108142F6D1144494F9DE035DF8044B32
:10B8100070474FF0FF305DF8044B7047903C0020BC
:10B8200030B5134C002304F5656C02E001331C2B8A
:10B830001BD05CF833508542F8D10CEBC30EDD0011
:10B840009EF804E08E45F1D10A4B02EB42022C44F3
:10B8500003EB820194F8554EC1F8684303F5587321
:10B8600003EB820081F8604330BD002030BD00BF93
:10B870004CFD060800000020F0B110B504460F484A
:10B8800094F804E0002300F5777C01E0152B11D03B
:10B8900003EB430201331CF802107145F6D1831803
:10B8A000617993F9DE232068D3B20D2B02D8BDE86D
:10B8B0001040B5E7002010BD00207047903C0020EC
:10B8C000800AA0F58010532807D8054B03441B7C41
:10B8D0000E2B02D8034AD05670470020704700BF95
:10B8E0004CFD0608209E070848B182880449B2FA38
:10B8F00082F208684FF00043D34003430B60704767
:10B90000003C01400120FDF7EDBB00BF0220FDF728
:10B91000E9BB00BF0420FDF7E5BB00BF0820FDF731
:10B92000E1BB00BF1020FDF7DDBB00BF4FF4787016
:10B93000FDF7D8BB4FF47C40FDF7D4BB40B338B51E
:10B9400005461446FEF708FEAB882968B3FA83F370
:10B95000C3F11F0303F00700800013F0F80F04FA8F
:10B9600000F20AD04B6A0F2404FA00F023EA000325
:10B970004B624B6A1A434A6238BD0B6A0F2404FAC1
:10B9800000F023EA00030B620B6A1A430A6238BD17
:10B99000704700BF2DE9F047DFF874A2542303FB82
:10B9A00000A384B0D3F8D481B8F1000F08D0D3E954
:10B9B00077490746002C00F0E48094F9063013B173
:10B9C00004B0BDE8F087B9F1000F00F0EA8099F902
:10B9D0000630002BF4D1431CDBB21522E371A271B7
:10B9E00089F80730162389F8063098F828005EF0A9
:10B9F0008FFB2046FEF7C6FF4846FEF7C3FF19211E
:10BA00002046FEF7CFFD19214846FEF7CBFD09265B
:10BA1000332524B9A6E0013D08D0FEF787FC236852
:10BA2000A28819690A424FF00A00F4D09A620520F0
:10BA3000FEF77CFC2368A2889A610520FEF776FC5D
:10BA4000013EE5D1332524B996E0013D08D0FEF74B
:10BA50006DFC2368A2881B691A424FF00A00F4D0DB
:10BA60002046FEF789FF0520FEF760FC4846FEF7FA
:10BA700083FF0520FEF75AFC2046FEF783FF0520D2
:10BA8000FEF754FC4846FEF77DFF0520FEF74EFC0E
:10BA90002046FEF767FF00287FD12046542407FB8D
:10BAA00004F40AEB040595F8E63195F8E421002B3F
:10BAB0000CBF162636263146FFF740FF95F8E521E4
:10BAC00031464846FFF73AFF49483C2200212044CE
:10BAD00063F000FFD5F8D43168465C68C5F8EC41E6
:10BAE00057F0B2FEB5F8E81103985DF085FA414BC6
:10BAF0009C4205465AD0404B9C4262D03F4B9C42F0
:10BB00006AD0542303FB07A3D3F8EC21136843F056
:10BB100001031360236823F0010323602561236878
:10BB200043F470632360A36823F48063A360A36875
:10BB30006FF30903A360A36843F40043A3600022EA
:10BB4000114698F92A0058F0C3F9002298F9290003
:10BB5000114658F0BDF9236843F0010323602FE735
:10BB6000FEF7E4FB013D4FF00A00F9D10520FEF796
:10BB7000DDFB62E7FEF7DAFB013D4FF00A00F9D189
:10BB80006EE7B9F1000F3FF430AF99F90630002BA2
:10BB90007FF416AF7B1CDBB222E74846FEF7E2FEDD
:10BBA0007BE71523A371431CE3711EE7144857F08C
:10BBB000BBFE144AD2F8203823F40013C2F8203810
:10BBC0009FE7114857F0B0FE0E4AD2F8203823F410
:10BBD0008003C2F8203894E70C4857F0A5FE094AC4
:10BBE000D2F8203823F40003C2F8203889E700BFD8
:10BBF0007C3E00200054004000580040005C0040A3
:10BC00001500200000300240160020001700200020
:10BC1000903C00202DE9F047794D05EB0013D3F857
:10BC20001C44002C00F0A58093F8267406464FEAC9
:10BC3000001838465EF06CFA7B09012207F01F07F6
:10BC4000013BBA40042B09D8DFE803F09B03A1A70E
:10BC500095006C494B6923EA02034B6105EB08032D
:10BC6000013693F82004FEF7C3FCF6B2824610B109
:10BC70001223C671837105EB080393F82104FEF7C4
:10BC8000B7FC814610B11323C671837105EB08031D
:10BC900093F82204FEF7ACFC074610B11423C671DA
:10BCA00083714544504695F823242621FFF746FE2C
:10BCB00095F8242448462621FFF740FE95F82524D0
:10BCC00006213846FFF73AFE4F4B9C4276D04F4B49
:10BCD0009C4268D04E4B9C427BD04E4B9C4200F025
:10BCE0008380636802210B436360636843F0010350
:10BCF0006360E36923F40063E361236823F4004392
:10BD00002360236823F480432360236823F4806343
:10BD10002360236843F400732360236843F4807333
:10BD20002360236843F004032360636823F40073F3
:10BD30006360636823F480736360236861F3C50301
:10BD40002360236823F080032360236823F40063C7
:10BD5000236023680B432360236843F001032360BF
:10BD60002369072262F30F032361236843F0400332
:10BD70002360BDE8F08723490B6A23EA02030B62C4
:10BD80006CE720490B6923EA02030B6166E71D4952
:10BD90008B6923EA02038B6160E71A494B6A23EA45
:10BDA00002034B625AE71C4857F0BEFD1B4AD2F80B
:10BDB000203823F48043C2F8203892E7184857F01F
:10BDC000B3FD164AD2F8243823F48053C2F824383D
:10BDD00087E7144857F0A8FD104AD2F8203823F41A
:10BDE0000043C2F820387CE70F4857F09DFD0B4A0E
:10BDF000D2F8243823F40053C2F8243871E700BF86
:10BE0000903C0020003802400030014000380040E3
:10BE1000003C0040003401400E0020000030024091
:10BE20000C0024000F0020000D0024002DE9F04F2D
:10BE30008FB000230793AB4BAB4CAC4FA3F57366AD
:10BE4000A84D4FF00009AA4BD5F800B093F86E2426
:10BE50004FEA9B23A3F58013532B00F2D280334487
:10BE60001B7C0E2B00F2CD80012A17F903A000F0F5
:10BE70000981022A02D1BAF1080F33D14FF001082B
:10BE80001FFA88F1504613F0E5FF14F06FF890F9AF
:10BE9000003013B1542B40F0098208F10108B8F1C9
:10BEA000050FEDD1079B0021002B00F0B4808E4AD6
:10BEB0000AE033441B7C0E2B0DD8FB5653450DD0A6
:10BEC000AC32944200F0A480906803689B0AA3F50A
:10BED0008013532BEDD900235345F1D14379687971
:10BEE0009842EDD109F10109B9F1080F05F11C05DE
:10BEF000A9D1079B0133042B079304F1AC049FD114
:10BF00000123DFF804B29A467A4B93F850250AF1E0
:10BF1000FF339A4272DD764BDBF80C609BF8102001
:10BF200093F882340892002E00F0E083B2883068E3
:10BF3000B2FA82F200F13F40C2F11F0200F57E002A
:10BF40000792800A6C4AD2F89052002D40F3AA80E2
:10BF500002F52572002705E00137AF4202F1AC027D
:10BF600000F09D8011688142F6D1079B5E4ACBF8B4
:10BF70000430AC2303FB0727CBF8187026B15FFA17
:10BF80008AF3F3710323B371079D7B6CF96B68002F
:10BF900001220324844002FA00F003437B64564BE1
:10BFA00093F88C322143F96302FA05F4B96C002B43
:10BFB00000F060812143B9646EB14D4BB28893F8B3
:10BFC000141C3368490141F0050101F0E5019A6153
:10BFD0003046FEF7C1FA786FA1B20122FCF750F8A3
:10BFE00038460AF1010AFCF78DF940F20113BAF163
:10BFF000090FABF81C300BF1200B85D10FB0BDE859
:10C00000F08F013A012A7FF66DAF4FF0000A35E755
:10C0100000297FF467AFA8683849002205E00132A3
:10C020000E2A01F10C0100F074834B689842F6D19E
:10C03000697952B25846FFF7F3FB314A40685168BC
:10C040000023884203F1010309D00E2B02F12402E0
:10C050003FF448AF5168884203F10103F5D1DBB2E8
:10C06000284A013B03EBC30302EB830393F98031BE
:10C07000002B7FF437AF1B4BC9EBC90903EB8903D6
:10C08000A36036E7BAF1010F3FF4F8AE09F10109F8
:10C09000B9F1080F05F11C057FF4D5AE29E7042F8F
:10C0A00000F00A811449AC2202FB0512D2F89C125E
:10C0B0000991002900F01183C2F894025421013043
:10C0C000C4B282F83C130C4982F83D436A1CC1F8A3
:10C0D0009022099A094817685179D2F808E09C46DD
:10C0E000002219E07C0C0708341D0020209E070860
:10C0F000903C0020982B0020A01A00206003002014
:10C100006801002000000020E41F002001320E2AF8
:10C1100000F10C0000F0FD8243689E45F6D152B25A
:10C120003846CDF82CC00A91FFF77AFBDFF8CC92A5
:10C13000A54BD0E90180AC22CC4602FB0532C2E916
:10C14000A980DCF8040000228045DDE90A1302F131
:10C1500001020AD00E2A0CF1240C3FF44FAFDCF898
:10C160000400804502F10102F4D1D2B29748013AAD
:10C1700002EBC20200EB820292F9800100287FF4F8
:10C180003DAFAC2082F8814100FB05F4601000EB6C
:10C19000A400C0EBC0100A9400EB803084010A9820
:10C1A00004EBA004640004EBA0044FF08C0C5420BA
:10C1B00082F880010CFB04F204EB4400844C00EB99
:10C1C000001004EB800004F54C7404EB420E7E4A30
:10C1D0000A9C14193268C4F898223322C4F80C233C
:10C1E0007A4AC4F80803062BC4E9CAECD2F8F02056
:10C1F00069D07848784C072B784B18BF03467848AD
:10C2000018BF20460139704CB2FBF0F0B2FBF3F3DB
:10C21000421EC8B2AC2101FB0541013BA1F810331D
:10C2200092B20023A1F8F0220B90FA62BB627A6905
:10C2300042F001027A613A6863F309223A603A688F
:10C2400063F306123A603B6843F080033B603B684F
:10C2500043F080033B604300D9B20C93072935D8E3
:10C26000DFE811F054003400AD013400180234004E
:10C27000DE01FB01079B103302FA03F30B43BB649F
:10C2800076B1584B326893F8141CB388490141F0D9
:10C2900005011B0401F0E50193613046FEF75CF9EE
:10C2A000786FA1B20022FBF7EBFE99E6079B012114
:10C2B000002B7FF4FCAD15E64A4A032382F8833451
:10C2C0000FB0BDE8F08F484B48489BE73B6823F030
:10C2D00001033B6001240023049302930093062290
:10C2E00023463846039401940D915EF07BFF0D992F
:10C2F0002246384658F0EAF90D990439032920D826
:10C30000DFE811F0E0011F00A601C3013B6823F044
:10C3100001033B60002101240A237B63062223469C
:10C32000CDE90341CDE90141009138465EF05AFF65
:10C3300022460021384658F0C9F9BB6943F008038A
:10C34000BB61099B1879002840F05A813B6843F093
:10C3500001033B600023D9F80420904503F1010359
:10C3600000F0B7810E2B09F12409F4D100234FF01E
:10C37000FF340993154A1E4804EBC40302EB830300
:10C380004FEAC409D3F86881804514BF38203620AD
:10C390005DF0BEFED8F8002142F00102C8F800218D
:10C3A0000B9B032B00F29381124B0C9A134433F82E
:10C3B000E81C054A1048AC2303FB05234FF0000C92
:10C3C000A3F8A012634622E0A01A0020000000207B
:10C3D0001441002044950800D0DD060010552200CD
:10C3E00040771B00903C0020882A1100A0BB0D0064
:10C3F00000640240440E07082C3E00206801002023
:10C40000974200F071810133042B00F07F8150F8D6
:10C410003320002AF4D1B84A9C461346D2F898211A
:10C420000132C3F8982103EBCC024FEACC03C2F8E7
:10C430009C7103440A9FB14A099817449A88114392
:10C4400099809022AE493B46FEF75CFFAD4BAE496A
:10C45000A14403EB8903AC2202FB0512D3F8883117
:10C46000D2F8A812186861F306001860D2F8A43256
:10C47000196841F0020119604FF480744FF440785C
:10C480001021A7F86C40A7F87080A7F86810B2F8E0
:10C490000CE3A7F86AE0D2F89802022100F1180C28
:10C4A00087F86E10C7F860C0D2F8085387F86F108D
:10C4B0001030099018687D664BF6EF7900EA0900A4
:10C4C0001860186840F010001860186840F4405078
:10C4D0001860186861F38B201860186861F30920F0
:10C4E0001860196841F080011960196821F0400155
:10C4F0001960196821F02001196059686EF30F0165
:10C500005960C3F808C0DD601968F961596839627B
:10C51000996879620020D968B962A7F88C40A7F8B9
:10C520009080A7F888000999B2F82C43C7F88010CA
:10C53000012187F88E10A7F88A40D2F8285387F88F
:10C540008F101A68C7F8845002EA09021A601A6844
:10C550001A601A6842F440521A601A6861F38B221A
:10C560001A601A6861F309221A601A6842F08002A0
:10C570001A601A6860F386121A601A6860F345122E
:10C580001A605A6864F30F025A6009999960DD6075
:10C590001A68FA625A683A639A687A63DA68BA6320
:10C5A0001A6842F002021A60089B8BF81030079B51
:10C5B000CBF80430CBF80C60CBF81870DFE43B68A4
:10C5C00023F001033B60012400230A22BA63022105
:10C5D000CDE90343CDE900340293062223463846D1
:10C5E0005EF000FE38462246022158F06FF8BB6923
:10C5F00043F40063BB61099B187900283FF4A6AEA1
:10C60000FDF7F6FF099B0446DA790A21FFF796F950
:10C610000CB15423E3807B6C43F400437B6495E6C8
:10C620000A233B643B6823F001033B6001240023A1
:10C630000622114604930293009338460394019412
:10C6400023465EF0CFFD22460621384658F03EF8DC
:10C65000FB6943F40063FB6173E60A237B673B6875
:10C6600023F001033B600124002304930293009311
:10C670000622072138460394019423465EF0B2FD5A
:10C6800022460721384658F021F83B6F43F0080353
:10C690003B6756E60A23FB633B6823F001033B60DC
:10C6A00001240023049302930093062204213846B8
:10C6B0000394019423465EF095FD224604213846FA
:10C6C00058F004F8FB6943F00803FB6139E60021E8
:10C6D0006FE6DBB209935C1E4CE6074A022382F840
:10C6E00083340FB0BDE8F08FDB00A2E64FF0FF32DD
:10C6F0000792104626E400BF903C0020341D002025
:10C70000C980000800000020A01A002000239B8898
:10C71000FFDE00235B68FFDE70B590F87A301C09FD
:10C72000013C072C0DD8184E054636F8140003F0CE
:10C730000F0340FA03F2D20703D595F87D20012AB2
:10C7400001D0012070BD9A40013A1040264463F0A8
:10C7500055F996F8C03D0D4A034402EBC30452F864
:10C760003320A38810691840ECD0002395F87B2073
:10C7700085F87D300A212046FFF7E0F8AA6ED368DD
:10C7800043F00803D360DCE74CFD0608AC1A002038
:10C7900038B505461446FDF7DFFEAB882A68B3FAC4
:10C7A00083F3C3F11F0303F00701890013F0F80FAF
:10C7B00004FA01F40AD0536A0F2000FA01F123EAC7
:10C7C00001035362536A1C43546238BD136A0F203D
:10C7D00000FA01F123EA01031362136A1C43146295
:10C7E00038BD00BFF8B50D4B93F8507597B10C4D9F
:10C7F000C7F109070924013C0ED0AE683079FDF776
:10C80000F7FE297DF27908B1FFF7C2FFA74205F1D3
:10C810004C05F0D10120F8BDA368FFDE982B002065
:10C82000E42000202DE9F04FDFF8A0A29AF815BC13
:10C830008BB0BBF1000F03D100200BB0BDE8F08F2F
:10C8400000222F21584613F0E5FB07460028F3D0BD
:10C850000568CAF8185CFFF70FF880460028EBD08F
:10C860004468CAF81C4C002CE6D08F4E0023324698
:10C8700001E00E2BE0D051688C4202F1240203F15A
:10C880000103F6D1DBB2DFF84892013B03EBC303AF
:10C8900009EB830393F98021002ACDD158464FF04C
:10C8A0002F0BA3F880B1FDF7A3FECAF8200C08B146
:10C8B000A0F806B00A21FA79FFF740F87B48002378
:10C8C00000F6A84151F83320954200F0D78101339A
:10C8D0000F2BF7D100205DF01BFC2B68744A23F06E
:10C8E00001032B60D9F8F0309342C0F0B78103F117
:10C8F000B772704902F55852A1FB0221890D013926
:10C9000089B24A1C0139B3FBF2F36B4A6B481B0A2C
:10C91000A2FB03321309A0FB03035B081209AAF868
:10C92000263C013A5B00EA62AAF8243CA9626B69E2
:10C9300043F001036B612B6823F440732B602B6879
:10C9400023F070032B6097F806A00AF001021AF09A
:10C95000020A40F086811046D64652460123797974
:10C96000089101F1FF3B5FFA8BFB4FEA4B01099104
:10C97000C9B20791072909D8DFE811F0570108006B
:10C980003E010800250108000C012200CDE901024A
:10C990000022039300920799CDF810E00622284662
:10C9A0005EF020FC2B6843F080032B60079B043B68
:10C9B000032B1DD8DFE813F01B011C000201180037
:10C9C0004FF0000CC5F874C00721CDE901020393B4
:10C9D000CDF810E0CDF800C0062228465EF002FC3B
:10C9E0002B6843F080032B602B6F43F008032B6709
:10C9F000BBF1030F00F24081314B099A134433F825
:10CA0000E83CEA681343EB60BAF1000F00F02E81B6
:10CA1000089B59000139C9B20122284657F056FE39
:10CA20003246002351688C4202F1240203F10103D3
:10CA300000F02E810E2BF5D14FF0FF3303EBC30333
:10CA400009EB83031F48D3F868A1824514BF38203F
:10CA500036205DF05DFBDAF8002142F00102CAF8F1
:10CA600000210023324651688C4202F1240203F176
:10CA7000010300F008810E2BF5D10020124900239C
:10CA80006022FEF73FFC236823F001032360204669
:10CA900056F058FF7B79013B032B00F2FC80DFE866
:10CAA00003F07673701900BF680100204CFD060882
:10CAB000006CDC02819F5E16598B4F01ABAAAAAABB
:10CAC000440E07080064024055830008903C002093
:10CAD0000000002005F1400223684BF6EF710B4087
:10CAE0002360236843F0100323602368012161F36E
:10CAF0000D3323602368022161F38B2323602368B5
:10CB000061F309232360236843F0800323602368D3
:10CB100023F040032360236823F02003236063682D
:10CB200040F22A4161F30F0363605D4BA260E36052
:10CB300000237268944206F1240603F1010300F019
:10CB4000A4800E2BF5D14FF0FF3303EBC30309EBA9
:10CB50008309D8F80810D9F888311A6861F30602F9
:10CB60001A60236843F00203236023680120034313
:10CB700023606B6C43F400436B642B6803432B60AE
:10CB80005BE605F13C02A7E705F13802A4E705F1F1
:10CB90003402A1E74FF0000CC5F840C0CDE9010216
:10CBA00006220393CDF810E0CDF800C011462846C8
:10CBB0005EF018FB2B6843F080032B60EB6943F4B5
:10CBC0000063EB6114E74FF0000CC5F83CC0042192
:10CBD000CDE901020393CDF810E0CDF800C00622A4
:10CBE00028465EF0FFFA2B6843F080032B60EB6968
:10CBF00043F00803EB61FBE64FF0000CC5F838C0CA
:10CC00000221CDE901020393CDF810E0CDF800C078
:10CC1000062228465EF0E6FA2B6843F080032B607C
:10CC2000AB6943F40063AB61E2E64FF0000CC5F87A
:10CC300034C06146CDE901020393CDF810E0CDF890
:10CC400000C0062228465EF0CDFA2B6843F0800330
:10CC50002B60AB6943F00803AB61C9E64FF0FF31CD
:10CC600053E600204FF0010E034678E607990122B3
:10CC7000284657F02BFDD3E60023C2E600EBC300A5
:10CC800090F8AC0C27E6D8B2F8E6DBB2013B5CE7E3
:10CC9000DBB2013BD2E605F1340202EB83021BE773
:10CCA0003CCB002010B40C49D1F81C3C1A6822F08F
:10CCB00001021A60D1F8182C40F22A4400205C606E
:10CCC0005062116841F0010111601A6842F00102DE
:10CCD0001A605DF8044B7047903C002030B40B4A5A
:10CCE0000B4B82B0CA25532402EB800200205D6208
:10CCF0005C62019001925D625C620198FF220160BA
:10CD00005A625A6202B030BC704700BF50280040DF
:10CD100000280040F0B50E4664493468D1F8F010A0
:10CD2000B1FBF2F1013B9BB2013987B0E362A16232
:10CD30006369BDF830C09DF8342043F0010363619E
:10CD4000236823F440732360236823F07003236077
:10CD50007579B37907460AB183F0010313F0020233
:10CD600003F001010DD1084601231146013D6D007C
:10CD7000EDB2072D09D8DFE805F01A084B085D0869
:10CD80006F81002001220346F0E704920022CDE9E2
:10CD9000010100922946039306222046043D5EF0DD
:10CDA00021FA032D13D8DFE805F052126476C4F897
:10CDB00034C0CDE9021300210492019000910622B3
:10CDC00020465EF00FFAA36943F00803A361636C89
:10CDD00043F400436364236843F0010323607379E1
:10CDE000013B032B5CD8DFE803F0100D0A0204F1CD
:10CDF00040030022C7E900341A6007B0F0BD04F117
:10CE00003C03F6E704F13803F3E704F13403F0E7F9
:10CE1000C4F838C004920022CDE9021301900092B8
:10CE20000221062220465EF0DDF9A36943F4006387
:10CE3000A361CCE7C4F83CC004920022CDE9021300
:10CE4000019000920421062220465EF0CBF9E369AE
:10CE500043F00803E361BAE7C4F840C0049200223B
:10CE600000920622CDE902130190114620465EF0A1
:10CE7000B9F9E36943F40063E361A8E7C4F874C057
:10CE800004920022CDE902130190009207210622AC
:10CE900020465EF0A7F9236F43F00803236796E767
:10CEA00004F1340202EB8303A3E700BF000000207B
:10CEB0002DE9F0478368046C93F8059093F8068099
:10CEC0001E68054686B0204656F03CFD09F1FF3A43
:10CED000002385F82C305FFA8AF35F00FFB208F078
:10CEE0000208072F0DD8DFE817F0F9000C00020147
:10CEF0000C000B010C0008001401F26922F400621E
:10CF0000F261B8F1000F14D0022B28D84FEA49097A
:10CF100009F1FF395FFA89F800224146304657F09F
:10CF2000D5FBBAF1030F00F20381DFE80AF0A59EFA
:10CF3000951DA9F10203022BEED84FEA49010239EF
:10CF4000424601F0FE013046A9F1030957F0BEFB4D
:10CF5000B9F1010F00F28780DFE809F07C044FF09F
:10CF60000008D9E74FF00608F36923F44073F36132
:10CF70004FF0060995F83B30049395F83A30039347
:10CF800095F83930029395F83830019395F8373099
:10CF9000009395F8363095F83520394630465EF0E6
:10CFA00021F9B9F1040F00F0BD80B9F1060F00F0CE
:10CFB000BC800023B36341460122304657F086FB14
:10CFC000072F09D8DFE807F0850880087B0804767A
:10CFD000F36943F40063F36123684BF6EF711022A9
:10CFE0000B402A842360236813432360236895F849
:10CFF000292062F30D332360236895F8272062F31C
:10D000008B232360236895F8262062F3092323608D
:10D01000236895F8252062F3C7132360236895F8E9
:10D02000242062F386132360236895F8282062F396
:10D030004513236063686A8C62F30F036360D5E96C
:10D040000623A260E360236843F00203236006B076
:10D05000BDE8F0874FF00408F36923F00303F361A0
:10D060004FF0040986E74FF00208B36923F44073D8
:10D07000B3614FF002097DE7B36923F00303B361A5
:10D0800095F83B30049395F83A30039395F839308E
:10D09000029395F83830019395F83730009395F85E
:10D0A000363095F83520002130465EF09BF800239D
:10D0B000736380E7336F43F0080333678CE7F369EA
:10D0C00043F00803F36187E7B36943F40063B36196
:10D0D00082E7B36943F00803B3617DE7B26922F0E8
:10D0E0000802B261B8F1000F3FF423AF0CE7B26958
:10D0F00022F40062B261B8F1000F3FF41AAF03E707
:10D10000F26922F00802F261B8F1000F3FF411AFAA
:10D11000FAE6326F22F008023267B8F1000F3FF4EE
:10D1200008AFF1E60023F36345E70023336442E7E9
:10D1300095F83B30049395F83A30039395F83930DD
:10D14000029395F83830019395F83730009395F8AD
:10D15000363095F83520394630465EF043F8A6E77C
:10D160002DE9F04FA84D95F88C3287B01BB90120FE
:10D1700007B0BDE8F08F2C68FCF7A6FCA34B93F832
:10D1800050150491002900F0378103F56A68A04B1F
:10D19000A04FA3FB04235B09A7FB0327FF089E4ABC
:10D1A00007EB8707A3EB4707D2F8C43105F24464C5
:10D1B000A0EB030BFBB2039308EB870702F188098E
:10D1C00000268A460594019410E0019C2046FFF752
:10D1D0006FFE013623464C335645019308F15C0837
:10D1E00007F15C0709F1140900F0BB80BBF1000FE7
:10D1F00004DB019B1B6B5B4500F3EA80824A4C23F6
:10D2000003FB062393F87036002BDED00198836869
:10D2100081891A68036C5C68D368A4B2C4F11604EF
:10D2200023EA0103072CD360CFD97B4A856CD2F85F
:10D23000903002960133C2F8903000222868AE4642
:10D240009446012115E0BCF1140F1EDC13F1080611
:10D2500048BF03F1170633110CEB261C5E1E02FAC1
:10D2600003F30122114402FA06F68C4246EA030255
:10D270000BD303465EF8040FA142A0EB0303E2D3F5
:10D28000CCF115034FF0150CE8E7BCF1150F029E29
:10D290005DD1624CC2F3842304EB830302F01F00D0
:10D2A00053F8E01CC2F3441304EB830304EB800047
:10D2B00053F8E03CC2F3C432090204EB820241EAB3
:10D2C000031150F8E03C52F8E02C0B4343EA0233E0
:10D2D00083EA132282EA121202F00F020F2A36D1D9
:10D2E000C3F30F134FF6FF72934230D0B3F5606F64
:10D2F00072D0A9F80C3098F858200398824210D0C8
:10D30000B968D8F80020521AC8F80020396BD8F84C
:10D310000420521AC8F804200022BA603A6388F840
:10D320005800D8F800200132C8F80020BA6801324D
:10D33000BA604FF6FF7293427FF447AFD8F80430DB
:10D340000133C8F804303B6B01333B633DE7324A9D
:10D35000D2F88C300133C2F88C309EB34FF6FF7395
:10D36000C9E72D4A059C049F0026012382F88C31D1
:10D37000C2F8C46103250FE05B00BCF1020F03F1AA
:10D38000FF331DD900210122013657F09FF9B74222
:10D3900004F14C043FF4EBAEA3681868426865F3EF
:10D3A00006124260217C5B7911F0020103F1FF3C1F
:10D3B000A3F10202E0D15B00022AA3F10203E2D84A
:10D3C000D9B2E0E729465822154862F02BFAC5E7A2
:10D3D000002007B0BDE8F08F0B4991F8A52802EBBB
:10D3E000420201EBC202324492F8B5280D2A80D1E4
:10D3F000802289F81E207EE7074B012283F88C21CA
:10D40000049AC3F8C421B2E6A01A0020982B002089
:10D410001F85EB51CDCCCCCC903C0020440E0708AE
:10D42000C43D00202DE9F047884600294AD046181F
:10D43000DFF89890DFF898A0451E013E8024EFF3B6
:10D44000118184F31288D9F84435D9F84805D9F800
:10D450004425D9F848C5C9B281F31188624512E064
:10D460000120FCF7F7FFEFF3118184F31288D9F85C
:10D470004435D9F84805D9F84425D9F84875C9B2D2
:10D4800081F31188BA428CBF002201221B1A03EBE0
:10D49000C223012BE4D0EFF3118284F31288D9F870
:10D4A000483515F8011F5344D2B283F8281CD9F827
:10D4B00048350133C3F30A03C9F8483582F31188AC
:10D4C000B542BCD14046BDE8F08700BF982B002094
:10D4D000903C0020F8B50C4E96F8483F032B00D046
:10D4E000F8BD37680D46144608E0FFF79BFF336828
:10D4F000DB1B322BA4EB00040544F1D8002C2146A1
:10D500002846F2DCF8BD00BFA01A0020344BD3F847
:10D51000683C596A91F85230012B56D170B5314CA4
:10D52000314AD4F8300360BBD2F84405D2F848350C
:10D53000984221D0D2F84405D2F84835984249D8CB
:10D54000D2F84835D2F844051B1AD2F8442591F890
:10D55000520088B1B3F5007F28BF4FF400731D4619
:10D56000002381F85230214921480A44ABB281217D
:10D5700057F0B0F9C4F830531E4B6FF001021A6136
:10D5800070BDD2F8445500F03F032844C2F844056A
:10D59000D2F84405B0F5006F04BF0020C2F844057E
:10D5A0000020C4F83003002BBED1D2F8442591F8F6
:10D5B00052000028E4D00D4881F852300244BDE802
:10D5C00070400B48812157F085B90A4B6FF001027A
:10D5D0001A617047D2F84435C3F50063B5E700BF60
:10D5E000A01A0020884D0020982B0020B848002069
:10D5F00004270020004C01402DE9F04FA94DD5F83B
:10D60000608CD8F81460D8F81820D8F81430DB07EC
:10D6100085B026D41640B70744BF0223C8F814309B
:10D62000740300F19880300300F12A81F20400F1C4
:10D630005F81310708D5D5F8683CDB690BB19A48A2
:10D6400098470823C8F81430B2040DD4F30640D428
:10D65000F70257D4B40262D4002EC0F2BB81300569
:10D660006BD405B0BDE8F08FD5F8644C8F49D4F881
:10D6700000396FF30A03C4F80039D4F8043823F4EE
:10D680008073C4F80438E368052262F38D23E360F5
:10D690004FF0400901272046C5F8D89DA5F8D27D56
:10D6A00057F040F800238249A5F8723C2046C5F89F
:10D6B000789C57F037F8D5F8683C85F8487F5B6868
:10D6C0000BB1794898474FF40053C8F81430F3066B
:10D6D000BED5D5F8643C9A6922F010029A611A6AA4
:10D6E000C2F343410229C2F30A1702F00F0200F00D
:10D6F0004582062900F0CA839A69F70242F01002B7
:10D700009A61A7D5D5F8683C1B6A13B16648052114
:10D7100098474FF48013B402C8F814309CD5D5F85C
:10D72000683C1B6A13B16048062198474FF4001308
:10D73000002EC8F8143092DA4CE1D5F8643CD3F8E6
:10D740000828D10700F13E824FF40063C8F8143076
:10D7500005B0BDE8F08FD5F8643CD3F81878D3F85D
:10D760001C281740BFB203F50061002F3FF45BAFE8
:10D770004FF0000ACDE901864E4C03F5106B56467A
:10D78000884608E07F0806F1010604F12C040BF13D
:10D79000200B00F04081F907F4D5D8F81020D8F814
:10D7A000343023FA06F94FEAC919DBF808305FFA7A
:10D7B00089F949EA020909EA030919F0010F40F061
:10D7C0003E8119F0080F1CBF0823CBF8083019F070
:10D7D000100F1CBF1023CBF8083019F0400F1CBFEE
:10D7E0004023CBF8083019F0020F1CBF0223CBF8FE
:10D7F000083019F0800FC5D0D5F8649CA26AE36A9E
:10D80000A16909F5106A0AEB461AA2EB030E8E45D0
:10D81000DAF8180028BF8E4680B20EF10301B0EB93
:10D82000910F40F2FF8009F5805C0CEB063C0396FB
:10D8300011468B4280F0F580A269C91A914228BF37
:10D84000114688B20330CE1C8010626A8E464FEAC1
:10D85000960609D00023013352F8041BCCF80010BF
:10D860009842F8D1626AE36A72446262DAF8182078
:10D8700092B273449642E36280F0D380A16AD8E703
:10D88000D5F8647CD7F81848D7F81C381C40240C0D
:10D8900007F5006C3FF4CAAE07F530674FF000099A
:10D8A000E34610E0A01A0020042700207028002082
:10D8B0001027002000270020640809F1010907F162
:10D8C00020073FF4B3AEE307F6D5BA68DBF81430AF
:10D8D00002EA030A1AF0010F40F011811AF0080F52
:10D8E00040F0D5801AF0100F1CBF1023BB60E3E797
:10D8F000D5F8644CD4F8043823F00103C4F8043894
:10D900005BF0B0F82269C14B102161F38A122261E9
:10D91000226942F0200204F50067226101E0013B28
:10D9200002D022699006FAD404F5106304F5206150
:10D93000FF229A60C3F8082220338B42F9D14FF0BE
:10D94000FF33BB614FF00113FB617B6943F00103BF
:10D950007B617B6943F002037B617B6943F00803D1
:10D960007B613B6943F001033B613B6943F0020388
:10D970003B613B6943F008033B61D4F8003823F472
:10D98000FE63C4F800380023C4F8103BD4F8103B01
:10D99000012161F3DC43C4F8103BD4F8103B18229A
:10D9A00062F31203C4F8103BD4F8103B43F0C043B9
:10D9B000C4F8103BD5F8683C85F8481F1B6A0BB1CA
:10D9C000934898474FF480533107C8F814307FF5D7
:10D9D0003BAE30E6D5F8643CD3F8042822F00102CF
:10D9E000C3F80428D3F8002E22F00102C3F8002E59
:10D9F00095F8492FD5F8683C85F8482F1B6A13B174
:10DA00008348032198474FF000433005C8F814308D
:10DA10007FF527AE91E6DDE9018630037FF506AE9E
:10DA20002EE7039EBEF1000F7FF4ACAED9F8343878
:10DA30000122B24023EA0203C9F83438A2E6D8F83A
:10DA40003430012202FA06F123EA0103C8F8343027
:10DA5000CBF80820002E72D195F8443F022B7FF4BA
:10DA6000B0AED5F8941CD5F8783C994240F250827B
:10DA7000C91A8B42C5F8941C88BF8BB2D5F8842C88
:10DA8000634898BF9BB2002156F024FF99E6082313
:10DA9000BB60B5F8382FB5F83E3FD5F83A1FA5F86A
:10DAA000302F02F01F0C0120BCF1010F85F8440F4C
:10DAB000A5F8363FB5F83C0FA5F8463FC5F8321F2C
:10DAC0005FFA82FE00F0C481BCF1020FC2F30722AC
:10DAD00000F07B81BCF1000F00F0898095F84A3F8F
:10DAE000002B3FF4FFAED5F8642CD2F800180020CC
:10DAF00063F30A11C2F8001885F84A0FF2E6012311
:10DB0000BB60B9F1000F29D195F8443F032B7FF496
:10DB1000E5AED5F8F41DD5F8D83D994240F2CF8155
:10DB2000C91A8B42C5F8F41D88BF8BB2D5F8E42D15
:10DB3000374898BF9BB2002156F0BAFFCEE6D5F821
:10DB4000683C5B69002B3FF43CAE95F8482F032AF4
:10DB50007FF437AEF1B22E48984732E6D5F8683CEC
:10DB60009B69002B3FF4BAAE95F8482F032A7FF447
:10DB7000B5AE5FFA89F126489847AFE6002F3FF42B
:10DB8000BBAD2C2101FB025107F1030CD1F8E49D40
:10DB90004FEAAC0C03F5805E484600210131DEF807
:10DBA000004040F8044B6145F8D12C2101FB0252A2
:10DBB00009EB0700D2F8EC1DC2F8E40D3944C2F8B5
:10DBC000EC1D99E595F8482F85F8492F042285F832
:10DBD000482FD3F80828D2071CD4D5F8683C1B6A14
:10DBE000002B3FF4B1AD022109489847ACE51EF087
:10DBF000600F40F0778189B2092A12D8DFE802F07D
:10DC00005D3B11BC11D29211791500BF420D03008A
:10DC100004270020D3F8002E42F00102C3F8002EA2
:10DC2000DBE7B44856F018FE58E7CAB2B2490343DE
:10DC300081F834230193F4D195F8483F022B00F08A
:10DC4000F481032BEDD1002A40F0D881D5F8683C4F
:10DC500085F84D2F022185F8481F5B68A548019281
:10DC60009847019AA348042385F8443F1146134678
:10DC700056F030FE32E795F8483F023B012BD0D8F2
:10DC800001297FF42BAFD5F8503FD5F8682C9B497C
:10DC900023F00203C5F8503F002385F84B3F9268FC
:10DCA000A1F533709047042285F8442F0023914852
:10DCB0001A46194656F00EFE10E795F8483F023B0B
:10DCC000012BAED895F84B3F2BB1D5F8503F43F020
:10DCD0000203C5F8503F8A4A02230021A2F53B7097
:10DCE000C5F8983CC5F8943C85F8443F56F0F2FDE1
:10DCF000F4E6012B95D195F8482F022A00F0C9814E
:10DD0000032A8ED17F4AC5F8983C02216FF43A7CF1
:10DD100085F8441F02EB0C000021C5F8943C56F036
:10DD2000D9FDDBE60B0A022B00F0E281032B00F0A9
:10DD3000D681012B7FF475AFD5F86C3C1B689847F2
:10DD400000283FF4CBAE0388002B3FF4C7AEB5F8F4
:10DD5000361F00293FF4C2AE8B4228BF0B4602217A
:10DD6000426885F8441F6348C5F8983C0021C5F80F
:10DD7000943C56F0AFFDB1E601297FF4AFAE85F8D3
:10DD80004B1FD5F8683C5D499B68A1F533709847F7
:10DD90000023042285F8442F56481A46194656F0A7
:10DDA00099FD9BE603437FF43CAF95F8482F032A87
:10DDB00001F07F013FF435AF00290CBF01220222A0
:10DDC00085F84A1F85F8482FE3E70EF0600E0B0C2C
:10DDD000BEF1200F0193C1F307430AD1D5F8682C97
:10DDE000464992680293A1F53370904795F8312F18
:10DDF000029B012A00F0CC80032A00F0AC80002AAC
:10DE00007FF40FAF95F8482F022A00F09C80032A78
:10DE10007FF407AF019A100600F1E8803A4A2C21FE
:10DE200001FB032202F5B872537B3248A3F10103D0
:10DE3000B3FA83F35B0942F8103F00210223C5F8CF
:10DE4000983CC5F8943C85F8443F56F043FD45E6C0
:10DE500095F8483F032B7FF4E4AE264BD5F8682CA9
:10DE60000193926803F5337118469047B5F8362F41
:10DE7000019B002A7FF432AE18460422002385F865
:10DE8000442F19461A4656F025FD27E607F1030CE4
:10DE90005FEAAC0C0AD01D4803F5805E0021013119
:10DEA000DEF8004040F8044B8C45F8D12C2101FBF2
:10DEB0000252D2F8EC1D3944C2F8EC1D1CE4D5F82E
:10DEC000683C1A690B4B1AB1184601939047019BA5
:10DED00018460422002385F8442F19461A4656F0A6
:10DEE000F9FCFBE4D5F8683C04499B68A1F5337064
:10DEF0009847F3E504270020884D0020D029002012
:10DF0000F0290020ED29002000270020D82900203A
:10DF1000D5F8902C93424CD0D5F8683CDB68002BA8
:10DF20005FD095F8482FDFF810A2032A01D15046A0
:10DF300098470023052285F8442F50461A46194673
:10DF400056F0B6FD3DE459063FF4C8AD7A4819468F
:10DF500056F052FCC2E595F8482F022AF3D0032A66
:10DF60007FF45FAEB5F8322F002A3DD15A063BD080
:10DF70001946714B0193184656F03EFC019BD5F8AB
:10DF8000682C0193184692686C499047019B73E78F
:10DF900095F8482F022AD6D0032A7FF442AEB5F86E
:10DFA000322F002A7FF49AAD13F07F0047D1624BE5
:10DFB00062E7D5F8982C9342AED8B5F8463F9A421E
:10DFC000AAD23346324631465B48C5F8906C56F0CB
:10DFD00081FC594833463246314656F069FDFFF719
:10DFE000F0BBDFF854A1A4E7534BC8E7544A03F051
:10DFF0007F032C2101FB0322103215E795F84D3FDA
:10E000009342D4D1D5F8683C4B485B6898474D495A
:10E0100091F8343385F84D3FD5F8683C1B68464885
:10E020009847042385F8443F40E6002ABFD085F88E
:10E030004D2F0322D5F8683C85F8482FEEE701996B
:10E04000D5F8642C11F0800F3D4943D12C2000FB02
:10E05000031101F5B871887850BB02F510630A7896
:10E0600003EB4213CA78D3F800C0023A60F3555C60
:10E07000012AC3F800C028D92F4BD5F8682C01938A
:10E0800000204873926803F5337118469047019B4E
:10E09000F2E685F8442F2C4AC5F8983C0021A2F5F9
:10E0A0003A70C5F8943C85F84C1F56F013FC15E502
:10E0B00002F530630A7803EB42131A6822F4001267
:10E0C0001A60CA78023A012AD6D81A6842F08052F9
:10E0D0001A60D1E72C2303FB00111031BBE7C9B252
:10E0E00005293FF6FFAEDFE801F0211C17120D08ED
:10E0F000D5F86C3C9B68984722E6D5F86C3C1B6AC7
:10E1000098471DE6D5F86C3C5B6A984718E6D5F849
:10E110006C3CDB69984713E6D5F86C3C9B699847E3
:10E120000EE6D5F86C3C5B69984709E6D5F86C3C7F
:10E130001B69984704E600BF04270020D02900206F
:10E1400000270020884D0020EC290020BFF34F8FCE
:10E150000549064BCA6802F4E0621343CB60BFF383
:10E160004F8F00BFFDE700BF00ED00E00400FA059F
:10E1700008B500210320FEF7B1FD72B6FFF7E6FFF8
:10E18000154C08B5D4F8383394F83E03ABB91420D5
:10E19000FCF760F900BFD4F838335BB11A689B888C
:10E1A000116994F83E230B4012B91BB1FFF7E0FF51
:10E1B000002BFBD0FAF72CFBECE719689A880B6967
:10E1C000134020B1002BE2D10B691340FAE7002B7A
:10E1D000DDD00B691340FAE7884D002008B572B610
:10E1E000FFF7B4FFF0B5AA4BB3F5C07F85B000F0E0
:10E1F000A78100F23381B3F5807F00F0A781B3F5EA
:10E20000A07F00F0A181802B14BF05240624A14B20
:10E210001B8A03F00703A34240F09A819E4855F001
:10E2200083FB9E499E4B0A689E4842F480720A60B6
:10E23000FF24CA2153225C6259625A62D0F87438B2
:10E24000DB0000F11481984A954B984FCA2553245E
:10E250000020FF215D625C62029002925D625C625E
:10E26000029E0432BA42306059625962F2D190493A
:10E270000020FEF733FD8F4B002103910393039B96
:10E280001B680093009B012B00F02E81824855F003
:10E290004BFB824A884B1169012060F30201116136
:10E2A000196E02F5E43260F3010119661368034345
:10E2B000136013689F07FCD59368804923F003031C
:10E2C00093608B6813F00C0FC3F38102F9D10B68D4
:10E2D0007B4C23F0867323F480334FF41F000B60D4
:10E2E0008A604C60C1F8A020C8600B686D4A43F496
:10E2F00080330B60D2F800389E0307D44FF44053AC
:10E30000D2F800188D0301D4013BF9D1D2F80038BE
:10E310009C03EFD56949634A0B6843F001030B6026
:10E32000D2F800389807FBD5644B5A6842F4800253
:10E330005A605A68482161F38E125A605968594AE6
:10E34000012060F303015960596860F3124159607C
:10E35000196841F080711960D2F800389901FBD535
:10E36000564A936823F0F00393609368042161F3A5
:10E370004F339360936861F38C239360D2F8A43099
:10E3800043F03003C2F8A4309368022060F3010325
:10E3900093609368C3F38103022BFAD1D2F8A430BF
:10E3A00023F03003C2F8A430D2F8A4300B2161F37B
:10E3B0000F33C2F8A430D2F8A03023F40053C2F8CF
:10E3C000A030936813F00C0FC3F3810100F0968026
:10E3D000022900F0A1803B4A38493B488B683B4CFE
:10E3E0003B4DC3F303131844E36810F8600CC240BC
:10E3F0004FF6FF00034043F0052343F47A03E36044
:10E40000344B486FC3F840032648334BA360D0F821
:10E41000343823F00043C0F834384B6F2F4843F0B2
:10E4200080734B67C5F8F02055F07EFAFAF706FCCA
:10E430002B4AD5F8F030A2FB03239B09013BB3F133
:10E44000807F09D24FF0E022F020536100210723A2
:10E4500084F823009161136105B0F0BDB3F5E07F4E
:10E4600070D0B3F5007F14BF05240024CFE61D4B08
:10E47000002201920193019A03F11973126803F5C6
:10E480009E3303F2E1139A427FF4DDAEF3E600BF60
:10E49000C000000000C0FF1F1C00400000700040D2
:10E4A0000028004000300240542800406C28004002
:10E4B000316665425C280040003C02400038024062
:10E4C0000230030000127A00440E070800ED00E05D
:10E4D00000000020884D0020000000081F003000D0
:10E4E000D34D6210502800400320FEF7F7FB3F4B4E
:10E4F0001A6882F308885B689847FEE7D2F8A03074
:10E500005B047FF568AFD2F8A010394B394A11F49B
:10E51000805F08BF1A465FE75368536851685068C8
:10E52000354D334CC0F30240C3F388122B5C01F02D
:10E530000F0104FB02F213FB01F3B2FBF3F24BE712
:10E54000022464E6012462E6032460E604245EE615
:10E550002A4D2B4A2B4B6A606B606A646B64E969D5
:10E56000AA6011F0020F14BF0026A526AB602B692C
:10E570009905FCD52B6943F020032B612B6943F0EF
:10E5800040032B614FF0004055F04AFC2B690328F3
:10E5900023F020032B6117D0184D194A194BAA609C
:10E5A000AB602B699A05FCD52B69174A43F0100321
:10E5B0002B614FF48010148255F032FC2B6923F04C
:10E5C00010032B61FFF70AFEA52EE5D12B690E4A39
:10E5D00043F010032B614FF48010168055F020FC9F
:10E5E0002B6923F010032B61D6E700BF0000FF1F4B
:10E5F00000127A00006CDC02189E0708003C024002
:10E6000023016745AB89EFCD00C0FF1F01490248D8
:10E61000FAF786BD6C2400200000014002494FF04B
:10E620008040FAF77DBD00BF9824002001490248D0
:10E63000FAF776BDC42400200004004001490248D6
:10E64000FAF76EBDF024002000080040014902489E
:10E65000FAF766BD1C250020000C00400149024865
:10E66000FAF75EBD4825002000100040014902482D
:10E67000FAF756BD742500200014004001490248F5
:10E68000FAF74EBDA02500200004014001490248D0
:10E69000FAF746BDCC2500200040014010B5064CDD
:10E6A000064804F6CC11FAF73BFD04F6583104484D
:10E6B000BDE81040FAF734BDA01A00200000014068
:10E6C0000044014001490248FAF72ABD24260020EF
:10E6D0000048014001490248FAF722BD50260020B7
:10E6E0000018004001490248FAF71ABD7C260020B4
:10E6F000001C004001490248FAF712BDA82600207C
:10E700000020004001490248FAF70ABDD426002043
:10E71000004C0140EFF31183502282F3128802680B
:10E7200022F00102DBB2026083F31188704700BF60
:10E7300070B5002486B0CDE90144CDE903440DF164
:10E74000040CC0E92944C0E92B44C0F8B440054694
:10E7500000F1B80EBCE80F00AEE80F00CEF80040A4
:10E7600095F8D130059444F23B36A5F8FC600BB91E
:10E7700006B070BD1C09013C072C03F00F0330D814
:10E780001E4E36F8140040FA03F2D20729D50122B2
:10E7900002FA03F3013B1840264461F02FF996F882
:10E7A000C03D174A034402EBC30452F83320A38848
:10E7B00012691340DCD12946124A2620E08041F834
:10E7C0000C2F20461A465AF067FB0F49A2880868AA
:10E7D000B2FA82F24FF00043D34003430B6006B01D
:10E7E00070BD2946074B41F80C3F00231A461846D6
:10E7F00006B0BDE870405AF04FBB00BF4CFD0608A4
:10E80000AC1A002069AC0008003C0140264A92F88E
:10E8100047367BB3D2F84816884235D0012B29D031
:10E82000D2F85016814233D0022B23D0D2F858169A
:10E8300088422FD0032B1DD0D2F8601688422BD0EF
:10E84000042B17D0D2F86816884227D0052B11D098
:10E85000D2F87016884223D0062B0BD0D2F8781647
:10E8600088421FD0072B05D0D2F88016814208BFFE
:10E8700007230AD002EBC30103F1010CC1F84806DB
:10E8800082F847C6184670470023DBB21846704727
:10E890000123FAE70223F8E70323F6E70423F4E76A
:10E8A0000523F2E70623F0E7982B002010B4037F3E
:10E8B000083300EB43035B88047F9BB214B984697F
:10E8C000022C4BD0FF2B046837D80382037F012B27
:10E8D00015D08369032B22D08369022B1FD0038AB2
:10E8E0006068DBB242EA03431F4A194300EA0203AD
:10E8F000194341F0007161605DF8044B7047836912
:10E90000022BE6D1038A6068DBB242EA0343164A6F
:10E910000B430240134343F080736360ECE741EA2A
:10E920000203028A616810480140D2B20B4343EAF5
:10E93000024363605DF8044B7047FF230382038A40
:10E940000948DBB242EA03426368114303401943BA
:10E9500041F0807161605DF8044B7047448A838A9E
:10E9600023449BB2AEE700BF009800FC2DE9F04FB6
:10E9700083B08DF80730431C00F08D8003280446D7
:10E9800000F38980BF4D542303FB00531646D3F890
:10E99000EC21002A7FD000200127C3F8040283F86D
:10E9A00008720DF10707C3F8F8710227A3F8007287
:10E9B00083F80A0283F80A0242F21173906907048D
:10E9C00015D4542303FB045393F80A32DFB2DFB1AA
:10E9D000542303FB0453012283F80A2293F80A32DA
:10E9E000DBB2002B3BD1012003B0BDE8F08F013B2F
:10E9F000E4D1542303FB0453122283F80A2293F830
:10EA00000A32DFB2002FE3D19F4B4FF0540909FBCC
:10EA100004F909EB030B4FEA4108A94441464FF4BE
:10EA200000525846FFF742FFD9F8EC1189F80A72F4
:10EA300042F211738A6990072FD5542303FB0453C4
:10EA400093F80A925FFA89F3A3B3542303FB0453A8
:10EA5000022283F80A2293F80A32DBB2C1E7542378
:10EA600003FB04530022D3F8EC1183F80A2240F68A
:10EA700071038A69920640F1B980542303FB04555F
:10EA800095F80A32814A2023CB61B2F8443301332E
:10EA90009BB2A2F844330020A6E7013BCAD154231D
:10EAA00003FB0453122283F80A2293F80A925FFAB6
:10EAB00089F3C9E78E62542606FB045696F80A22AB
:10EAC000002A40F09F80B6F8FC21013A92B2A6F8E5
:10EAD000FC2196F808224FF02A0A0AFB04FA524455
:10EAE000143205EB4202B2F8D611013989B2A2F80C
:10EAF000D61196F808225244143205EB4202B2F8BD
:10EB0000D62192B2002A52D0994606F20A27122341
:10EB1000D6F8EC0187F8009042F2117281698907FA
:10EB200077D53A78D2B2002A40F0A18096F808C290
:10EB300004EB4401C1EBC1016144083105EB8101E3
:10EB4000D1F8D4C10CF1010EC1F8D4E19CF8001049
:10EB50008162B6F8FC11013989B2A6F8FC1196F869
:10EB600008125144143105EB4101B1F8D6C10CF142
:10EB7000FF3C1FFA8CFCA1F8D6C1B6F8FC1189B293
:10EB800051B996F808125144143105EB4101B1F81E
:10EB9000D61189B200294ED196F808225244143277
:10EBA00005EB4202B2F8D62192B2002AB0D154232A
:10EBB00003FB04530022D3F8EC1183F80A2242F23B
:10EBC00011738A6990062AD5542303FB045393F8E2
:10EBD0000A32DBB2002B5BD0542303FB0453062222
:10EBE00083F80A2293F80A32DBB2FAE6013B7FF49B
:10EBF00040AF542303FB0453122283F80A2293F8F4
:10EC00000A323FE7032386F80A3296F80A32DBB26B
:10EC1000E7E6013A82D13B703A78D2B283E7013B12
:10EC2000CFD1542303FB0453122283F80A2293F812
:10EC30000A32DBB2CEE73A7042F2117281690B06FA
:10EC400009D53A78D2B2002A3FD141465846FFF75B
:10EC50002DFE1223A0E7013AF0D1542202FB045208
:10EC6000122182F80A1292F80A22D2B2EBE7542358
:10EC700003FB0453042283F80A2293F80A32DBB21E
:10EC8000AFE600BF903C00207C3E0020884D002075
:10EC90002022CA614A6863F309024A604A6863F342
:10ECA0000C324A604A6863F317424A604A6863F369
:10ECB00018624A604A6863F38A22542303FB0453B0
:10ECC0004A6093F80A32DBB28BE6542303FB045309
:10ECD000052283F80A2293F80A32DBB281E600BFEC
:10ECE000B0F1FF3F00F0D2802DE9F04F032883B050
:10ECF00004467EDCBD4D542606FB0056D6F8EC01DA
:10ED0000002876D00C9FC6F8F8710127C6F8047267
:10ED100086F80872A6F80032002386F80A3286F8D0
:10ED20000A3240F671038669360415D4542303FB76
:10ED3000045393F80A32DBB2DBB1542303FB0453D0
:10ED4000012283F80A2293F80A32DBB2002B35D174
:10ED5000012003B0BDE8F08F013BE4D1542303FB55
:10ED60000453122683F80A6293F80A32DBB2002BAE
:10ED7000E3D146689E4F3E4046EA410646F490364F
:10ED80004660542606FB04564FEA410A86F80A32CA
:10ED900040F671038669B7072DD5542303FB04534E
:10EDA00093F80A32DBB293B3542303FB04530222D9
:10EDB00083F80A2293F80A32DBB2C7E7542303FB35
:10EDC00004530022D3F8EC1183F80A2240F67103B1
:10EDD0008A69920629D5542303FB045595F80A3213
:10EDE000844A2023CB61B2F8443301339BB2A2F8AA
:10EDF00044330020ADE7013BCCD1542303FB045343
:10EE0000122683F80A6293F80A32DBB2CBE78262F9
:10EE1000542202FB045292F80A628EB1032382F854
:10EE20000A3292F80A32DBB290E7013BD0D1542388
:10EE300003FB0453122283F80A2293F80A32CFE725
:10EE400082F80A3240F671038269560611D55423BE
:10EE500003FB045393F80A825FFA88F6C6B1542381
:10EE600003FB0453042283F80A2293F80A32DBB22C
:10EE70006CE7013BE8D1542303FB0453122283F8CF
:10EE80000A2293F80A825FFA88F6E7E700207047C3
:10EE9000594B542704FB07F7FB182F4418464FF42F
:10EEA0001052514601934FF02A09FFF7FFFC97F8E3
:10EEB000083209FB04F94B44143305EB4303B3F860
:10EEC000D6319BB2002B4DD004EB440BB046CBEBBC
:10EED000CB0B07F20A26D7F8EC0186F8008040F643
:10EEE0007103826951075CD53378DBB20BB105231E
:10EEF000337097F80832426A5B44083305EB8303AA
:10EF0000D3F8D401411CC3F8D411027097F8083229
:10EF10004B44143305EB4303B3F8D621013A92B2C4
:10EF2000A3F8D621B7F8FC31013B9BB2A7F8FC311E
:10EF3000B7F8FC319BB253B997F808224A4414320F
:10EF400005EB4202B2F8D62192B2002A3CD197F8E2
:10EF500008324B44143305EB4303B3F8D6319BB26C
:10EF6000002BB8D1542303FB04530022D3F8EC1137
:10EF700083F80A2240F671038A69900618D5542353
:10EF800003FB045393F80A32DBB2002B3DD0542329
:10EF900003FB0453072283F80A2293F80A32DBB2F8
:10EFA000D4E6013B9DD1122333703378DBB29DE769
:10EFB000013BE1D1542303FB0453122283F80A22BC
:10EFC00093F80A32DBB2E0E7D7F8EC01337040F691
:10EFD00071038269120611D53278D2B2002A31D17A
:10EFE00001985146FFF762FCB1E700BF903C00205A
:10EFF000009800FC884D00207C3E0020013BE8D1B9
:10F00000122333703278D2B2E8E72022CA614A680C
:10F0100063F309024A604A6863F30C324A604A6843
:10F0200063F317424A604A6863F318624A604A68A9
:10F0300063F38A22542303FB04534A6093F80A3291
:10F04000DBB283E6542303FB0453062283F80A222F
:10F0500093F80A32DBB279E638B58369023B04469D
:10F06000072B0CD8DFE803F048482F2F0C0C0404C2
:10F0700003689A69D20672D51022DA61A37F38BD7F
:10F080000568AA6912F0100253D01023EB612B68B7
:10F0900043F020032B60AB69980744BF0023AB62A9
:10F0A000AB69D90703D4AB6943F00103AB61237F9C
:10F0B000083304EB43035B889BB2002BDED01123A3
:10F0C000A377A37F38BD03689A69D50640F1BA805B
:10F0D000027F083200EB4202528892B2002ACBD162
:10F0E0009969890748BF9A629A69D207C4D49A6914
:10F0F00042F001029A61BFE703689A69D50677D5A5
:10F100001022DA619A69900701D500229A629A6901
:10F11000D20703D49A6942F001029A61237F08332F
:10F1200004EB43035B889BB2002BA7D01123A3778A
:10F13000A4E7AB6913F0800300F0EC802B6823F0A8
:10F1400040032B60037F083300EB43035B889BB2D3
:10F15000002B40F01F810D238377837F38BD9A6990
:10F1600012F0080240F0968099698D0686D520211C
:10F17000D961196821F0FE011960596862F309012B
:10F180005960596862F30C315960596862F317414C
:10F190005960596862F318615960596862F38A21AD
:10F1A00059609969880748BF9A629A69D10703D460
:10F1B0009A6942F001029A619A69520715D5227F35
:10F1C000596A04EB82039A68501C98601170238A74
:10F1D0009BB253B1227F04EB4202538A013B9BB2A4
:10F1E0005382238A013B9BB223820123637745E745
:10F1F0009A69910751D5027F00EB82029168481C01
:10F2000090600A789A62227F04EB4202538A013BA3
:10F210009BB25382238A013B9BB22382237F083314
:10F2200004EB43035B889BB2002B7FF427AF237F63
:10F23000002B7FF423AFA369022B7FF41FAF0123C0
:10F2400023771BE79A69100724D49A69950700F180
:10F25000B0809A6912F0040286D0227F083204EB53
:10F260004202528892B2002A3FF408AF227F596AC4
:10F2700004EB82039A68501C98601170227F04EBA3
:10F280004202538A013B9BB25382238A013B9BB2C9
:10F290002382F3E60822DA61F0E69A6915066BD458
:10F2A0009A695007E2D49A6912F0400240F0A480B3
:10F2B000996989067FF5E2AE2021D961596862F328
:10F2C00009015960596862F30C315960596862F359
:10F2D00017415960596862F318615960596862F3BF
:10F2E0008A2159609A69D00644BF1022DA619A696E
:10F2F000910744BF00229A629A69D20703D49A699F
:10F3000042F001029A611A68012122F0F6021A60A5
:10F310006177B3E6AA6992067FF5B0AE2022EA6172
:10F320006A6863F309026A606A6863F30C326A60B0
:10F330006A6863F317426A606A6863F318626A6016
:10F340006A6863F38A226A60AB69DB0644BF1023F4
:10F35000EB61AB69980744BF0023AB62AB69D90787
:10F3600003D4AB6943F00103AB612B68012223F0A6
:10F37000F6032B60627781E6028A92B23AB9017F86
:10F38000083100EB4101498889B200292ED10D23B3
:10F39000A37773E66968C1F30901FFF787FA238E43
:10F3A000102B2B680CBF43F4804343F400432B60C5
:10F3B00064E6227F083204EB4202528892B2002AAD
:10F3C0003FF45CAE227F04EB82029168481C90609F
:10F3D0000A789A62238A013B9BB22382227F04EB44
:10F3E0004202538A013B9BB2538247E65968C1F3FC
:10F3F0000901FFF75BFA41E6227F083204EB420283
:10F40000528892B26AB9227F12B9A269032A0BD03C
:10F410005A6895013FF532AE5A6842F480425A600C
:10F420002CE60E23A37729E60122227759684FF4B0
:10F430001052C1F309012046FFF738FA1EE600BF5B
:10F44000004809E67C3E0020004805E6D03E00204A
:10F45000004801E6243F002000B5224B224D85B034
:10F46000CA24532100225C625962019201955C62B8
:10F470005962019903240C60FF215962596272B6E6
:10F480001A4BD3E9D21351EA03041DD11046154B90
:10F490001749CA25532400265D625C6202960291D8
:10F4A0005D625C6202990860FF21124859625962EC
:10F4B0005D625C62039603905D625C620398026029
:10F4C00059625962FEF78AFE0B4A12684EF66024B2
:10F4D00004FB00F0521843F10003821843EBE07084
:10F4E000D5E700BF002800405C280040884D002080
:10F4F0006028004064280040A01A0020164A174BDC
:10F500009042D3F8F03028BF1046B0EB930F14D2DE
:10F51000B0EBD30F13D2B0EB131F12D2B0EB531FCB
:10F5200011D2B0EB931F10D2B0EBD31F0FD2B0EBC0
:10F53000132F0ED24FF480707047022070470420C2
:10F5400070470820704710207047202070474020E7
:10F5500070478020704700BF005125020000002046
:10F5600011F001010ED1F0B590F82850C668012DB8
:10F5700083B0044607D0B6F1807F01D90123037719
:10F5800003B0F0BD70470A4B476AD3F85003FFF74A
:10F59000B5FFB6F1807FB880F2D9B7260A46257745
:10F5A0002B46384601A98DF8046050F093FCE7E73C
:10F5B000884D00202DE9F0410546406A94B014467C
:10F5C00000681F460E465BF0C3FE0B94264C0C975A
:10F5D00004F582630093254B0193022300220293DA
:10F5E0000123CDE90922CDE90E22CDE910228DF8C3
:10F5F0000C308DF834308DF8483006922B7F8DF822
:10F60000202013921A4A049204F5816205921A1D71
:10F61000079223B3330E84F8093404F20A44330CFE
:10F62000DFF850802370330A6370A670D8F8500357
:10F630006C6AFFF763FF6B7FA0809BB16946204631
:10F6400050F08EFC6C6A20685BF082FED8F858039C
:10F65000FFF754FFA080384614B0BDE8F08104F2F3
:10F660000944DCE705A9EAE700000020DC5000209F
:10F67000D5890008884D0020704737B590F85F386D
:10F68000032B04462FD100231F4D8DF807309DF822
:10F69000073094F860289A4201D803B030BD9DF835
:10F6A000073005EBC30393F860338BB181F001039E
:10F6B00083B19DF8073005EBC303D3F85C03FBF778
:10F6C00061F99DF807300133DBB28DF80730DEE7D2
:10F6D0000B46EDE79DF8073005EBC303D3F85C0359
:10F6E000FBF74AF9EDE7D0E910039B7903F001033A
:10F6F000994204D003B0BDE83040FBF743B903B0F2
:10F70000BDE83040FBF738B9884D002038B50446D5
:10F7100000790D4650B1FAF76BFF08B10323C3809F
:10F72000E2792946BDE83840FCF708B938BD10B584
:10F7300004462A21FFF7EAFF62792068013A022392
:10F740009340DB43036161790122BDE810405CF026
:10F7500073BE10B504460921FFF7D8FF6179206810
:10F760000022BDE810405CF067BE38B510F8133CCD
:10F77000A0F664041BBB94F850388BBBD4E9092372
:10F780009A421CD05A1CA169A262CB5C21695B0021
:10F7900043F40073A4F854380A2384F85238012340
:10F7A00084F8503894F85F388A4228BF0022012B31
:10F7B000A26201D0042B02D1606CFFF7CAFF94F85B
:10F7C0004C38002B6FD194F84D380133DBB2092B44
:10F7D00084F84D3825D12046BDE83840F9F756B8B1
:10F7E00094F952586DB1B4F854184B08A4F8543831
:10F7F00001F001012046013DFFF73FFF84F8525818
:10F80000DDE7D4E909239A4284F85058D7D194F817
:10F810005F38012B01D0042BD1D1606CFFF787FF3B
:10F82000CDE70A2B3FD194F84F382BB9B4F85638AE
:10F8300043F00103A4F856382379D9070AD5B4F860
:10F840005608820501D4C3071AD4B4F85C380133D2
:10F85000A4F85C38012284F84C2894F84F2800233F
:10F86000012A84F84D381ED184F84F386279636CD0
:10F8700002F0010259791868BDE838405BF012B80F
:10F88000E36AC0F3470013B1216B9847E2E7E369ED
:10F890006269D054E369E2680133B3FBF2F102FB21
:10F8A0001133E361D6E738BD2DE9F84310F8133C76
:10F8B000A0F664048BB1B4F8583801339BB2082B1E
:10F8C000A4F858381DD9636C002284F85128A4F894
:10F8D0005828597918685AF0E5FF384F97F89C83F3
:10F8E000B8F1000F03D101212046FFF7C6FE94F8BE
:10F8F000503853BBD4E909239A4204D1002387F836
:10F900009C33BDE8F883B8F1020F12D808F1010862
:10F9100014BFFF237F2387F89C83A4F8543808235F
:10F9200084F85238012384F85038606CBDE8F843FD
:10F930000FE75A1CA169A262CB5C21698A4228BFE9
:10F940000022DBB228BFA262E7E794F952685EB3F7
:10F95000B4F8549897F89D5319F001010BD0012D7C
:10F9600001D8012103E0AB1E012B09D8002120465C
:10F97000FFF783FE04E015F0FD03F2D0012BF6D073
:10F980000135EDB2032D87F89D53BAD9013E4FEAF8
:10F99000590976B20023A4F8549884F8526887F87D
:10F9A0009D33002EA6D0ACE7D4E909239A42A8D112
:10F9B00084F85068606CBDE8F843B8E6884D0020D4
:10F9C0001A4B00B5A3F5687C03F1300EDA794AB121
:10F9D0005A790CEB82010CEB4202D1F8E81389B2A0
:10F9E000A2F800140C337345F0D100EB40030CEB8C
:10F9F000830393F8A72332B10438012893F8A53381
:10FA00000BD9052B02D900205DF804FB0CEB430C4D
:10FA1000BCF8002490B25DF804FB052BF3D80CEB86
:10FA20008303D3F8E80380B2EEE700BF285100203B
:10FA30000548D0F8B83523B1DB6A13B100F5B760DB
:10FA400018470248704700BF982B0020F40D0708A4
:10FA500038B51D4CD4F80C341B8843B91B4D00231A
:10FA600084F81B3485F8B035C5F8AC3538BDD4F80A
:10FA70001024002AF2DDD4F81414012A488806D094
:10FA80000123124DA4F8180484F81A34E7E78A8891
:10FA90000132121A9A42F3D10C4DD5F8B835002232
:10FAA0001B69C5F8E42505F5B7609847D5F8B83562
:10FAB0009B68002BD3D005F5B76098470028CED1BE
:10FAC00059F02AFDCBE700BF884D0020982B00207D
:10FAD0000748D0F8B4351BB1064B93F81A340BB174
:10FAE00000207047D0F8B83500F5B7605B6818475C
:10FAF000982B0020884D002030B4174A174B92F8FD
:10FB0000B0C503F21C4505EB0C04C0E9004593F8B1
:10FB10001B3492F8B005834292F8B00514D88342A2
:10FB200006D300231A46184630BCC1E9003270479C
:10FB300092F8B0051A1EC0F1800330BC0CBF012042
:10FB40000220C1E9003270471B1A0022012030BC9C
:10FB5000C1E90032704700BF982B0020884D00207B
:10FB60000E4B0F4A93F8B01592F81B0493F8B0258A
:10FB7000904293F8B0250CD8904238BF93F8B02546
:10FB8000D3F8AC353ABFC2F1800280180020184487
:10FB90007047D3F8AC35801A18447047982B002072
:10FBA000884D002038B5194D194CD5F80C24937B9D
:10FBB000012B08D0D4F8AC3503F2FF736FF30A03BE
:10FBC000C4F8AC3538BDD4F8B8355B6A63B104F518
:10FBD000B7609847D4F8B8359B681BB104F5B76097
:10FBE000984778B1D5F80C24D4F8AC355288013B4D
:10FBF00013445242134003F2FF736FF30A03C4F835
:10FC0000AC3538BD59F088FCECE700BF884D0020CA
:10FC1000982B002070B51E4C1E4D94F8B03594F80A
:10FC2000B01584B005F21C421344029395F81B34BE
:10FC300003928B4220D894F8B025934214D294F8C2
:10FC4000B0151E46C1F18001F3B98C460122CDE901
:10FC5000001610B9BCF13F0F06D90023694602A86F
:10FC60005CF050FB95F81B3494F8B005C01AB0FA5C
:10FC700080F0400904B070BD94F8B0C5A3EB0C0C43
:10FC8000614600260122E2E701EB030C0222DEE7D7
:10FC9000982B0020884D00202DE9F043164685B0B2
:10FCA000002936D0441E254D254F04EB01084FF0A6
:10FCB000000901E0A0452CD095F81B0414F8013F81
:10FCC000411C2844C9B280F81C340B0648BF0020F0
:10FCD00097F8B03585F81B144ABF0146084685F8E9
:10FCE0001B94994297F8B03536BFC3F18003C01A10
:10FCF000C0183F28DED997F8B0359942DAD0114BB9
:10FD000093F89430002BD5D00020FFF783FFA04557
:10FD1000D2D1694602A8FFF7EFFE20B1DDE900323B
:10FD200013443F2B02D805B0BDE8F08302463346AA
:10FD300002A85CF0E7FA05B0BDE8F083884D00202A
:10FD4000982B00200000002030B585B0694602A83D
:10FD5000FFF7D2FE58B9094C04F5B765D4F8B835A9
:10FD600028465B6898470028F8D005B030BD0246A9
:10FD7000012302A85CF0C6FAEDE700BF982B002033
:10FD800070B5134D134C0023C5F8B43558F0A4FAE0
:10FD9000C4F81404FFF74CFED4F81434C4F80C046F
:10FDA000A3B19A885B88D21A436802FB0333C5F873
:10FDB000B435F8F70FFF95F8B03594F81B249A4244
:10FDC000064601D0FFF7C0FFC5F8AC6570BD00BFA7
:10FDD000982B0020884D00202DE9F041104ED6F8D8
:10FDE000B435154682189A420E4A88BF1D1A92F8F9
:10FDF0001B2496F8B0359A4204460F4601D0FFF70F
:10FE0000A3FFD6F8B82508480023C6F8E4352B46EA
:10FE1000956A21463A46AC46BDE8F041604700BFCE
:10FE2000982B0020884D0020503100208C4613462E
:10FE3000014662461846CFE72DE9F04F41F62C7295
:10FE40008DB00021A8485FF045FDA84A0023099322
:10FE500009920999043209680A930A920A9A126867
:10FE600051EA020040F03181A14B0393039BA14969
:10FE70009D48D3F84444E4225FF0D4FC9A4BC3E994
:10FE80000744C3E91A445C621C67C3F8B4401F46C8
:10FE9000C3F8B840C3F8BC405AF0BAFDFFF770FF92
:10FEA000002108460DF0EEF9F8F794FEB0F10008D5
:10FEB00040F3AC81904DDFF864C2904ECDF808C09D
:10FEC000002407F1E40943460194C8462746A346A7
:10FED00005F29C4A994604E00BF5006BD94540F3C6
:10FEE000B080874B029A1B68C2F85435F8F790FC33
:10FEF000202251465846FFF76FFF82491222504692
:10FF00005FF025FD0028E7D1BB4525D001997E4B48
:10FF100001EB410203EB820301934A1C18467B4923
:10FF20000592ABEB0703049301F020FC4146019BD3
:10FF300041F84C3B049B059AC8F80C70C8E904339F
:10FF4000D8F81C300192C8E90833714BC8F8283042
:10FF50000123C8F808308846039BD3F84434C8F816
:10FF60001C305F461222A918335D91F89C14994207
:10FF700002F101020BD00024202AF4D12037B94528
:10FF80005146384653DBFFF727FF0022EBE70134E9
:10FF9000152CF1D1D0195F492022FFF71DFF002356
:10FFA0000A220BA95B48CDF82CA001F011FD0746F1
:10FFB0000B98002301300A220BA90B9001F008FDD9
:10FFC00007900B98002301300A220BA90B9001F037
:10FFD000FFFC06900B98002301300A220BA90B901E
:10FFE00001F0F6FC05900B980BA9013000230A22C2
:10FFF0000B9001F0EDFC04900B98002301300A22D5
:020000040801F1
:10000000194601F0E5FC97B1DDE9063243EA4212F8
:10001000049B05995B0143EAC123A7F2BC7143EA43
:10002000600342EA412243EA0243C8F81C30019BC4
:10003000642B00F0B8805F460BF5006BD9453FF7A5
:1000400050AF4B46C1469846019B642B00F0AC80F4
:10005000BB451DD0019B2C4C2C490C2202FB0344B8
:1000600001331A462046019301F080FBD9F81C2089
:10007000C9F80040ABEB0705C9E90822C9E90375D7
:10008000234AC9F828200122C9F81450C9F80820C9
:10009000019B002B03F1030100F389804FEA480321
:1000A000B3F1805FC0F2B3800F4B986830B91A4645
:1000B0001B791BB11368002B40F0DF80002108463C
:1000C0000DB0BDE8F04F0DF0DDB898184FF47A721E
:1000D00000235DF00FF9104BA3FB00231B0C40F233
:1000E000B27240F26D141DE010AC00206028004098
:1000F00000000020080E0708884D0020689D0708B2
:10010000A01A0020449D070844520020589D07086B
:100110002DFE00082452002007452EC2982B0020F7
:100120005B1A013212F0030514BF21464FF4B77178
:100130008B42F5DAA449002D00F0998003910399D0
:10014000D1F81414994200F33C81A04D01245B1AAC
:1001500055F8041F994204F10104F8DD013343EA24
:100160004413A2F2BC7243EA4223994A039DB0FBB6
:10017000F2F102FB11024FF461603C24B2FBF0F19A
:1001800000FB11221C20C5F81804B2FBF4F004FB9C
:100190001022521042EA401242EAC12242EA0343CC
:1001A000C5F8443462E6C8466423019367214C26AF
:1001B0008848DFF83492884F06FB01F4051932466F
:1001C000002128465FF086FB3246002128465FF07A
:1001D00081FB8048814E40F8049004F110034FF0F9
:1001E000010AC5F808A02F62AE6240F803800344FC
:1001F000021DC3F804801834039B0199D3F84434DA
:100200001351A018043143606B6247E70321714B1F
:10021000DFF8D8914C2606FB01F41D193246002167
:1002200028465FF057FB3246002128465FF052FB1C
:10023000684B694E43F80490039A2E62684ED2F8D8
:10024000440404F1100104F118020127341FC8F11D
:100250000063BB404FF0020A85F805A0AF60635011
:1002600021444B60B0503244506068621CE70C4639
:1002700003911D21C4F8181461E756490022002398
:10028000C1E9102388640A46C86305460146D46C58
:1002900002F14C03B4B19C689D644E1EB442C2E9A5
:1002A0002355DD6300F086804E1CB44274D113F8F0
:1002B000481C00293FF402AF1A6443F8083C214669
:1002C0001A46E4E7434A0226254615E0D36B166337
:1002D0005B0118BF03F6FF73C2E9045514BF01EBBD
:1002E0001333334653631946916352F84C7FCB1A4C
:1002F0001C444E1C0130CFB11379711E002BE5D187
:10030000136916635BB103F6FF73576901EB13338F
:1003100053634FB107F6FF7701EB1731E4E75769F5
:1003200033465363002FF5D13146DDE7DFF8C0C017
:100330002C4BCCF8984501390CF5AE62CCF87C35E5
:100340003E2440233F25CCF8A405CCF88835C2E9EB
:100350000445CCF89415880F8B00D9B140F2FF14F6
:100360001B1940F100005B0A43EAC0531948C2E977
:100370000B0003F14000034403EBC101CCF89035BE
:10038000CB0D53604B02CCF88C05CCF87815CCF82B
:10039000703593E60123E9E78C427FF48FAE0029A4
:1003A0003FF48CAE146CE66B0136E6631C64936418
:1003B0001A466CE700293FF481AE53F80C2C214615
:1003C000EDE70124CAE600BF00000020140400206D
:1003D0008051010010AC00200068214C2DFE000867
:1003E00014AC00209C9D0708809D0708909D07087D
:1003F000982B00202DE9F043DFF82881474D93B07A
:10040000FFF726FB98F8B03595F81B249A4201D0E7
:10041000FFF79AFCD8F8B4750024C8F8AC45002F53
:100420006CD03F4E0AE098F8B03595F81B249A42FC
:1004300001D0FFF789FC2034A7421BD92246314660
:10044000684601F093F968465CF0F6FA012201462D
:100450006846FFF721FCA3B2002BE4D1D8F8583549
:10046000002BE0D09A881B6859690A4218BF120411
:100470009A61D8E7FFF796FB98F8B03595F81B24FA
:100480009A4201D0FFF760FC0023DFF89490C8F88F
:10049000AC351E461C4601E0A74229D922464946F2
:1004A00009A801F063F92122002168465FF012FAE1
:1004B000202269462046FFF78FFC2022054609A925
:1004C00068465FF044FA08B9202D00D00136A3B287
:1004D0002034002BE0D1D8F85835002BDCD01A6836
:1004E0009B8851690B4218BF1B04A7429361D5D862
:1004F000B6FA86F0400913B0BDE8F083FFF752FB6F
:1005000098F8B03595F81B249A4201D0FFF71CFCEF
:100510000023C8F8AC350120EDE700BF884D00206E
:10052000A49D0708982B0020704700BFD0ED007AEB
:10053000D0ED016A30EE677AE6EE877AB0EE670AB0
:10054000C0ED007A704700BFD0ED017AD0ED026AAD
:1005500030EE677A90ED000AE6EE877A37EEC07AE1
:10056000C0ED017AA6EE870A80ED000A704700BF51
:1005700090ED017AD0ED036AD0ED027A30EE470AB1
:10058000A6EE807A90ED000A80ED017A37EE676A78
:10059000E6EE867A37EEC07AC0ED027AA6EE870ADA
:1005A00080ED000A704700BFD0ED056AD0ED017AFA
:1005B00090ED066AD0ED025A90ED035AC0ED066A3E
:1005C000B0EE407A26EEA70AD0ED007A80ED057AEB
:1005D000A7EE870AD0ED077AA5EE860A90ED086AA5
:1005E000D0ED045AC0ED087AA5EE670AA5EEC60A5A
:1005F00080ED070A704700BFF0EE406AD0ED007A48
:1006000090ED050A90ED067A90ED016AD0ED035A5F
:10061000A7EEA60AA6EE267AD0ED047A90ED026A3D
:1006200067EEC07AA5EEC07AE6EE267A80ED057A0E
:10063000C0ED067A704700BF2DE9F047DDF820A035
:1006400055460F4615F8011B002B064614460CBFF5
:100650004FF020094FF0300939B3002A2BDD2B462B
:1006600000E09CB113F8012BA046013C002AF8D110
:10067000A8F1020854B1444649463046B847013C07
:10068000FAD29AF8001008F1010459B13046B8477F
:100690002B4615F8011B0029F8D1A4EB0A04181900
:1006A000BDE8F0872046BDE8F087002A02F1FF3858
:1006B000E1DC0846F4E70024E8E700BF03685A1CC1
:1006C00002601970704700BF10B500F10044024687
:1006D000013C04E0B3EB0E0015D1A24214D012F895
:1006E000013BA3F14100192811F8010BA0F1410CC5
:1006F00098BF2033BCF1190F00F1200EEAD91B1A64
:1007000004D10028E9D110BD002010BD184610BD4D
:10071000884210B54FF001043ED301FB04F4B0FB56
:10072000F4FC8C45F9D2CCB122BB08E0A14203F81D
:1007300001EBB4FBF1F211D8B0FBF2FC1446BCF1B2
:10074000090F0CF1570E0CF1300204FB1C00EDDC1C
:10075000A14203F8012BB4FBF1F2EDD900221A708B
:1007600010BDA14203F801EBB4FBF1F2F6D8B0FBE7
:10077000F2FC1446BCF1090F0CF1370E0CF13002FB
:1007800004FB1C00EDDCA14203F8012BB4FBF1F2E9
:10079000EDD900221A7010BD8446002AEAD1CEE7B6
:1007A000002870B503DA2D2301F8013B40420928E7
:1007B00086464FF0010307DD03EB83035B00B0FBCC
:1007C000F3F2092AF8D8E3B10F4CA4FB0320BEFBD7
:1007D000F3F2092A02F1570602F130054FEAD00080
:1007E00007DD092B01F8016B03FB12EE09D9034663
:1007F000EBE7092B01F8015B03FB12EE01D903467D
:10080000E3E700230B7070BDCDCCCCCC0378202B5C
:10081000024600F10100F9D0092BF7D02D2B28D08A
:100820002B2B03BF5378B7EE000A0246B7EE000A3F
:10083000A3F13001C8B209289FED567A10D8F2EE24
:10084000046A07EE901AF8EEE77A12F8013FE7EE35
:10085000267AA3F13001C8B20928B0EE677AF0D940
:100860002E2B5ED003F0DF03452B07D020EE070AC6
:1008700070475378BFEE000A0246D9E710B45178AA
:100880002D2978D02B296AD0A1F13003092B02F150
:1008900001026BD80024002303EB830301EB430325
:1008A00012F8011FA1F130000928A3F13003F3D998
:1008B000B3F59A7F1A4628BF4FF49A72072B66D970
:1008C000DFED356A1346F7EE007A083B072B67EE3B
:1008D000A67AFAD802F00702DAB1F2EE046A012A27
:1008E00067EEA67A15D0022A67EEA67A11D0032AFF
:1008F00067EEA67A0DD0042A67EEA67A09D0052AFB
:1009000067EEA67A05D067EEA67A062A18BF67EECC
:10091000A67A6CB387EE277A5DF8044B20EE070ABF
:1009200070475378A3F13001C8B2092802F10102DF
:1009300098D8F2EE046AF0EE665A07EE901AF8EED6
:10094000E77A12F8013F87EEA66AA3F13001C8B238
:10095000092866EEA56A37EE067AEED982E7917825
:10096000A1F13003092B02F1020293D9F7EE007ACC
:1009700027EE277AD0E79178A1F13003092B02F115
:10098000020288BFF7EE007AC4D8012483E7F7EEAD
:10099000007AA1E70000000020BCBE4CF0B506794B
:1009A00006F0E003402B03D145794FF0FF3406E019
:1009B000602B4FF00105F8D1447905FA04F40023C7
:1009C000012006F00706AB4200D1F0BD052E0FD87E
:1009D000DFE806F00308101D242448B1C85CD75C8A
:1009E00078400FE020B1C856D756C71B78427841EF
:1009F0000133E8E70028FBD031F8130032F8137018
:100A0000784080B220420CBF01200020F0E700288F
:100A1000EED031F9130032F91370E6E70028E7D081
:100A200051F8230052F82370DAE7F8B50C4E33780A
:100A300005468BB9F8BD25B12388C3F30B039D424E
:100A400004D0D4E90201A2885EF0ECFE1C34BC4262
:100A5000F1D300233370EDE7024C034FF7E700BFFB
:100A6000E4DB0020643A0808CC430808037903F06B
:100A70001803102B1CD003D833B9B0F80B00704703
:100A8000182BFAD000207047104BB0F80B0093F9E8
:100A90000030591C06BF0E4B1B78DBB203EB430240
:100AA00003EB820303EBC30300EB430080B2704708
:100AB000064BB0F80B0093F901305A1C06BF044BEB
:100AC0005B78DBB200EB4310F0E700BFA804002026
:100AD000F4560020032870B518D80D4BC60003EB60
:100AE000C000C943057A427A01F0010181EA050498
:100AF000A2420BD042683AB14D1B694210689288FD
:100B0000694109018A40826133445C7270BD00BF53
:100B1000E4DB00200379062B0FD1C9B20E2998BF60
:100B2000074BC26894BF5956002101238B401342E2
:100B300014BF08464FF0FF307047481C704700BF95
:100B4000209E0708092900D001B9704701394A00E1
:100B500002F00802930001F00301A3EB9203C1EB42
:100B60000111C3EB0313C1EB011100229B008900AB
:100B70000260818043807047B5EEC00ADFED347AB1
:100B8000F1EE10FACCBF30EE270A30EE670ADFED47
:100B9000317A20EE270A30B5FDEEC07A87B017EE25
:100BA000904A054684EAE470002303A9A0EBE470B0
:100BB000CDE90033029356F0E5F8002CB4BF2D23A5
:100BC000202303A88DF800305BF036FF012829D0E0
:100BD000022833D003281DD003A968465EF082FEA8
:100BE00068465BF029FFC41EE4B2224669462846E7
:100BF0005EF018FE00232B5528465BF01DFF2E23C8
:100C00002B5401300DEB040128445EF098FE284679
:100C100007B030BD302303A968468DF801305EF07F
:100C200061FEDDE743F23002302303A96846ADF8E8
:100C300001208DF803305EF055FED1E743F230031A
:100C400003A96846ADF801305EF04CFEC8E700BF6E
:100C50006F12033A00007A440CF072B838B50546BA
:100C600058B14C1E14F8011F284619B9BDE8384088
:100C70000CF07AB80CF064F8F4E738BD70B50546AE
:100C8000B0F8090052F072FD054B1E780446284664
:100C9000FFF7ECFE16B1E368184470BDA368FBE7EC
:100CA000E4DB002038B505460C46FFF7E7FF2A795C
:100CB00002F0070302F0E002602A29D1052B0CD8CC
:100CC000DFE803F0030B0F0B1B1B6A790123934032
:100CD000DBB2027814B11343037038BD22EA030378
:100CE000FAE76A79012393409BB2028814B1134357
:100CF0000380F2E722EA0303FAE76B7901229A40C4
:100D0000036814B113430360E7E723EA0203FAE739
:100D1000052BE2D8DFE803F003030505070704709D
:100D2000DBE70480D9E70460D7E708B520215EF04F
:100D3000E8FD0346184623B10278202A03F1010397
:100D4000F8D008BD08B5CB0701D4FDF747FA08BDB8
:100D50002DE9F341124D134F002305F8243F0446BB
:100D600000EB8106B44203D10F4802B0BDE8F08128
:100D7000394628465EF0B6FD214668465EF0DFFD46
:100D80004FF00008202168465EF0BBFD28B9694697
:100D900028465EF0A7FD0434E4E780F80080F1E720
:100DA000E4DB00207B1E080808DC00202DE9FF475B
:100DB000914604468A461E46FFF7ACFE421CBDF82B
:100DC0003070DDF8348005461FD0B9F1FF3F1FD0E9
:100DD000CDE90009144A236831463846C0474A46DF
:100DE00020795FFA8AF1FAF7C7FC024600B102885F
:100DF000D3B20393C2F30323120BCDE90052029343
:100E000023680A4A31463846C04704B0BDE8F08737
:100E10007B06FAD40C902368054A31463846C4460E
:100E200004B0BDE8F0476047B0120808BD120808DA
:100E3000E21208082DE9F043154685B06A1C894680
:100E4000BDF830600D9F194628D04FEA101800F009
:100E50000F0408F14008CDE90045174A43463046E3
:100E6000B847C0B1EBB20D2BD9F8000099F80510C6
:100E700011D82A46FAF7D4FC68B1038802780392A5
:100E8000C3F303221B0BCDE90043029243460B4AF6
:100E900000213046B84705B0BDE8F0837306FAD4A8
:100EA0000309074A00F00F000C9040333046BC465F
:100EB00005B0BDE8F0436047F112080803130808C5
:100EC0002D1308082DE9F04387B04FEA1018DDF81C
:100ED000389015461F4608F1400800F00F0421B372
:100EE0000EF056FFC379164ACDE900430646434645
:100EF00029463846C847A8B13068FAF7E1FCB3790B
:100F00001049727913F0020F0F4B18BF0B46F1799D
:100F10000094CDE90331CDE9010243460B4A00219B
:100F20003846C84707B0BDE8F083094A0E944346E7
:100F300029463846CC4607B0BDE8F043604700BFBD
:100F40004113080838170808A72808085313080889
:100F50007513080800B501EB020E714516D0013972
:100F60000EF1FF3E41F2210C11F8013F082280EA08
:100F7000032003B2002B4FEA4000B6BF8CEA4303C4
:100F800080B298B2013AF4D18E45EDD15DF804FB00
:100F90004840082341B240000029C0B2B8BF5040C9
:100FA000013BF7D1704700BF30B505688D4204465C
:100FB00018D901F1FF3E681E00231EF801CF082159
:100FC00083EA0C034FFA83FC5B00BCF1000FDBB239
:100FD000B8BF53400139F5D17045EED16A1C22608B
:100FE0002B7030BD00236A1C22602B7030BD00BF07
:100FF00010B52DED028B08EE101AB8EE488ADFED21
:101000007E7ADFED7E0A28EE008A044628EE278AE3
:10101000B0EE480A5DF038FB9FED797AB4EEC70A6E
:10102000F1EE10FAF0EE407A40F3BD809FED736A66
:10103000DFED746AB0EE677AB4EEE67AF1EE10FA9C
:1010400077EEC67AF6DC9FED707AF4EEC77AF1EEB1
:1010500010FA40F3C5809FED6A7A77EE677A27EE43
:10106000A76ADFED6A5ADFED6A6A9FED6A7A9FED43
:10107000660ADFED620AE6EE256A67EE865AA6EE9C
:10108000267A38EE000AE5EE877AB0EE678A5DF0E0
:10109000FBFADFED5B7AB4EEE70AF1EE10FA5BDD06
:1010A000DFED566A9FED577AF0EE407AF4EEC77A9C
:1010B000F1EE10FA30EE660AF6DCDFED537AB4EEAC
:1010C000E70AF1EE10FA62DDDFED4D7A37EEC00A85
:1010D000F7EE007ADFED504ADFED4C5A9FED4C7A87
:1010E000C4ED097AB0EE675AA8EE245A0023A36132
:1010F00060EE006A87EE856A63612362E361A6EEB3
:10110000A57A9FED445AA6EE875A20EE264AF0EEC5
:10111000675AA4EE050AE8EE645ABDEC028BB6EEFF
:10112000007AF8EE006A77EEC07A26EE077A66EE6D
:10113000266A27EE277A66EE806A67EE867A25EEC3
:10114000866A84ED007AC4ED017A84ED027AC4EDFA
:10115000036A84ED046A10BDDFED307AB4EEE70A6D
:10116000F1EE10FAA9D5DFED256A9FED2D7AF0EEAC
:10117000407AF4EEC77AF1EE10FA30EE260AF6D491
:10118000DFED217AB4EEE70AF1EE10FA9CDCDFED38
:10119000257AB4EEE70AF1EE10FA44BFDFED1F7ACC
:1011A00037EEC00A94E79FED1D7AB4EEC70AF1EE60
:1011B00010FA7FF548AF9FED116ADFED196AB0EEC6
:1011C000677AB4EEE67AF1EE10FA77EE867AF6D424
:1011D0009FED0D7AF4EEC77AF1EE10FA3FF73BAFD0
:1011E0009FED107AF4EEC77AF1EE10FA44BF9FED4E
:1011F0000B7A77EE677A32E727D4D236DB0FC94015
:10120000DB0F4940E4CB1641DB0FC93F92E741B900
:101210009730083C15A82ABEF304353FDB0F49C0C0
:10122000E4CB16C1DB0FC9BF08B5DFED2D0A5DF0B9
:101230002BFADFED2C7AB4EEE70AF1EE10FA28DD96
:10124000DFED276A9FED287AF0EE407AF4EEC77A58
:10125000F1EE10FA30EE660AF6DCDFED247AB4EE39
:10126000E70AF1EE10FA2FDDDFED1E7A37EEC00A45
:1012700020EE007A9FED1E6ADFED1E6ADFED1E7A1A
:10128000E7EE066A20EE076AE6EE877AA6EE270A00
:1012900008BDDFED1A7AB4EEE70AF1EE10FADCD5FC
:1012A000DFED0F6A9FED167AF0EE407AF4EEC77A22
:1012B000F1EE10FA30EE260AF6D4DFED0C7AB4EE39
:1012C000E70AF1EE10FACFDCDFED0E7AB4EEE70AB2
:1012D000F1EE10FA44BFDFED097A37EEC00AC7E736
:1012E000DB0FC940DB0F4940E4CB1641DB0FC93FA0
:1012F00092E741B99730083C15A82ABEDB0F49C0D8
:10130000E4CB16C1DB0FC9BFDFED2F7ADFED2F0A6B
:1013100030EE270A08B55DF0B7F9DFED2D7AB4EEAF
:10132000E70AF1EE10FA28DDDFED286A9FED297A51
:10133000F0EE407AF4EEC77AF1EE10FA30EE660A7B
:10134000F6DCDFED217AB4EEE70AF1EE10FA2FDDDC
:10135000DFED1F7A37EEC00A60EE006A9FED1E6A6D
:101360009FED1E7ADFED1E7AA6EE867A20EE266AC3
:10137000E6EE877AA6EE270A08BDDFED1A7AB4EE0C
:10138000E70AF1EE10FADCD5DFED106A9FED167A70
:10139000F0EE407AF4EEC77AF1EE10FA30EE260A5B
:1013A000F6D4DFED097AB4EEE70AF1EE10FACFDCFD
:1013B000DFED0E7AB4EEE70AF1EE10FA44BFDFED8E
:1013C000097A37EEC00AC7E7DB0FC93FDB0FC94018
:1013D000DB0F4940E4CB164192E741B99730083C16
:1013E00015A82ABEDB0F49C0E4CB16C1DB0FC9BF6D
:1013F000B0EEC07AF0EEE06AF4EEC76AF1EE10FAF1
:10140000B4BFF0EE475AF0EE665AF5EE405AF1EEF0
:1014100010FAF0EE407A44D0F4EEC76AF1EE10FA1A
:101420008CBFB0EE475AB0EE665A85EE256A9FED46
:101430001E2A9FED1E3A9FED1E4ADFED1E4ADFED8C
:101440001E2ADFED1E3A9FED1E5AA6EE423AE6EE48
:10145000223AA6EE034AF7EE005AE6EE044AE6EE1A
:10146000235AA6EE245A85EE250AF4EEC76AF1EE59
:1014700010FA48BF9FED137AF5EEC00A48BF37EE69
:10148000400AF1EE10FA48BF9FED0F7AF5EEC07AF0
:1014900048BF37EE400AF1EE10FA48BFB1EE400AFD
:1014A00070479FED070AE0E739094E3DE3B59E3EE0
:1014B00088FA163E45FE7F3F99FB243F69A2163EFF
:1014C000A7DFA834DB0FC93FDB0F49402DE9F04F00
:1014D000144689B08846217801320392002900F031
:1014E0001681002507461E46A94609E03846C04732
:1014F000039C01352178631C0393002900F08F8041
:101500002529F3D16078A31C3028CDE9033923D0F5
:10151000A0F13003DBB2092B4FF0000A26D96C286A
:101520002AD078287FD8572878D9A0F15803202BC3
:1015300079D8DFE803F0BD787878787878787878AB
:101540007882AF787878787878787878AA787878A8
:10155000789E788A7878BD00A078E31C0393A0F188
:101560003003DBB2092B4FF0010AD8D804AA03A933
:1015700056F0C6FE6C28D4D1039C22780134782A18
:101580000394B7D8572A40F28E80A2F15803202B3B
:10159000B0D801A151F823F0CF160108F5140108C5
:1015A000F5140108F5140108F5140108F5140108F3
:1015B000F5140108F5140108F5140108F5140108E3
:1015C000F51401083D160108EB160108F514010891
:1015D000F5140108F5140108F5140108F5140108C3
:1015E000F5140108F5140108F5140108F5140108B3
:1015F0008D160108F5140108F5140108F514010809
:10160000F514010875160108F5140108FB16010808
:10161000F5140108F5140108CF16010828B9284669
:1016200009B0BDE8F08F039C64E72528FBD1039C3B
:1016300025213846C04701355CE7039C56F8041B5A
:101640003846C9B2C047013554E70DF1140B56F8BE
:10165000040B039C5B4600220A21FFF759F8049A09
:10166000CDF800B0534641463846FEF7E5FF054445
:1016700040E7039C56F8043B0093049A002341463C
:101680003846FEF7D9FF054434E7039C56F8043B7F
:101690001D602FE70DF1140B56F8040B039C5946FF
:1016A000FFF77EF8DBE7002AB9D0252AC0D021E772
:1016B000A0F15802B2FA82F20DF1140B56F8040BA5
:1016C00052095B461021FFF723F8039CC7E7A2F1FC
:1016D00058020DF1140BB2FA82F256F8040B5209BB
:1016E0005B461021FFF714F8B9E70DF1140B56F81B
:1016F000040B5946FFF754F8B1E70DF1140B56F8F7
:10170000040B5B4600220A21FFF702F8A7E70D460B
:1017100085E7F8B5104C0746A06C0D461646A0B1FB
:101720000E49FFF79BFAA06C3946FFF797FA0C4970
:10173000A06CFFF793FA0B49A06C33462A46FFF7DB
:10174000C5FE0949A06CFFF789FA94F84C3013B133
:10175000012384F84D30F8BDE4DB0020871308082E
:101760009E2D0808590C0108941308080EB400B502
:1017700084B005AB019053F8042B0649039301A8EC
:10178000FFF7A4FE019B00221A7004B05DF804EB81
:1017900003B07047BD060108F7B5114E0746304645
:1017A000002300F84E3F0C460E4B0F49002F18BF88
:1017B000194615465EF096F80C4F04EB45054E367B
:1017C000AC4202D10A4803B0F0BD394634F8022BCE
:1017D0006846FFF7CBFF694630465EF083F8EFE7D7
:1017E000E4DB002098130808A1130808AA130808CE
:1017F00032DC0020F7B50C4E0C4F002306F87F3F7B
:10180000044600EB4105AC4202D1094803B0F0BDEB
:10181000394634F8022B6846FFF7A8FF6946304680
:101820005EF060F8EFE700BFE4DB0020F634080864
:1018300063DC0020F8B5084F4E1E054601F11F0479
:1018400016F8012F28463946FFF790FFA64205F10A
:101850000205F5D1F8BD00BFAF1308080246531CBE
:10186000084605D1034B1A681B790A600B71704753
:1018700001497BE7EC120808F734080810B501317C
:1018800014460EF085FA28B9054B1A681B792260B8
:10189000237110BDC27903492046BDE8104065E7B9
:1018A000EC1208084E13080803685A1C02601970ED
:1018B0000368090A5A1C02601970704710B4026864
:1018C0001346511C016013F8021B0360D31C5478AB
:1018D000036093781B0443EA0423141D0460D0784A
:1018E0005DF8044B0B4343EA00607047A0F13003FE
:1018F000092B07D920F02000413819288CBF00207F
:101900000120704701207047303809288CBF002023
:1019100001207047413819288CBF002001207047F2
:10192000613819288CBF002001207047202805D07D
:10193000093804288CBF002001207047012070471F
:10194000A0F14103192B98BF20307047A0F161032B
:10195000192B98BF2038704702B310B584468418FD
:1019600003E0981A15D1A44514D01CF8013BA3F14B
:101970004100192811F8010BA0F1410E98BF203346
:10198000BEF1190F00F12002EBD91B1A04D1002877
:10199000E9D110BD002010BD184610BD104670479B
:1019A00070B5044608460D465BF046F8064602E070
:1019B00014F8013F43B1324629462046FFF7CCFFD9
:1019C0000028F5D1204670BD1C46204670BD00BFE2
:1019D0002DE9F043064686469EF800C0BCF1200F74
:1019E0007446ACF109050EF1010EF5D0042DF3D9C2
:1019F000BCF12B0F64D0BCF12D0F26D10127102A8A
:101A000094F801C004F1010423D04FF0FF35B5FB79
:101A1000F2F502FB05FE6FEA0E0E5FFA8EFE9046AF
:101A2000002014F801CBBCF1390F4CF02009ACF1C7
:101A3000300C29D85FFA8CFC944528DAA842264657
:101A40001ED81BD000FB08C0EBE7102A4FF00007A0
:101A5000DBD1BCF1300F0AD16078A0F14105192D1E
:101A600098BF2030661C78280CBF023434466FF0D3
:101A700070454FF00F0E4FF01008D1E7F445E1D953
:101A80004FF0FF301F40CCE7B9F1600F0AD801B129
:101A90000E6067B923B16FF00043984228BF184623
:101AA000BDE8F083A9F157095FFA89FCC4E723B1C7
:101AB000B0F1004F28BF4FF000404042BDE8F08336
:101AC00000279CE773B50E4610490546FEF7FCFD5E
:101AD00018B93070012002B070BD2C78602C8CBF1A
:101AE000613C413C082C0FD8013501230A2201A991
:101AF0002846FFF76DFF019BAB4205D00F2803D8A6
:101B0000013440EA0410E4E70020E4E7EC1208089E
:101B100001230A2200215BE770B50D461446FFF74A
:101B200004F90646A0B1FFF7F3FF40F634039842EC
:101B3000A8BF1846B0F5617FB8BF4FF46170A0F53B
:101B400061731922B3FBF2F32B70237801332370F6
:101B50003046FFF7EAF80646A0B1FFF7D9FF40F696
:101B600034039842A8BF1846B0F5617FB8BF4FF460
:101B70006170A0F561731922B3FBF2F36B702378E7
:101B800001332370304670BD2DE9F04116461F46E3
:101B90000446394630464FF47A7200235BF0AAFBC4
:101BA0003C4D3D4B054483FB05602844E917C1EBE0
:101BB000601183FB01030B44384EC817C0EB631060
:101BC00086FB003CC317364EC3EBAC0386FB0376A3
:101BD0004FEAE37ECEEBE61EC1EB0116A5EB860CC9
:101BE000C0EB0015A1EB8501617103EB4301A0EB94
:101BF000C10040F2B55101FB1E33B3F5896F84F883
:101C000006C020714FEA8E0633DA40F2DA218B42A9
:101C100037DCB3F5B77FB4BF4FF0000E4FF0010EC5
:101C2000204F0EEB4E0107EBC1017546C88A4FEA03
:101C30004E0808EB0E0C07EBCC0C0CF1160C0B212C
:101C400001E03CF8020D984210DD0139F9D1F04471
:101C5000012137F83800A170013306F5FA6E1B1A1E
:101C60007544E37022812580BDE8F0810131C9B25D
:101C7000F1E703250B4F40F29650AE464FF00608B1
:101C8000D7E70225074F40F22940AE464FF004083F
:101C9000CFE700BF80BC92C789888888ABAAAA2AF0
:101CA00073B06D16B42307080C4B10B5D3E900438D
:101CB00054EA030209D1014640F201130020C1F8A1
:101CC000023088710880088110BD054A1268121917
:101CD00043F10003FFF758FF012010BDD050002052
:101CE000A01A00202DE9F04104469442154608460A
:101CF00009D2B4FBF2F6154B05FB16441B5D00F848
:101D0000013BBDE8F081B4FBF2F69642B6FBF2F778
:101D10000CD20E4B05FB176705FB1644DA5D00F885
:101D2000012B1B5D00F8013BBDE8F081BA42B7FB17
:101D3000F2F807D9054B05FB187813F8082000F8CE
:101D4000012BE7E74046FFF7CDFFF3E7309E07089A
:101D500030B5694CB4F8D434B4F8DA24B4F8DC14EF
:101D6000B4F8DE04B3F57A7F88BF4FF47A7383B09A
:101D700088BFA4F8D434B4F8D634B3F57A7F84BFDE
:101D80004FF47A73A4F8D634B4F8D834B3F57A7F24
:101D900084BF4FF47A73A4F8D834B2F57A7F84BF45
:101DA0000022A4F8DA24B1F57A7F4DD94FF47A7184
:101DB0008842A4F8DC1467D89A4224BF0023A4F810
:101DC000D834884224BF0023A4F8DC34B4F8EC34BF
:101DD000B4F8EA249A4284BF0023A4F8EA34474BBB
:101DE0001B88EBB1464DAA78062A3FD929790029EC
:101DF0006FD19FED447A444A117807EE903A06EE8F
:101E0000901AF8EEE77AB8EEE66AAB79C6EE276A82
:101E10000BB137EE077AB4EEE67AF1EE10FA3BDC5E
:101E20003A4B597803291DD8394A02EB41121978E7
:101E3000C4F8F42403290ED8364AEA2301FB03220E
:101E4000354B1A6003B030BDB0F57A7F84BF0020F7
:101E5000A4F8DE04B0E7002119702E4A2E4B1A6058
:101E600003B030BD00212A4A5970E0E72B4901EB4D
:101E7000820191ED187A29790029BCD0531F032BD8
:101E8000CED9002ACCD029E000219A42A4F8DE1451
:101E90009CD3A4F8D81499E767EE877ABCEEE77A6A
:101EA0008DED017A9DF8043007EE103AB8EEC77A4E
:101EB000F4EEC77AF1EE10FAC4BF0133DBB2CBB156
:101EC000102BA8BF1023DBB28B4238BF0B46137018
:101ED000A6E7053A032AA3D99FED0A7AB7EE000ACE
:101EE00080EE070A5CF042FC2B88834228BF034641
:101EF0002B8095E70123E6E7E4DB0020885E0020E5
:101F0000EC4000206F120338805E0020F456002061
:101F10008CDC00200CDD00202C620020B42307089C
:101F20002DE9F04FA84B83B01B78A3F11702022ACA
:101F300000AF13D9A54A12F83310002940F0B68239
:101F4000DB001A4452784AB1A14A3A60134493F82C
:101F50007C302BB99C4A1823137001E09C4B3B60EA
:101F60009C4B9D4E93F808809C4B4FF0000A03F168
:101F70006C059B461FE09BF90430142B00F0918206
:101F800020465DF03BFDA30323D5012800F08982A4
:101F9000082800F38682B9F1000F01D0344206D13F
:101FA0004146204659F010FA002800F07A820BF1E1
:101FB0000C0B5D4513D0DBF8004014F00109DAD0BA
:101FC00020465DF01BFD0AF1010AA3035FFA8AFABD
:101FD000DBD40128DCDC0BF10C0B5D45EBD10AF105
:101FE000FF33022B00F25D827D4DDFF8109200235B
:101FF000022085F8683512F0D9FA95F86C35D9F8D1
:102000000040022B00F0D582002800F02383DFF887
:10201000F0A1744B95F8C5C5C7F804C003F56A7BF9
:102020004FF47A784FF0000E6422264633F8081CED
:10203000B1F57A7FB3F8461088BF23F8088CB1F564
:102040007A7F33F8061C88BFA3F84680B1F57A7F03
:1020500033F8041C88BF23F8068C33F8060CB1F55E
:102060007A7F84BF002123F804EC8842B3F85A0039
:10207000B3F85C1098BF23F806EC884293F86B1015
:1020800088BFA3F85AE00139632993F86C1088BF20
:1020900083F86B200131C9B2092988BF83F86CE04D
:1020A00003F16500002113F8314010F801CF013130
:1020B000A44538BF80F800E00329F4D179680129EC
:1020C00018BF83F886E0EA339B45AFD13446464ECD
:1020D000B378042B00F09E8233B93388B3F5F07FD8
:1020E00084BF4FF4F0733380FFF732FE3F4895F81A
:1020F000D815FEF727FD95F8F7151030FEF722FDED
:10210000B5F80616B5F804360B43B5F808160B43B8
:102110001BB213B10123A5F80A36354B2340002B1F
:1021200000F0A582E00700F16082610400F1C9813E
:10213000220740F12F822F49DAF800300C400B4083
:10214000C9F80040CAF8003014F4004300F00882D7
:10215000204A0023D373D377E00440F10A8295F834
:102160001736DFF89480022B04BF012385F8173659
:1021700008F17804434602E006339C420CD01A78FA
:102180000A2AF9D19978DA78914202D35A79002A49
:10219000F2D00A2026F0A8F900234FF4806085F8D9
:1021A000683512F003FA002800F047821249C7F898
:1021B00004A08B468A469AF8050078B39AF8001076
:1021C00049B3434621E000BFBC5B0020A8110708CB
:1021D000B42307080C570020BC020200DCE00020FA
:1021E000E4DB002016DD0020EC400020CCE10020E4
:1021F00009600002FE9FFFFD00E20020E066002073
:102200000857002006339C4208D01A788242F9D140
:102210005A79002AF6D0084626F066F90AF1060A2D
:102220005445C8D196F80280D7F804A0B8F1080F39
:10223000594600F0B48195F8C535DAF800C0A3F12D
:102240000103B3FA83F35B0985F8943695F8C63534
:10225000A3F10103B3FA83F35B0985F89A3695F885
:10226000D134032B84BF002385F8D134AA4BCCF39F
:10227000C030DA7B85F89706D9F80030A7480340CC
:102280000CEA0000C9F80030CAF80000002A00F08B
:10229000AE81DFF8C492B9F80430002B40F0998188
:1022A0009F4A1368B3F5000F24BF0023136093689F
:1022B00023F4007323F0020313B140F2022393606E
:1022C0001379013B042B84BF01231371A8F1050886
:1022D000944BB8F1030F93F800B040F20C814FF02B
:1022E0000008BBF1000F25D0DFF870927C605C46DF
:1022F000CB46894606E0AAF1060AAAEB060A54452F
:1023000040F2E180DA461BF8010F0028F3D00DF00F
:1023100067FD0028EFD082799307ECD57C684946A9
:102320000122B8F1000F05D0737C3BB97379012B02
:1023300000D01AB1B3790BB10023B3717A4BDA88AC
:1023400002F00F00042803D8C2F30312022A02D9B4
:102350004FF42062DA801A8902F00F00042803D8B3
:10236000C2F30312022A02D940F601221A8195F81B
:10237000AD0695F8B92695F8AC36904205D90022FD
:1023800085F8AD2653B1A5F8B02695F8B8269A423F
:1023900004D2002385F8AC36A5F8B03695F8A237FC
:1023A00095F8AE26614ED7F800809A4284BF00238C
:1023B00085F8AE3606F18009334613F8032D02EB9B
:1023C0004202424492F854E192F855C192F8560103
:1023D00013F801AF9A79F245A8BFF2466245A8BF4B
:1023E00062469A71DA7883F800A08242A8BF02465A
:1023F000B342DA70ECD103F120064E45DCD14C4BF0
:10240000DA6A002A00F0FB80002601200B782B2BD3
:1024100007D14B78043300FA03F313421CBF9A43ED
:10242000012606318C42F1D10EB1414BDA62414CAA
:102430006E4604F10808234601E0434547D013F8EF
:10244000012F072AF9D9002304F8013F0133082B93
:10245000FAD1B5F8BE25B5F8BC359A42B54602D3D7
:10246000354BC5F8BC35354B354CFF2285F8D427A4
:1024700003F16C0013F9082C142A05D053F80C1C36
:1024800034EA010100F0C3800C339842F2D12D4BA5
:102490005A79022A01D100225A710C37BD46BDE893
:1024A000F08F2949294851F077F99DE502EBC301E6
:1024B000DB00496800297FF444AD254817210170ED
:1024C0003FE5244938E67C684946002229E788B080
:1024D000E9462022FF2148465DF0FCF9154A03E059
:1024E000424549F82330B4D012F8013F59F823107F
:1024F0000131F5D0A7E7002333714FF00108BBF19C
:10250000000F7FF4F1AE737C002B7FF417AF73796B
:10251000012B7FF413AF0DE7F4560020BCD75718FA
:1025200034620020D05B0020B465002091DC0020E4
:102530000C570020FE400020AE014A01E8E00020D8
:1025400001000200583E0020DCE00020203D080889
:10255000BC5B0020F6DFFFFDD45D0020F3400020CF
:10256000474AD17B00293FF4F7ADE004D3773FF52C
:10257000F6AD21067FF5F3AD424B1978182904D842
:10258000414BCB40DA073FF5EAADDFF80C8108F1AB
:10259000780401E6A3047FF5D7AD3C49CCE5B379D7
:1025A000002B3FF448AE737C012B04BF02237374ED
:1025B00041E600283FF42BAD90F904604FF0FF088E
:1025C00001E080F8088030460FF092FA0028F8D138
:1025D0001DE599F8000079600DF002FC796800288B
:1025E0007FF45EAEA9F804005AE62949A4E5294A19
:1025F00013431043C9F80030CAF8000049E62B2005
:10260000796025F071FF1E4B7968DA6AFCE685F87F
:10261000D4273CE7DAF8003023F48053CAF80030BE
:10262000338C24F48054B3F57A7FC9F80040BFF4AA
:102630005BAD4FF47A73338456E5D9F8003023F05C
:102640000063C9F80030DAF8003023F00063CAF8FC
:102650000030ABE5DFF844A0DAF8003024F0800465
:1026600023F08003C9F80040CAF80030D1E4DAF85A
:10267000003043F0080344F00804CAF800305AE57B
:102680000C570020BC5B002000410001F6BFFFFD9D
:10269000F79FFFFD0004050000E20020085700201E
:1026A0002DE9F04FDFF8EC816F4ED8F80C30DFF8F1
:1026B000E89103F2DC534E4583B0C8F80C3080F04B
:1026C000CF8001230193694BDFF8D0B106F11C05DF
:1026D0009F1C664B5988002900F0AD807A185A4536
:1026E00080F0A9803C4608E0118814460A4400297D
:1026F00000F0A1805A4580F09E80052940F29B8021
:1027000035F81C3C6188C3F30B039942ECD1637923
:102710009B07E9D155F8141C238894F804A0009372
:10272000304651F039F835F81C1CBAEB113F00F077
:1027300088800023019335F8181C55F8140C55F8BF
:10274000044CC1F30B0155F079FA1C364E4520605C
:1027500005F11C05BDD3464A464B474F474C12680E
:102760001A60FFF7DDFB3878454D7A78454EEA214F
:1027700004F5947300FB01332B6004F1A80303EB11
:102780004213C4F8F43425F081F84FF0FF33286881
:10279000736030F0B9FE25F0EFFE04F21C6304F222
:1027A000946102E00633994255D01A78002AF9D193
:1027B0009D78D878854202D358790028F2D094F8D1
:1027C0001436327203EB830303EB83039B00642B09
:1027D000B4F81826B8BF6423C8F80430642303FB98
:1027E00002F2642AB8BF64220023C8E90223C8F8B1
:1027F0002020254AA8F82430C8E90433C8E9063364
:1028000088F82630214B936233F0E8F9B4F8D80702
:1028100094F8DA1726F0BEFC42F006FA17F034F905
:102820001B4A01981268C8F80C20012388F825304B
:1028300003B0BDE8F08F55F8141C304650F0ACFFE3
:1028400077E7009BA11D9A1F304650F0DBFF002860
:102850007FF471AF6DE73A7C003A18BF0122AEE712
:102860000123019377E700BF643A0808004000089D
:10287000E066002008570020F4560020E4DB00202A
:102880002C620020A804002070620020E8E10020F3
:10289000A01A002044620020CC43080800800008F1
:1028A00038B50122184D84180328034685F8DC2723
:1028B000E4B217D9FF2825D0144A002341F202417F
:1028C00000E034B10233402B22F8021B04F1FF3444
:1028D000F7D11D44FF2385F8E037BDE838400E20CE
:1028E00011F0C4BF05F59470EA2203FB0200084909
:1028F000084A0860137030F007FE27F025F827F02B
:1029000007F9D9E70023E4E7E4DB0020C4E3002073
:102910002C620020F4560020054BD3F82428012116
:1029200042F4001283F82118C3F82428704700BF2E
:10293000E4DB00207047F8B5164D6B78BE2B26D12E
:10294000022229464FF6FF70FEF704FB124FAC1C23
:1029500022884AB1A618BE4219D2052A17D92146A3
:10296000FEF7F8FA3446F3E721460222FEF7F2FAC0
:102970000222A118FEF7EEFA0634084B641BA3F8F6
:10298000284841F60F53C31A58425841F8BD002059
:10299000FCE700BF0040000800800008E4DB0020E6
:1029A0002DE9F8430468C4F30A0906460F4604F10A
:1029B0007848B9F1000F16D0B8F5002F3B6834D233
:1029C000314D2A6942F001022A614FF480102360E0
:1029D00051F026FA2B6923F001032B6103282BD039
:1029E0006FF002002CE0B8F5002F16D2264D2B69AF
:1029F00043F002032B616C612B6943F040032B61B0
:102A00004FF0004051F00CFA2B6969F341032B6140
:102A10000328D1D04FF0FF3012E004F1774303F5E3
:102A20007803B3F5002F0DD30B6804F1774202F55C
:102A30007802B2F5002F18D33368043333600020D6
:102A4000BDE8F883104D2B6D43F002032B656C65D8
:102A50002B6D43F040032B654FF0004051F00AFA14
:102A60002B6D69F341032B65D2E7074D2A6D42F0C8
:102A700001022A654FF48010236051F0FBF92B6DA1
:102A800023F001032B65A9E7003C02402DE9F04348
:102A90005C4F3B78B12B8BB062D1FFF74CFF80F0DD
:102AA0000104E4B2584B594DB3F86331DFF870813B
:102AB000ADF8043004F00104454553D3002C00F078
:102AC0009F80534B5349544A0597DB1B0693534B46
:102AD0004E4D00260996CDE9076659605A60596443
:102AE0005A6401228DF825203422DA6001A90222DD
:102AF00005A88DF8246059F051F8022201A94FF67B
:102B0000FF70FEF727FA0446454538D3022202A992
:102B100005A80025ADF8085059F040F8022202A996
:102B20002046FEF717FA40BAC043ADF80C00022267
:102B300005A803A959F032F80898002849D1374B65
:102B40001A6942F080021A611A6D42F080021A6519
:102B50009DF92400B0FA80F040090BB0BDE8F08385
:102B600001249FE7A988AB69A8681E68C1F30B011F
:102B700055F064F81C35864218BF01249CE7AF88E5
:102B80008DF81160C7F30B07BB1DADF80C302B8817
:102B9000C3F30B02ADF80E201B0B062203A905A8F8
:102BA0008DF8103058F0FAFF062203A92046FEF7F0
:102BB000D1F9D5F8089004463A46494605A858F098
:102BC000EDFF20463A464946FEF7C4F91C35044657
:102BD0009AE707ABC0F10402294618445CF07AFE7C
:102BE0009DF9240018B907A905A8FFF7D9FE00230D
:102BF00008939DF825308DF82400002BA8D09EE77F
:102C00000120AAE700400008B4230708643A080836
:102C10000080000823016745AB89EFCD003C0240EE
:102C2000CC430808F8B5184D184E194FFFF778F93E
:102C3000EB68012203F2DC53EB6086F82A280324B8
:102C4000FFF724FF58B13B78B12B08D1FFF773FE93
:102C5000013C0BD060B9FFF719FF0028F3D1013C0C
:102C6000EED1052057F016F956F080FA0028F8D07A
:102C7000084A1168E9600122002385F8252086F8BA
:102C80002A3886F82B38F8BD44620020E4DB0020A7
:102C900000400008A01A002010B50B4A0B4C01237D
:102CA00084F8DC37D373FFF7BDFFFFF7F9FC41F27F
:102CB0000242FF23A4F8E02784F8E237BDE8104081
:102CC0000E2011F0D3BD00BFF4560020E4DB00203D
:102CD00090F89230DFED6B6A6B4A07EE903A90F80D
:102CE000963005EE103A90F8943004EE903A90F851
:102CF000953005EE903A90F89830F8EEE77AB8EE15
:102D0000C55A04EE103A67EEA67A25EE265AF8EE7A
:102D1000E44AF8EEE55AB8EEC44A25EE275A64EEC6
:102D2000A64A65EEA65A24EE264AF0B5B7EE007A1A
:102D300090F8917064EE854A65EEA75A24EE274A12
:102D400000F16F06014602F11A050024B0EE476A51
:102D5000B0EE473A137807EE903AF8EEE77A67EE6E
:102D6000857A67EE867AFDEEE77A17EE903AFA2BCF
:102D7000A8BFFA2323EAE3730B72537807EE903A65
:102D8000F8EEE77A67EEA47A67EE867AFDEEE77AE8
:102D900017EE903AFA2BA8BFFA2323EAE3734B729B
:102DA000937803EE903AF8EEE33A63EEA57A67EE95
:102DB000877AFDEEE77A17EE903AFA2BA8BFFA234E
:102DC00023EAE3738B72938807EE903AF8EEE77A82
:102DD00067EE847A67EE867AFDEEE77A17EE903A30
:102DE000B3F57A7FA8BF4FF47A7323EAE3738B813C
:102DF0002B68D5ED007A002BF8EEE77A3FDD90F8EE
:102E0000973002EE903AF8EEE22AB0EE436AA2EE74
:102E1000E66A63EE863A83EEA76AA2EEA66A0134FA
:102E200065EEA77A67EE877A67EE867AFDEEE77A37
:102E300017EE903AFA2BA8BFFA2323EAE373BC42B9
:102E400006F8013F00DDF0BD012C13D190F893305E
:102E500007EE103A90F89B3006EE103AB8EEC77ABB
:102E6000B8EEC66A27EE267A26EE266A04350832C0
:102E700008316FE7B7EE007AB0EE476AF6E7B7EED3
:102E8000006ACCE70AD7233C1A25070890F8993046
:102E90006BB3B0F864308BB190F89A2002EB8203E8
:102EA0006421C3EB0313B3FBF1F3A0F86430962362
:102EB00012FB03F3B3FBF1F3A0F8663043884BB188
:102EC00090F89A3003EB8303C3EB03136422B3FB44
:102ED000F2F34380B0F850304BB190F89A3096221C
:102EE00013FB02F36422B3FBF2F3A0F850307047F7
:102EF00090F821304BB3438B83B190F82230FA2203
:102F000013FB02F203EB8303B3F57A7FA8BF4FF400
:102F10007A7364218383B2FBF1F24283838843B1E5
:102F200090F82230FA2213FB02F36422B3FBF2F38F
:102F30008380C3884BB190F8223003EB8303B3F551
:102F40007A7FA8BF4FF47A73C380704770B50B4C7B
:102F5000002504F56A7694F8913013B12046FFF706
:102F6000B7FE2046FFF792FF01353046FFF7C0FF5E
:102F7000042D04F1EA04EED170BD00BF0CDD002089
:102F800010B5064C4FF48072002104F62C005CF062
:102F9000A1FC0023C4F82C3910BD00BFE4DB0020E5
:102FA000034BD3F8300908B109F0DEBE704700BF0B
:102FB000E4DB002008B50B4605490246D1F830098C
:102FC00028B10449FEF782FABDE80840E8E708BDE9
:102FD000E4DB0020590C0108024B0146D3F830090C
:102FE000FDF73CBEE4DB00200048F5E7A528080813
:102FF0000CB4C30607B500D561B9049805A90191C1
:10300000FFF7D8FFFFF7F0FF012003B05DF804EBF6
:1030100002B070470020F8E70FB407B504A951F8D3
:10302000040B0191FFF7C6FFFFF7DEFF03B05DF869
:1030300004EB04B070470349034801F5FD610EC974
:10304000EAE700BF00F0FF1FB413080870B5134C87
:10305000134D144E002294F8F33403F0010302B12F
:1030600070BD002BFCD001212846FFF7D5FF75204D
:1030700033F022FA01463046FFF7CEFF1A2033F034
:103080001BFA01460848FFF7C7FF1B2033F014FA6C
:1030900001460648FFF7C0FF0122DCE7E4DB002021
:1030A000C8130808D4130808E7130808FA13080817
:1030B00008B5FFF791FFBDE8084095E72DE9F0431B
:1030C00085B0FCF7B5FC02698389018802928268A9
:1030D00001924288009242681B4EDFF88080DFF840
:1030E00080901A4F04461A48FFF796FF002515B93D
:1030F0001848FFF7DDFFD8F800309D4213DA337827
:10310000052B96BF09EB83030022D3F88C21B388EB
:1031100000937388294638460135FFF77DFF062D59
:1031200006F10606E3D155F0D7F842888388646833
:103130009B1A03FB0444FCF713FD02460648214694
:1031400005B0BDE8F04367E718E5002077140808EC
:103150000D1408086B1408088614080898510020FC
:10316000B423070810B504460348FFF735FF20468F
:10317000BDE810409CE700BFA314080808B503464B
:1031800010460AB9002008BDDB0601D50029FAD097
:10319000FFF7E8FFF6E72DE9F04F0A468DB0002172
:1031A0008346FFF7EBFF714CDFF8CC91039004F1FD
:1031B000800A0025A37A99F80060AB4200F393805F
:1031C00010345445F5D140F2162050F0CFFAD0E932
:1031D00002450DF1180A002E4FF015024FF00001C4
:1031E000504604BF254634465CF074FB00272E7819
:1031F000002E3ED06978059130460CF0C9FD95F956
:103200000290049009F1010253425341002C00F056
:10321000A98005990022A05CB04240F09F80224422
:1032200092F90280C14540F0978052788A4208BFE7
:10323000012301220AF8072003F0010383F00101B2
:10324000039A05935846FFF799FF059B039044B1F5
:10325000474A0499CDE900B230464246FDF7EAFDFF
:10326000059B444A0499CDE900B230464A46FDF731
:10327000E1FD0137152F05F10305B8D184B3DFF85F
:10328000F080DFF8F090564604F13F0716F801ABE6
:10329000BAF1000F21D12078F8B194F9023001334E
:1032A0001BD061780CF074FD039A05460121584645
:1032B000FFF764FF94F902200390534620782946D3
:1032C000CDE900B8FDF7B6FD20785346CDE900B949
:1032D0004FF0FF322946FDF7ADFD0334BC42D5D196
:1032E0000DB0BDE8F08FE08850F040FAD0E902312F
:1032F000627A207A002E08BF194605FB002208BF1B
:1033000033468F562BB39E56039A0493B74214BF8D
:103310000121002158460CBF4FF001084FF0000872
:10332000FFF72CFF049B039043B1114B3246CDE9CC
:1033300000B3294643462046FDF738FD0D4B29468C
:10334000CDE900B33A4643462046FDF72FFD01354F
:1033500030E74FF0FF36D7E700236AE703323F2A12
:103360007FF459AF4FF0FF3868E700BFB404002086
:10337000F5340108F12F0108E4DB002010B5084600
:103380000749FDF7A1F9002815BF012400240548CD
:103390000548FFF7E7FE2046BDE8104009F0BEBA39
:1033A000A8140808B1140808D81408082DE9F04F2B
:1033B00007468BB040F216200C4650F0D7F9224653
:1033C000054600213846FFF7D9FE424BD5E90245B4
:1033D0001B78002B08BF254606464FF015024FF01C
:1033E000000104A808BF1C465CF074FA05F13F0315
:1033F000039395F80090B9F1000F31D095F801A032
:10340000002C65D0224600231178494558D1283335
:103410006B4492F80180012203F8182CD045324603
:1034200014BF0121002138460CBF4FF0010B4FF0B3
:10343000000BFFF7A3FE064654B1B8F1000F07D00A
:10344000254B00935A463B4641464846FDF73AFD18
:10345000224B00935A463B4651464846FDF732FD03
:10346000039B03359D42C4D13CB3DFF86C90DFF879
:103470006CA0651C0DF11008403418F8013BCBB965
:1034800015F8013CB3B116B13046FFF76BFE297851
:1034900015F8010CCDF800903B460022FDF712FD17
:1034A000002215F8010CCDF800A03B461146FDF7AF
:1034B00009FD00260335A542DFD10BB0BDE8F08F32
:1034C0000133152B02F103029ED14FF00008A5E74E
:1034D000A046A3E7E4DB0020F5340108F12F010842
:1034E000034B0146D3F8300908B109F029BC7047F5
:1034F000E4DB00200CB407B510F020000BD079B944
:103500002320FFF7EDFF049805A90191FFF752FD75
:10351000FFF76AFD012003B05DF804EB02B07047CD
:103520000020F8E72DE9F04F914687B00C461A4687
:1035300000218046FFF722FE4D4606460027B9F1DE
:10354000000F66D02946062220465CF047FA002884
:10355000324614BF0121002140460CBF4FF0010A42
:103560004FF0000AFFF70AFE0646287816F054FAD4
:103570008346F8B1687916F04FFAAB78EA789BF891
:1035800005E095F801B04FF461714FF0190C1CFB88
:1035900003131CFB0212297900B14079CDE9041014
:1035A000CDE90232CDE900EB1B4A3B46514640468D
:1035B000FFF7A0FF207816F02FFA8346F8B1607964
:1035C00016F02AFAA378E2789BF805E094F801B0A7
:1035D0004FF461714FF0190C1CFB03131CFB02121A
:1035E000217900B14079CDE90410CDE90232CDE96D
:1035F00000EB094A3B4651464046FFF7F9FC0137CC
:10360000142F04F1060405F1060598D107B0BDE8B2
:10361000F08FCA46CEE700BFF41408082DE9F04F3A
:10362000904689B01A460C4600218146FFF7A6FD58
:103630003B4EDFF8F0B008F16C03074645460793B0
:1036400094F904000EF054FA00285DD0B8F1000F90
:1036500063D029460C2220465CF0C0F900283A4687
:1036600014BF0121002148460CBF4FF0010A4FF062
:10367000000AFFF783FD074695F9040053F06CFB41
:10368000EA7906EB82020346D2F8A42104922A7A50
:1036900006EB82025146D2F8A4210392AA7906EBE6
:1036A00082024846D2F8A42102926A7906EB82028D
:1036B000D2F8A42101922A6800925A46FFF71AFF15
:1036C00094F9040053F048FBE27906EB82020346CA
:1036D000D2F8A4210492227A06EB82025146D2F853
:1036E000A4210392A27906EB82024846D2F8A421D3
:1036F0000292627906EB8202D2F8A421019222683A
:1037000000925A46FFF774FC079B0C35AB4204F15C
:103710000C0495D109B0BDE8F08FC246D0E700BFD8
:10372000B42307080D1508082DE9F04F90468BB01B
:103730000C461A4600210746FFF720FD4546099032
:1037400000264FF0190A4FF46179B8F1000F4BD001
:1037500029460A2220465CF041F90028099A14BF44
:103760000121002138460CBF4FF0010B4FF0000B38
:10377000FFF704FD2A890692EA8805922A790492C5
:10378000EA780392AA7809901AFB029202926A7868
:103790001AFB029201922A7800923346134A594644
:1037A0003846FFF7A7FE22890692E2880592227921
:1037B0000492E2780392A2781AFB02920292627853
:1037C0001AFB0292019214F80A2B00923346074A20
:1037D000594638460136FFF70BFC1E2E05F10A0547
:1037E000B3D10BB0BDE8F08FC346DCE72A1508085B
:1037F0002DE9F04F2DED088BDFF828A195B080461C
:1038000091461E460C461546002794ED008AB5EEFB
:10381000408AF1EE10FA7DD0D4ED019A94ED029A2F
:10382000D4ED038AB9F1000F49D0D5ED00BA95ED7A
:1038300001BAD5ED02AA95ED03AAB4EE6B8AF1EEBA
:1038400010FA6CD1F4EE4B9AF1EE10FA67D1B4EEA7
:103850006A9AF1EE10FA62D1F4EE4A8AF1EE10FAA9
:103860000CBF0121002132468B46404681F0010108
:10387000FFF784FCB0EE6B0A064611A8FDF77CF951
:10388000B0EE4B0A07900EA8FDF776F9B0EE6A0A83
:1038900006900BA8FDF770F9B0EE4A0A059008A84B
:1038A000FDF76AF90599069A079B03900291019228
:1038B000009352463B4659464046FFF71BFEB0EE8A
:1038C000480A11A8FDF758F9B0EE690A83460EA818
:1038D000FDF752F9B0EE490A06900BA8FDF74CF936
:1038E000B0EE680A059008A8FDF746F9069B059A10
:1038F0000390CDE900B302923B4652460021404678
:103900000137FFF775FB082F04F1100405F11005CE
:103910007FF47BAF15B0BDEC088BBDE8F08F0021C4
:10392000A1E700BF4D1508082DE9F74F92460C4658
:103930001A4600218146FFF721FCDFF870B080466F
:1039400056460025BAF1000F2ED0314604222046FB
:103950005CF044F80028424614BF0121002148468B
:103960000CBF01270027FFF709FC738801933AF881
:103970002530009380462B465A4639464846FFF785
:10398000B9FD6388019334F8043B00935A462B46F3
:10399000394648460135FFF72BFB042D06F1040696
:1039A000D0D103B0BDE8F08F5746EAE761150808AB
:1039B0002DE9F04F89468FB0174600211A4606467A
:1039C000FFF7DCFBDFF874A0054600240DF1240BA3
:1039D00059F82480CDF80880594602A853F06AF9B6
:1039E00057B357F82430039398452A4614BF012152
:1039F000002130460CBF4FF001084FF00008FFF7E0
:103A0000BDFB04A9054603A853F054F904A900918D
:103A10002346524641463046FFF76CFD2346CDF81B
:103A200000B05246414630460134FFF7E1FA202CFF
:103A3000CED10FB0BDE8F08FB846EFE77215080899
:103A40002DE9F04F924685B00C461A46002181467A
:103A5000FFF794FBDFF874B0804655460026BAF1B4
:103A6000000F31D02946042220465BF0B7FF002822
:103A7000424614BF0121002148460CBF0127002700
:103A8000FFF77CFBEB780293AB7801932B880093D4
:103A9000804633465A4639464846FFF72BFDE378C1
:103AA0000293A378019334F8043B00935A463346BB
:103AB000394648460136FFF79BFA102E05F10405FA
:103AC000CDD105B0BDE8F08F5746E8E77C15080872
:103AD0002DE9F04F85B0144602911A4600210546A3
:103AE000FFF74CFB4FF000080646062303FB08F7E0
:103AF000C0374FF00009029B13F807B0002C7ED0AE
:103B0000E35D03939B45324614BF01210021284603
:103B10000CBF4FF0010A4FF0000AFFF72FFB039B89
:103B2000394ACDE900930646434651462846FFF7F9
:103B3000E1FCCDE9009B344A43465146284609F151
:103B40000109FFF755FAB9F1060F07F10107D2D1C4
:103B500008F10108B8F1060FC7D1E427029BA7F1CD
:103B6000E40913F807A0002C4BD014F807B0DA458D
:103B7000324614BF0121002128460CBF4FF0010836
:103B80004FF00008FFF7FAFACDE9009B06461E4AFF
:103B9000062341462846FFF7ADFCCDE9009A1A4AB4
:103BA0000623414628460137FFF722FAEF2FD5D1E9
:103BB000029B93F8EF70B4B194F8EF80474532461A
:103BC00014BF0121002128460CBF01240024FFF767
:103BD000D5FA002300930C4ACDF804800723214630
:103BE0002846FFF787FC00230093074A0197072325
:103BF00021462846FFF7FCF905B0BDE8F08FA24644
:103C000097E7A046C9E700BF8E1508082DE9F04FD9
:103C10000E46154689B01A4600210446FFF7AEFA53
:103C2000B04681462F464FF0000B002D7CD0394620
:103C30000C2240465BF0D2FE00284A4614BF012108
:103C4000002120460CBF4FF0010A4FF0000AFFF799
:103C500095FA97F90B20049297F90A200392B7F985
:103C600008200292B7F906200192B7F904200092C9
:103C70008146384A5B4651462046FFF73BFC98F99F
:103C80000B20049298F90A200392B8F908200292B6
:103C9000B8F906200192B8F9042000925B462D4A3B
:103CA000514620460BF1010BFFF7A2F9BBF1080FBB
:103CB00008F10C0807F10C07B7D1DFF89C804FF032
:103CC000000B0C2303FB0BF985B3002755F8090003
:103CD00056F80920012303FA07FA42403AEA0202A1
:103CE00014BF1946002110EA0A0F07D000975B465F
:103CF000424620460791FFF7FDFB079956F8092039
:103D00001AEA020F05D000975B4642462046FFF7AD
:103D10006FF901370E2FD9D10BF1010BBBF1080F51
:103D2000CFD109B0BDE8F08FAA46A8E72F4656F8D4
:103D30000910012303FA07F20A4206D000975B46F6
:103D4000424601212046FFF753F901370E2FEED1ED
:103D5000E2E700BFA2150808BA1508082DE9F04FE0
:103D600089468DB0164600211A460746FFF706FA27
:103D7000DFF8DCA005460024C4EBC40309EB030212
:103D800059F8030091889279089040F30748ADF8FC
:103D900024108DF82620B8F1000F54D0002E55D0F5
:103DA000F218F058918893790A90ADF82C100722F8
:103DB0000AA908A88DF82E305BF010FE00282A46CC
:103DC00014BF0121002138460CBF4FF0010B4FF00A
:103DD000000BFFF7D3F99DF82E3006939DF92D3097
:103DE00005939DF92C3004939DF82B3003939DF996
:103DF0002A3002939DF8293001939DF828300093D2
:103E000005462346524659463846FFF773FB9DF850
:103E1000263006939DF9253005939DF924300493AF
:103E20009DF82330CDE902839DF8213001939DF860
:103E30002030009352462346594638460134FFF756
:103E4000D7F8102C98D10DB0BDE8F08FB346DEE75F
:103E5000CF1508082DE9F04F924689B00C461A4656
:103E600000210746FFF78AF9002607905546B3461A
:103E70004FF019094FF46178BAF1000F28D02946A4
:103E8000062220465BF0AAFD0028079A14BF0121F4
:103E9000002138460CBF4FF0010B4FF0000BFFF72D
:103EA0006DF96A79079019FB028205922A7919FB4C
:103EB00002820492EA780392AA7802926A780192C6
:103EC0002A7800923346124A59463846FFF712FBC9
:103ED000627919FB02820592227919FB028204920F
:103EE000E2780392A27802926278019214F8062B8B
:103EF00000923346064A594638460136FFF778F8AD
:103F00000A2E05F10605B7D109B0BDE8F08F00BF54
:103F1000EC1508082DE9F04F0F468BB01446002130
:103F20001A460646FFF72AF90546002C00F0DD8008
:103F300022783B789A4218BF0121024608BF00212F
:103F400030460CBF4FF001084FF00008FFF716F99C
:103F500023789E4A054641463046FFF7CBFA3B7828
:103F60009A4A41463046FFF743F8002C00F0BF80E4
:103F700062787B789A4218BF01212A4608BF002147
:103F800030460CBF4FF001084FF00008FFF7F6F87D
:103F900063788F4A054641463046FFF7ABFA7B7897
:103FA0008B4A41463046FFF723F807F1C9030593D2
:103FB000A31C0693822307F1020A04F1CA0B07939C
:103FC0004FF000093B784B4500F39380002C00F044
:103FD000F68097F8EA3094F8EA209A4218BF012157
:103FE0002A4608BF002130460CBF4FF001084FF0B1
:103FF0000008FFF7C3F894F8EA30764A05464146D0
:104000003046FFF777FA97F8EA30724A4146304671
:10401000FEF7EEFF002C00F0D48004F1EA0307F174
:10402000EA0204F1FA014FF0010833F802CF32F846
:10403000020F844518BF4FF000089942F5D188F06F
:1040400001012A46C9B23046FFF798F80821054613
:1040500004F1EC00FDF7CEFB5F4A034641463046D3
:10406000FFF748FA97F8EA1007F1EC00FDF7C2FBFA
:10407000594A034641463046FEF7BAFF002C00F08D
:10408000A2804FF0FC094FF0010807EB090104EB97
:104090000900FCF719FB09F10409002818BF4FF0CB
:1040A0000008B9F58E7FF0D188F001012A46C9B227
:1040B0003046FFF763F8082104F1FC00FCF748FEE6
:1040C000464A034641463046FFF714FA97F8EA108D
:1040D00007F1FC00FCF73CFE404A034641463046EF
:1040E0000BB0BDE8F04FFEF783BFA04637E7A04610
:1040F00055E7079BFB180993002C5ED0079B099896
:10410000E31819460893FCF7DFFA059B5A789BF8E9
:1041100000309A42069A06BFB0FA80F84FEA581863
:104120004FF00008AAF10203023A0AF10E0133F837
:1041300002CF32F8020F844518BF4FF000088B42BF
:10414000F5D188F001012A46C9B23046FFF716F8CA
:104150006278069905469BF81800FDF71DFB029052
:104160009BF800300193089B00931D4A09F101035D
:1041700041463046FFF7BEF9059B7A78587E514696
:10418000FDF70AFB059A029012F8013F019309F12D
:104190000109099B05920093114A4B46414630465E
:1041A000FEF726FF069B10330693079B09330AF19F
:1041B000100A0BF1010B079304E7A046DCE7A046C9
:1041C00021E7A0464EE7A04680E700BF0516080895
:1041D00017160808451608085D160808741608081A
:1041E0002C1608082DE9F04F89B00F4690460021A3
:1041F000139A03930646FEF7C1FF87EA08086FEAA1
:104200000803DFF8849006930446002528460DF045
:104210000DFC129B184230D0069BDFF870B00340B3
:1042200014BF4FF0010A4FF0000A049310EA07038D
:104230000CBF4A465A462846059307920DF008FCE3
:10424000039B079A0090804651463046FFF752F98B
:10425000049BB3FA83F1224649093046FEF78EFFEC
:10426000059A039BCDF800800446002A0CBF5A46ED
:104270004A4651463046FEF7BBFE0135172DC5D1E3
:1042800009B0BDE8F08F00BF8B1608085B15080861
:104290002DE9F04F0A4689B000210546FEF76EFF72
:1042A000384C059094F9000009F0D0FA81466088F6
:1042B0004FF05CFA344BD0F808B01F7817B15F4666
:1042C000D0F80CB0A379012B38BF01230693002648
:1042D0002279637906FB02331BF80380002F3BD061
:1042E000FB5C059A0793434514BF01210021284632
:1042F0000CBF4FF0010A4FF0000AFEF73FFF079B8B
:104300000590013653B303F00F021B094033CDE98A
:10431000006302924B461D4A51462846FFF7EAF8D1
:10432000B8F1000F24D008F00F034FEA18180293D9
:1043300008F14003CDE90063144A4B465146284634
:10434000FEF756FE069BB342C2DC114B0834A34273
:10435000A8D109B0BDE8F08F3B46C2E7002FDFD0FF
:104360000C4A00964B4651462846FFF7C3F8D7E75C
:104370006B06E7D4074A00964B4651462846FEF79F
:1043800037FEDFE798250708E4DB002092160808CF
:10439000D0260708A81608080FB407B504A951F8D5
:1043A000040B0191FEF706FE03B05DF804EB04B0C8
:1043B00070472DE9F041037903F0E002402A4DD027
:1043C00009D83ABB03F00703052B1ED8DFE803F03A
:1043D000181D181D0910602A47D0802A41D0BDE859
:1043E000F081D0F805102348BDE8F041FEF714BE77
:1043F000D0F8052051422048BDE8F041FEF70CBE40
:10440000B0F80720B0F80510F5E7B0F90720B0F9CB
:104410000510F0E74679194D194805EBC605FEF77A
:10442000DBFD95F8207300240123A74203D8BDE8E3
:10443000F041FEF7D9BDD5F81C6356F824204FEAA9
:1044400084084AB113B90F48FEF7C6FD56F80810A4
:104450000D48FFF7A1FF00230134E6E741790B483F
:10446000C2E7827941790A48C6E7BDE8F0410948C8
:10447000FEF7D2BDBC160808D2160808B4230708F8
:10448000E91608086E1808085B2D0808FA160808CF
:104490000B17080822170808194B1B682DE9F04173
:1044A00063B31848184FDFF86880FEF701FEFEF787
:1044B00077FDFBF7CDFA0025FBF70AFB044648B170
:1044C000132010F0D3F9FEF78FFDBDE8F0410F483F
:1044D000FEF7EEBD3B78012BF2D04046FFF75CFFC4
:1044E000792D05F1010602D1FEF77EFD2646FEF785
:1044F00057FD6420F5F7AEFF3546DDE7BDE8F081F6
:104500004C3100203A170808A2510020541708081F
:10451000252E08082DE9F047BC4BBD4C1A68BD4953
:10452000BD4BBE48B2FBF3F290B0FFF735FFB4F8D5
:104530005829BB4DBB4F4FF47A73B2FBF3F103FB29
:1045400011220A20B4F95A3992B2B2FBF0F2B648FD
:10455000FEF762FDB54AB649B648FFF71DFFFEF704
:1045600043FDB54BB54AD97BB54BB64805EB810148
:10457000D31AD1F8E414B4F82828FEF74DFDFEF75D
:1045800033FDB148FEF728FD94F85C19AF48FFF7FA
:1045900003FFAF48FEF720FDAE4B94F85D191A8873
:1045A000AD4892B2FFF7F8FEFEF71EFDAB49AC48EE
:1045B000FFF7F2FE4FF000084646DFF8249394F828
:1045C000EF3403F00103B8F1000F00F0E880002E93
:1045D00040F01981A348FEF76BFDA34FD4F864891E
:1045E000DFF80093012607F1180A0123B34013EA0C
:1045F000080F14D019F8062057F826305AF826105C
:1046000053F822209948FFF7C7FE012E05D194F8F0
:10461000851911B19648FFF7BFFEFEF7E5FC01369C
:10462000062EE2D19348FEF7D7FC934B1B681B067E
:1046300040F18B8194F8F039032B8CBF8F48904860
:10464000FEF7CAFC94F86C35022B40F04D818D4882
:10465000FEF7C2FC94F8F039042B00F26D818A4811
:10466000FEF7BAFC94F8003A002B00F06C8105EBE1
:10467000C303D3F888158548FFF78EFEFEF7B4FC18
:10468000834B84481E68844B1B7805EB8303D3F867
:10469000BC15FFF781FE26B1327A717A7F48FFF7A9
:1046A0007BFEFEF7A1FCFBF7C3F9016921B182682B
:1046B0007B48120DFEF7B0FCFEF796FC794B7A486A
:1046C00019684FF47A73B1FBF3F1FFF765FE05A8A3
:1046D000FDF7EAFA38B105A908A857F027FD734895
:1046E00008A9FFF759FEFEF77FFCD4F88C8AB8F1D1
:1046F000000F00F02E8107EE908ADFED6D6AB8EEB4
:10470000E77AC6EE877AFDEEE77A17EE903A694FC0
:1047100097F8CC0130B1684A039392ED250A5AF01C
:1047200025F8039BD4F80C6A5EB107EE906ADFEDC2
:10473000606AF8EEE77A86EEA77AFDEEC77A17EEA2
:10474000906AB7F8CE116429A8BF6421CDE90006AC
:1047500042465A485A4EFEF75FFCB7F8D0215948F6
:104760006423B2FBF3F103FB112297F8E13105EB6F
:10477000830592B2D5F8D035009397F8E031FEF773
:104780004BFC5148FEF728FCD4F824480125002CA6
:1047900040F0E180FEF728FC10B0BDE8F087002B68
:1047A0003FF415AF16B14846FEF716FC4748012105
:1047B000FFF7F2FD94F86039414805EB8303D3F825
:1047C000EC14FFF7E9FD97F87E33DA0702D540488D
:1047D000FFF7E2FD97F8C830032B09D03D48FFF7FB
:1047E000DBFD97F8C830012B02D13B48FFF7D4FD21
:1047F000FB6C5B7B0126B342B0467FF6E0AE3748E8
:10480000FFF7CAFDD9E6FEF7EFFBE6E6F000002071
:10481000E4DB00206217080840420F006C1708080C
:10482000B4230708885E00207E170808F0FF0220E6
:1048300000080000A0170808F456002000800008B7
:1048400000400008B2170808C9170808DB17080855
:10485000E3170808CC500020E5170808F9170808E6
:10486000FE1708081D1808080829070880250808E9
:104870002218080826180808085700202C180808CD
:104880003818080848180808A53008088C180808BF
:1048900030660020A81808082C660020B118080807
:1048A000BB180808A01A0020D6180808F018080835
:1048B00000247449DCEC0020A80400200319080837
:1048C00098180808491908086E19080803180808F4
:1048D000571D0808081808081018080815180808AF
:1048E0006E1808083405002002200FF07FFE0646EF
:1048F00008B92048ACE690F9040052F02DFA0746BA
:1049000040F07CF905EB80003946D0F8A4211A4824
:10491000FFF742FD94F86F35012B04D11748FEF7DD
:104920005BFB174894E6B379164805EB8303D3F88D
:10493000A411FFF731FDF4E794F86E350BB9124876
:104940008EE612488CE6124995E61248FEF744FBC3
:1049500094E64346DBE694FAA4F0B0FA80F005FA58
:1049600000F024EA00040DF049F801463046FFF754
:1049700013FD0CE74E1808085818080868180808AE
:104980006D18080826150808711808088118080805
:104990005A1708089C1808082DE9F04FDFF87081B5
:1049A00098F8033099B0002B00F094804F48504E97
:1049B000DFF860B1DFF86091DFF860A1FEF778FB07
:1049C00000252F460BA9E8B215F0DAFA9DF834302D
:1049D000002B53D0139C54B107EE904A9FED450A2B
:1049E000F8EE677A80EE270A59F0C0FE04460B9A6B
:1049F00029465846FFF7D0FC109A002A6CD002FBDB
:104A000004F04FF47A73B0FBF3F30993DDF848C078
:104A1000BCF1000F62D00CFB04F142F21073B1FB49
:104A2000F3F198F80330082D18BF7F18002B57D0EA
:104A30001798079015980690169805900A231198D4
:104A40004FF47A7EB0FBFEFE0998CDF810E0B1FB82
:104A5000F3FE03FB1E11CDE902E10999B1FBF3F16D
:104A600003FB1100CDE90010BCFBF3F321465046D7
:104A7000FEF7D2FA0023C6E90D33B3620135232DC8
:104A800006F140069ED198F8033003B31A4C1B4838
:104A9000D4E979124FF47A73D208B1FBF3F3D4F866
:104AA000EC11FEF7B9FA0A22154897FBF2F102FB66
:104AB0001172FEF7B1FA134B1B78432B04D1D4E9E2
:104AC0007C211148FEF7A8FA0023C4F8EC3119B094
:104AD000BDE8F08F0D486AE7099297E76146A0E7C5
:104AE00021464846FEF798FAC4E700BF8419080833
:104AF000E8E500208096184BDCEC00202B1A080813
:104B00004B1A0808263A00206F1A0808E21908080C
:104B1000F4560020EC190808051D0808FB190808C0
:104B200010B586B0104B0493104B0393104B0293B7
:104B3000104B0193104B1149114A00930446114B3D
:104B40001148FFF729FCFEF74FFA10491048FEF70D
:104B500063FA3CB10F4A1049104806B0BDE8104056
:104B6000FEF75ABA06B010BDCF1A0808D41A0808C2
:104B7000DE1A0808E71A0808F31A0808991A08083C
:104B800062170808FB560020A41A0808FD1A080836
:104B9000051B0808161B08081E1B0808221B08080E
:104BA0000120BDE770B5224C2248FEF715FA94F8B3
:104BB000CC31002B37D0204B93ED250A59F0D6FD90
:104BC00001461E48FEF728FA1D4D1E48FEF704FA5E
:104BD0001D4B95F821001D4A00280CBF10461846B1
:104BE000FEF766FA95F821300BB3B4F88A1218482C
:104BF000184E194DFFF7D0FB94F8880200280CBF1F
:104C000030462846FEF754FAB4F88C121348FFF7E2
:104C1000C3FB94F8890200280CBF30462846BDE843
:104C20007040FEF745BA0E48FEF742FACCE770BD79
:104C3000DCEC00205F1B0808A8040020791B080892
:104C40000C570020881B0808371708080736080883
:104C5000991B0808581B08084F1B0808C01B0808A8
:104C60007E1B080838B50B4D05EBC0050C4695F9C1
:104C7000E40108F0EBFD01460748FFF78DFB95F8CE
:104C8000EA3133B1611C0548BDE83840C9B2FFF7CD
:104C900083BB38BDB42307085B2D0808F634080829
:104CA0002DE9F04F6B4B1B7887B0002B00F0CB80C9
:104CB000694D6A48A968FEF7AFF969686848FEF768
:104CC000ABF9684B6848D3E90031C91A674B1A68D9
:104CD000B1FBF2F2FEF7A0F9FEF786F96448FEF7A1
:104CE000E7F96448FEF7E4F94FF00008624B1B78DF
:104CF0005FFA88F4A34222D8FEF776F95F4D604E42
:104D0000002455F8041F30460134FFF745FB162CEC
:104D1000F7D1FEF769F95B4D594E01242B466968BE
:104D20001B683046C91A0134FFF736FB162C05F113
:104D30000405F3D107B0BDE8F04FFEF755B9524B6B
:104D4000142603EB840306FB045693EDA60AB6F87B
:104D50000E9059F00BFD96F81EA01AF0010F0CBF33
:104D60002D2252221AF0020F0CBF2D2354231AF0C9
:104D7000040F0CBF4FF02D0C4FF0560C1AF0080F1B
:104D80000CBF4FF02D0E4FF0430E81B21AF0800F82
:104D90004FF03C0BB1FBFBF105914FF064010CBFF0
:104DA0004FF02D0A4FF0530A80B201FB09F1671C46
:104DB000CDE902A10490CDE900CE34483946FFF791
:104DC000EBFAB37FDB073AD55C23314A6343D11852
:104DD000D05891ED010A70B1DFED2E7AB8EE400A9D
:104DE00020EE270A07EE900AF8EE677A80EE270A8F
:104DF00059F0BCFC00B2642290FBF2F102FB1102FC
:104E00002548FFF7C9FA142101FB075701FB045499
:104E1000F988628A0491218B0391E18A0291A18B26
:104E20000191A18A009102F0030319214B431B4811
:104E3000218A9208FEF7F0F808F1010856E71848B1
:104E4000FEF7CAF8DFE7174807B0BDE8F04FFEF7F6
:104E50002FB900BF2C1D0020183D0020E01B0808C2
:104E6000F01B08084C3E0020071C0808A81A002068
:104E7000341C0808901C0808D05B0020C03D0020AE
:104E8000401D0808C43D0020DCEC0020EC1C080894
:104E9000383A002000401C46091D08081E1D08085D
:104EA000151D0808441D08080EB403B503AA52F8DE
:104EB000041B0192FCF72DFC064BD3F830291AB9DC
:104EC0000549986CFBF7CAFE02B05DF804EB03B02D
:104ED000704700BFE4DB0020A52808082DE9F04753
:104EE00098460B7903F0E005402D81460F461646A3
:104EF00032D1644DDFF8A881DFF8B091002416E0CC
:104F00003B7903F00703013B042B04D8DFE803F0EF
:104F100014171A1D2100315D5A48FFF73DFA7B79BD
:104F2000013BA34202DD4846FEF756F801347B7987
:104F3000A342E5DCBDE8F08731572846EDE736F8B7
:104F40001410FAE736F91410F7E756F82410404623
:104F5000E3E756F82410F0E703F00703052B57D8D2
:104F6000DFE803F0031F27292C3E3478602D55D04D
:104F70002CD8002D75D1B7F80550B7F80760414817
:104F80002146FFF709FAAC4239DBB44237DCB8F10D
:104F9000000FCFD0324629463B48BDE8F047FFF727
:104FA000FBB996F90040602D38D00FD8002D58D1AC
:104FB00051E03488DAE7B6F90040F4E7D6F800A00B
:104FC000202D54464DD034D9602D27D0802DB1D11D
:104FD00032782E4B2E48002A14BF3146194635E050
:104FE000202D34683DD0EFD821462648FFF7D4F96C
:104FF000D7F80510A14202DB4B42A34221DDFDF7A9
:10500000F3FF3A68234923464846BDE8F0474BE79B
:10501000202D25D01ED9602DD8D100247B7944FACB
:1050200003F3DB07BDE8F0474CBF1B481B48FFF705
:10503000B3B951461A48FFF7AFF9D7F805108A45BA
:10504000DDD8B8F1000F3FF475AF1648BDE8F04762
:10505000FFF7A2B90024B7F90550B7F907608EE74A
:1050600000247A79104B03EBC20393F82023A24269
:10507000C5DDD3F81C3353F82400BDE8F047FDF735
:10508000ABBF00BFF7340808E51508080E2F080865
:105090005B2D0808661D080837170808073608083A
:1050A000CF160808601D0808B4230708E31708088E
:1050B0002DE9F04F164685B0CDE901011A460021D1
:1050C0003046FEF75BF8314C009006F010034FF0CD
:1050D0000009A2460393FDF763FF2379029A03F0C8
:1050E0001803934203D0002A44D1182B42D14FF029
:1050F0000D0B0BFB09A3B3F809004EF037FB8046FC
:105100002046FBF7B3FCD8E90221074602440144DC
:105110002046FBF743FC80F00101009A0546C9B226
:105120003046FEF72BF8039B009003B115BB0BFB39
:1051300009FBB3065AF80BB00ED56DB914485946A1
:10514000FFF72AF9D8F8082001982B463A4421465F
:10515000FFF7C4FEFDF748FF0E485946FFF71CF95C
:10516000D8F80C20019800233A442146FFF7B6FEF8
:10517000FDF73AFF09F1010940F27B23994504F15B
:105180000D04A8D105B0BDE8F08F00BFC4320708F8
:10519000801D0808811D080870B50546084616469A
:1051A0000C46FBF76BFD3346024621462846BDE818
:1051B000704093E60EB403B503AA52F8041B0192A3
:1051C000FCF7A7FA044B0549986CFBF747FD02B0C2
:1051D0005DF804EB03B07047E4DB0020A528080865
:1051E0000049E7E78B1D080838B50C460546154908
:1051F0002046FBF769FA30B9FDF7A8FE1248BDE872
:105200003840FDF755BF11492046FBF75DFAA0B9BC
:105210000F4B83F8B90183F8C10183F8A30283F827
:10522000AB0283F88D0383F8950383F8770483F842
:105230007F0483F8F1040748E1E72846BDE83840D9
:10524000CEE700BF9A1D0808A01D0808BB1D08086E
:10525000E4DB0020C31D08080049ABE7DF1D080898
:10526000F8B5064608460C46FCF752FC20210546D8
:1052700020465AF046FB044618B93046BDE8F840CF
:10528000EAE7124F124E3B7832789A4204F1010459
:1052900001D0FAF759FD0F4B20461D6057F0CCFBAB
:1052A000012201462046FAF7F7FC3B7832789A4211
:1052B00001D0FAF749FD204657F0BEFB2A460146C9
:1052C000BDE8F8400448FDF7A7BE00BF4831002004
:1052D000A351002044310020F61D08082DE9F041BB
:1052E000064688B008460D46FCF712FC202104460D
:1052F00028465AF006FB20B9304608B0BDE8F04118
:10530000AAE7FCF705FC2246054601460F48FDF7D3
:1053100083FE85B1202D2A46694628BF20222046DB
:10532000FAF75AFDE84606460027B74208DBAD1BF0
:105330003444002EEDD1FDF757FE08B0BDE8F081F2
:1053400018F8010BFEF7CCF80137EEE70C1E080841
:105350002DE9FF47074608460D4657F06DFB082824
:1053600045D105F1FF3801AE073531464246B14619
:1053700012F8010FFCF7EAFAAA4201F8010BF7D183
:105380000023DFF87CA08DF80C30A84517D11B490D
:1053900048462FF005FC19481949082310F8012B3D
:1053A00011F8014B10326A44013B02F80C4CF5D164
:1053B00014488DF80C3001A9FDF72EFE14E018F802
:1053C000010FFCF7C3FA06F8010B044601465046EC
:1053D0005AF097FA28B1214630465AF092FA00283E
:1053E000D3D03846FFF7FCFE04B0BDE8F0870028B4
:1053F000D1D0384604B0BDE8F0472DE70C57002067
:105400002CAD0708241E080807B5009313460A466A
:105410000249FFF7CFFE03B05DF804FB2B1E08081E
:105420002DE9F04FDFF8A4828BB006460D462846E2
:1054300057F002FB034638B99649024601200BB0EB
:10544000BDE8F04FFEF78ABC934905222846FCF7D9
:1054500083FA0446C8B9914D0146702205F52E70B5
:105460005AF038FAC5F82843C5F83443C5F8404324
:10547000C5F84C43C5F85843C5F86443C5F87043B4
:10548000C5F87C430BB0BDE8F08F042241462846A6
:10549000FCF762FA044628BB2846FBF746FC814627
:1054A0000028EFD057F0C8FADFF824B282465BF844
:1054B000047B37B97A492A4630460BB0BDE8F04F35
:1054C00078E6524639464846FCF746FA40B9204647
:1054D0002EF044F97348744D3946FDF79DFDA6E75B
:1054E0000134E4E7714907222846FCF735FA0746FC
:1054F00000287AD1202128465AF003FA044670BBCE
:105500006B486C4DFEF748FF214628460134FEF7F4
:1055100043FF0E2CF8D1FDF767FDDFF8B891664F19
:10552000DFF8B481002529464846FEF735FF0C26F2
:10553000DFF8A8A16E430024F25960480123A3407C
:1055400013420CBF414651460134FEF725FF0E2C95
:10555000F2D10135FDF748FD082DE4D192E7584915
:10556000574D01AA5AF099F902AC002848D0022FF1
:1055700011D1029A072A07D8039C0D2C04D803786E
:10558000722B13D06E2B25D04E49082300223046B3
:10559000FFF73AFF76E7FCF7BBFA01AA44F8040BE1
:1055A0002946002001375AF078F9DEE73B490C2301
:1055B00003FB02110123D1F82813A3400B43374901
:1055C0000C2000FB02123949C2F828333046FFF79D
:1055D00027FF57E7314B0C2000FB02330121D3F8A2
:1055E0002833A14023EA0103E9E728463449344F30
:1055F00001AA5AF052F902AD002480B1082C03D15F
:105600003046FFF729FE3DE7FCF782FA01AA45F88C
:10561000040B3946002001345AF03FF9EDE7082C1D
:10562000EED1029B0F2B30D8DDF80CE0BEF1070F56
:105630002BD8DDF810C0BCF10D0F26D8059F07F15F
:105640006402C82A21D8069DFF2D1ED80798642819
:105650001BD80899642918D8884216DA099C032CAB
:1056600013D8C3EBC3020D4B134483F8BD1283F868
:10567000B8E20D4983F8B9C283F8BA7283F8BB5215
:1056800083F8BC0283F8BE42A0E70F493046FFF71B
:1056900091FDF7E694EF0020441E0808DCEC0020A2
:1056A0004F1E0808601E0808A72808086A1E080878
:1056B0005C2D0808721E080804F00020771E0808F8
:1056C0007B1E08087D1E0808831E08084A1E08085D
:1056D00098290708F7340808342D0808CD1508085C
:1056E00010B504460748FDF7E3FCFAF783FE20B146
:1056F000BDE810400448FDF7DBBC20460349BDE887
:10570000104057E5991E0808A31E0808AB1E08089C
:105710002DE9F04F8FB0044602AA0846B1495AF06D
:10572000BCF8054640B903460246AF494120FEF7A2
:10573000F1FB0FB0BDE8F08FAC49FAF7C5FF0646A4
:1057400028BBA84902AA5AF0A8F8FCF7E1F90828F2
:10575000054606D9A649082332462046FFF754FEDF
:10576000E7E7A44C94F8B83683420CDC84F8B856CA
:10577000DFE73146384637F027FF013694F8B83670
:10578000B342F6DCF2E7064604F5D767F6E79A4936
:105790002846FAF799FF0646E0B9924902AA5AF05C
:1057A0007CF8FCF7B5F90828054603D99349082386
:1057B0003246D2E78F4C94F8B936834202DC84F843
:1057C000B956B6E730462946013651F091F9082E10
:1057D000F8D1F4E78A492846FAF776FF064600BB77
:1057E000804902AA5AF059F80028A2D0FCF790F993
:1057F0000828054603D9834908233246ADE77D4C86
:1058000094F8A237834209DD014604F5D76037F0EA
:105810001FFF294604F5D76037F028FF84F8A25708
:1058200087E779492846FAF74FFF064618BB714BC0
:10583000DFF8B09193F8A27706AD01461022284612
:105840005AF048F8A846BE4202AA80F20A814946A8
:1058500000205AF022F810B96C493A460AE1FCF7E8
:1058600057F9013628F8020BEDE795E80F00684C70
:1058700084E80F005DE767492846FAF725FF0646EA
:10588000C0BB5C4BDFF85C9193F8A27706ADBE42DB
:1058900002AA80F2F3804946002059F0FEFF01463B
:1058A00010B95D493A46E5E0032228465AF061F80E
:1058B000AA464FF00008284657F0BEF8404502D8E7
:1058C00001360435E3E79AF80000FCF73FF808F1E9
:1058D00001080AF8010BEEE7504DB6000446B44249
:1058E0003FF427AF06AB19192819032237F056FEEB
:1058F0000434F4E74A492846FAF7E6FE074600284A
:1059000040F0AC80DFF8EC80364998F8B86602AA1F
:1059100059F0C3FF00283FF40CAFFCF7F9F8451E1F
:1059200001D4AE4203DC3F493346012215E72D493D
:1059300002AA002059F0B1FF014600283FF4F9AE59
:105940000026082203A88DF814605AF012F80DF111
:105950000C0903A857F070F8B0421BD8214902AADD
:10596000002059F09AFF00283FF4E3AE037898F83E
:10597000B9A601930026B14656451A4902AA4FF02E
:10598000000080F2858059F088FF834650B926498F
:1059900052466FE099F80000FBF7D8FF013609F88E
:1059A000010BD6E7A6B99BF80030303B092B0FD985
:1059B0001E49FAF789FE38B11D495846FAF784FEA8
:1059C00070B11C495A4655E04FF001094FF0FF36BF
:1059D0005846FCF79DF8002830DA17495A4649E046
:1059E000B146F3E77B1E08089CE20020B21E0808BF
:1059F000B81E0808E4DB0020C31E0808CC1E0808F7
:105A0000DA1E0808E61E0808F81E0808E71F08083E
:105A100088E30020221F08080720080898E30020D8
:105A20004C1F0808511F0808272008089913080868
:105A30005D1F0808641F0808991F08080EAB03EBD8
:105A40004603013623F8200C96E72049524611E020
:105A500033F8022B24F8022F013730E01C492A4684
:105A600008E01C49002059F018FF00283FF4FDAE63
:105A700019493A462046FFF79DFB5AE61549002092
:105A800059F00BFF00283FF427AF14493A46F1E7DD
:105A900059F003FF0028D8D1114C05EBC500823026
:105AA0002044082203A937F079FD0198FBF74EFF47
:105AB00008EB050304EB051483F8820706ABBE422E
:105AC000C6DC454485F89A9733E600BFAE1F080848
:105AD000D11F08087B1E0808041F08082E1F08088D
:105AE0009CE200202DE9F041144B1B6888B004466D
:105AF000F3B11A6804A9D56A18466A46A84706464B
:105B000088B1DFF8448004AC6D46002735F8022BDD
:105B100034F8021B40460137FDF77EFABE42F5DC41
:105B200008B0BDE8F08106492046FFF743FBF7E7E0
:105B3000044908B0BDE8F041FFF73CBBAC6200206F
:105B4000662008087E2008084C20080870B5054625
:105B500008460C4656F070FF024670B1072804D183
:105B60000948214659F0F3FE38B12846064B074A4A
:105B70000749BDE87040FFF71DBBBDE87040024912
:105B80000448FDF749BA00BF161B0808852008081D
:105B900090200808BA20080870B5054608460C464B
:105BA00056F04AFF024670B1032804D10948214645
:105BB00059F0CDFE38B12846064B074A0749BDE8E3
:105BC0007040FFF7F7BABDE8704002490448FDF79E
:105BD00023BA00BF1E1B0808C82008089020080828
:105BE000D82008082DE9F04307469BB008460C462C
:105BF00056F022FF20220646002101A859F06AFE35
:105C000036B3402E08D03B494023324638461BB0BD
:105C1000BDE8F043FFF7CEBA01AD04F140084FF004
:105C2000000902222146684659F0A3FE00231022F3
:105C300009A968468DF80290FBF7CAFE099B0DF191
:105C40000202934223D10234A04505F8010BE8D1AA
:105C500009AC41220021204659F03CFE264D002E81
:105C60003BD095F88863D6B1202205F2893101A88E
:105C700059F0B4FE98B105F289312046FBF7DAFD00
:105C80001E4A1F4923463846FFF794FA04E01A7863
:105C90001C493846FFF78EFA1BB0BDE8F0831A4B5B
:105CA0001B78D3B9CEB9194E01AB1A4603CAA2422A
:105CB00030607160134606F10806F6D101232046D4
:105CC000124985F8A933FBF7B5FD1148FDF74AFAEB
:105CD00010482146FDF7A0F9DEE795F8A9331BB976
:105CE00095F88833002BF3D008492046FBF7A2FD36
:105CF000EEE700BFEB200808DCEC002029210808B3
:105D0000902008080D210808E4DB002065F0002041
:105D100033210808422108082DE9F74F8346084639
:105D20000C4656F089FEDFF818810646D8F8007058
:105D300028B1024633492046FBF70EFE80B93946AA
:105D4000314850F08DFF3149314821EA070150F0C8
:105D500087FF3049304803B0BDE8F04F50F080BFB6
:105D600023782D2B2D4B03BF013406F1FF364FF066
:105D7000010A4FF0000A4FF000094FF0FF3553F8C9
:105D8000041B51B1324620460193FBF7E5FD019B10
:105D900000280ABF4D460021012109F1010991B9EE
:105DA000B9F11D0FEBD11E492246584603B0BDE89C
:105DB000F04FFFF7FFB93B43C8F8003019491A4BC1
:105DC00012E01A4913E0114A0123AB401A40002A9D
:105DD000F7D007EA0302BAF1000FECD027EA030379
:105DE000C8F800301249134B002A18BF1946124B4D
:105DF000124803EB8503D3F8542603B0BDE8F04FF7
:105E0000FDF70AB9E71908087A210808BCD757181E
:105E1000842108084328A8E790210808082A0708D1
:105E20004F1E0808722108086B2108084F21080836
:105E30005B21080862210808B42307085B150808DD
:105E4000E06600202DE9F74F019008460E46174600
:105E5000984656F0F1FD0446E8B93F483F4DFEF73D
:105E60009BFA20460BF0E2FD3B68184206D0204624
:105E70000BF0EEFD01462846FEF78EFA0134172C92
:105E8000EFD13B6813B93648FDF7A6F803B0BDE87B
:105E9000F04FFDF7A9B8024632493046FBF75CFDEA
:105EA0000546A8B93048FDF797F82C462F4D2046F7
:105EB0000BF0BCFD10EA080F06D020460BF0C8FD21
:105EC00001462846FEF768FA0134182CEFD1DDE7C9
:105ED00033782D2B03BF013604F1FF340125002553
:105EE0004FF0000948F4000B48460BF0B1FD224684
:105EF000824601463046FBF72FFD00BB48460BF0BB
:105F000095FD1BEA000F1AD08DB1B9F1170F1CBF18
:105F10003B6840EA03081648C7F80080FDF75CF8C4
:105F20001248514603B0BDE8F04FFDF775B8B9F11E
:105F3000170F1CBF3D6885433D600E48EEE709F131
:105F40000109B9F1180FCFD10B490198324603B0BE
:105F5000BDE8F04FFFF72EB99E21080897180808F2
:105F6000A8210808E7190808AF21080898180808A8
:105F700062210808722108084F1E0808014A40F2F1
:105F800002235FE73C620020014B024A5AE700BF50
:105F9000FFFF7F003462002010B504462EF070FE33
:105FA00028B920460449BDE81040FFF703B9BDE811
:105FB00010400248FDF730B8BA210808C921080886
:105FC000074B10B50446D3F8AC033EF077FD28B973
:105FD00020460449BDE81040FFF7ECB810BD00BFF3
:105FE000DCEC0020D421080870B5054608461646AA
:105FF000FBF78EFD0D4B041E1A780EDB944205DA7A
:106000000B482146FDF708F8204670BD2EB1FF2C45
:1060100003D10848FDF700F8F6E70749013A28469A
:10602000FFF7C8F84FF0FF34EEE700BFD05B002069
:10603000EA210808FB2108080E2208082DE9F04F84
:10604000074691B08248834D0E46FCF7E5FF824932
:10605000C5F8B0D3002385F8B433062201230978AC
:106060003046402485F8B54306F038FE0A20F4F7A0
:10607000F1F995F8B4330C2BDAB240F2E4809DF8D4
:106080000C60FE2E2CD0FF2E15BF0F2415240025EA
:106090000125944240F0D780611EC9B2684647F09E
:1060A0001DFC04F140030DEB030414F8413C834252
:1060B00040F0C4806A1E012A9DF80D3012D903F009
:1060C0001F0761375C096548FCF786FF022D39D050
:1060D000013C042C34D8DFE804F00B2D2F333100C1
:1060E0000225D6E79DF80E709DF80F401E46EAE7A0
:1060F0005B48DFF8C491DFF8C4A1DFF8C4B1FCF756
:10610000D7FF5848FCF768FF6C464FF0000814F8BA
:10611000011B484608F10108FEF73EF9B8F10C0FE3
:1061200016D00AFB08F3B3F1553FF0D85846FCF7F8
:1061300053FFECE74C48DCE74C48DAE74C48D8E73B
:106140004C48D6E700238DF83F300DF11F00D0E713
:10615000FCF74AFF022D3AD06422B6FBF2F102FBB3
:1061600011623B464448D2B2C9B2FCF755FF85F0F4
:1061700001035B42DBB2012B59D8404A404B9DF8EA
:1061800010104048404E00290CBF11461946FCF73C
:1061900043FF9DF811103D4B3D4800290CBF31468F
:1061A0001946FCF739FF022D41D19DF812403948BC
:1061B000FCF712FF8CB1FF2C1FD00A23B4FBF3F1C4
:1061C00003FB11423448D2B2FCF726FF08E0334803
:1061D0003A463146FCF720FFCFE73046FCF768FF30
:1061E0009DF813402E48FCF7F7FE44B1FF2C21D058
:1061F0002C482146FCF710FF04E02B48EEE722482C
:10620000FCF756FF204E214FDFF89C800DF113055F
:10621000002415F8013F7BB1FF2B14BF3A464246DC
:10622000214622480134FCF7F7FE042CF1D111B0CD
:10623000BDE8F08F1C48E3E73246F1E71C493846D9
:10624000FEF7B8FFF3E71B48FCF732FFEFE700BFAC
:1062500054220808DCEC0020D05B002065220808EE
:106260007022080896220808772208087F2208086A
:10627000872208085A170808A82208083D2208089B
:1062800034220808DF22080844220808772C08086E
:10629000F6220808FD22080811230808C42208086D
:1062A00019230808F7340808482208082923080891
:1062B0003423080844230808AF130808ABAAAAAA85
:1062C0000E2F08082DE9F843DFF8A49007460C4686
:1062D000204656F0B1FB064658B91D4B1D481A78AA
:1062E0001D4B03EB8203D3F8E015BDE8F843FCF740
:1062F00093BE024649462046FBF72EFB60B1DFF80D
:106300006480002558F8041BB1B922463846134969
:10631000BDE8F843FEF74EBF1148124C124DFCF792
:106320005BFE54F8041B19B12846FEF735F8F8E770
:10633000BDE8F843FCF758BE32462046FBF70CFB9D
:1063400001350028DED1024B084C1D70C0E700BFAC
:10635000BC5B00204D230808B42307084F1E080823
:10636000AF2108089829070898180808A7280808DE
:10637000E719080838B50D4604461A49052228468B
:10638000FBF7EAFA68B9184B93F84C2022B90121BF
:1063900083F84C1083F84D20BDE838401348FCF7D3
:1063A00087BE134903222846FBF7D6FAA0B90E4D43
:1063B00095F84C3063B195F84D304BB10D492046FE
:1063C000FEF7F8FE002385F84C3085F84D3038BDD7
:1063D0000948FCF76DFEF5E720460849BDE838405E
:1063E000FEF7E8BECE2B0808E4DB002057230808A0
:1063F000202D08086D230808A4230808B8230808DE
:1064000070B5184C94F84C3005467BB194F84D307B
:1064100063B11549FEF7CEFE28461449FEF7CAFEC1
:10642000002084F84C0084F84D0070BD104B93F8A8
:10643000A923AAB193F8882392B903F2893203F50C
:106440006E7503F2A936106851682C4603C40832F1
:10645000B2422546F7D1012283F8F3230AF066FA07
:106460000120E2E7E4DB00206D230808C7230808C9
:10647000DCEC00202DE9F04F80468BB008460D463D
:1064800056F0DAFA024600283AD0A8492846FBF727
:1064900063FA0446A0BBFCF7A7FDA548A54DA64E90
:1064A000A64FDFF8DC82FCF703FE142050F034FB2B
:1064B0000721B4FBF1F1C1EBC102A21A304601324F
:1064C0000131FDF769FF95F8199095F91800B9F1B8
:1064D000000F0ED007F0BAF94A4601464046FCF7D5
:1064E0009BFD01340E2C05F12405E1D10BB0BDE874
:1064F000F08F07F0ABF901463846FCF78DFDF0E769
:1065000028468F4905AA59F0C8F9054620B9014621
:106510004120FCF740FEE9E78A49FAF7D5F820B9AF
:1065200089494046FEF746FEE0E7884E08270024EA
:1065300031682846FAF7C8F8002808BF3446013FFA
:1065400006F11006F4D154B981492846FAF7BCF88F
:1065500028B180492A464046FEF72CFEC6E70020B7
:1065600077498DF8130005AA59F097F90646002CD3
:106570004DD0002849D0FBF7CBFA031E42DB22792D
:10658000062A3AD1E168012202FA03F0084239D022
:106590007148DBB240FA03F1C90733D59A40013A9A
:1065A000104059F02BFA0546E0884DF0DFF86B49B2
:1065B000D0E902230978002918BF1A46217A637AA4
:1065C00005FB0133D118002712F9039002910397BC
:1065D0005B4905AA002059F060F9834600283FD1A5
:1065E0005F4901239CB3029A204692F90020CDE92D
:1065F00000312946FAF7DAFB78E75D1E13B1A37A7A
:106600009D42D1DB57493246A5E7574EFAE768B1BC
:106610000DF11301FBF756FA28B19DF813502846E7
:10662000F3F7E6FF20B95149324694E74E4EFAE7B8
:106630002846F5F7D9F88146284609F095FB0390DE
:10664000284609F0CDFB254607460294C0E7CDE970
:1066500000319DF813004A463946FAF7EBFB45E74F
:106660003849FAF731F8064600282FD1ACB1404F2F
:10667000EDB2207972B22946F5F77EF800283FF492
:1066800035AF0288037800933146C2F303233846BE
:10669000120BFCF7C1FC0136EBE738687979344C12
:1066A00072B2F5F7BDF800283FF420AF02880378F6
:1066B00000933146C2F303232046120B0136FCF748
:1066C000ABFC0E2E38687979EAD10FE72949584694
:1066D000F9F7FAFF002876D05846FBF719FA8246F8
:1066E00042B29CB12079E9B2F5F746F800284DD1C5
:1066F00029462046FAF70EFA26681F49CDF800B061
:10670000034632464046FEF755FDEFE65FFA8AF64D
:106710000D2E3868797935D99DF813301749CDF8A1
:1067200000B01A09403203F00F03EBE7E523080835
:10673000EA230808680100200024080898180808BF
:106740007B1E0808E719080812240808B404002072
:106750004927080826240808FE7F1000E4DB0020F3
:10676000F12F010835240808A7280808452408083F
:1067700057240808AA210808792408089C24080836
:1067800071250808F5F74CF80028C5D006AE31464B
:106790005046FBF763F808A94846FBF75FF8CA457F
:1067A00020D04FFA8AF38CB1029A29461370204602
:1067B000FAF7B0F9276800960246154808AB394643
:1067C000FCF72AFC92E64FF0FF3ADFE7039A114804
:1067D00093709DF813200096110908AB02F00F0288
:1067E0004031EDE75CB129462046FAF793F9266877
:1067F0000246094808AB3146FCF70EFC76E69DF8E8
:1068000013200648110908AB02F00F024031F3E7EC
:10681000C4240808E72408080F2508082A250808C2
:106820002DE9F04F07468DB008460D4656F004F9A5
:10683000044630B9014601200DB0BDE8F04FFCF729
:10684000B5BD0246A5492846FBF786F830B9A449EC
:1068500038460DB0BDE8F04FFEF7ACBCA14922466A
:106860002846FBF779F8002857D1FCF7BDFB9E4876
:10687000DFF8B482DFF88492DFF8B0A2FCF718FCEE
:10688000172050F049F90F2518F9016B002E38D068
:1068900096483146FDF780FD01240023A1B2304621
:1068A000039309F0D7FA074609F060FB90F900203E
:1068B000039B8346D2B10BB9FCF796FBBB799BF8DF
:1068C00001109BF90000039103F00203002B0CBFA1
:1068D0004F465746C1B106F0B9FF039900910346F0
:1068E0003A4683482146FCF797FB01230134052CE7
:1068F000D4D113B97F48FCF7DBFB013D15F0FF0550
:10690000C2D10DB0BDE8F08F06F0A0FF3A460346B5
:1069100021467948FCF780FBE7E7002477498DF8AA
:106920001B4007AA284658F0B8FF18B93846FEF7AA
:1069300057FCE6E70DF11B01FBF7C4F88146002880
:10694000F4D09DF81B502846F3F752FE20B96C494D
:106950003846FEF72FFCD4E7DFF8D48123464FF00A
:10696000FF3403EB430218F8022095420BD0002CB1
:1069700002DA002A08BF1C460133152BF1D1002C86
:1069800016DA6049E4E71C465C4907AA002058F083
:1069900084FF0646002800F094805049F9F794FEE1
:1069A00020BB594FDFF88481DFF88891044614E05A
:1069B0004FF00009E8E7306896F807A0F4F780FF89
:1069C000B179737911F0020F0CBF39464146024686
:1069D000009148465146FCF71FFB013421462846EA
:1069E00009F0D6F906460028E5D18AE74749022290
:1069F0003046FAF7B1FF4FEA151A0AF1400A05F0DE
:106A00000F0B002845D10390B01CFBF781F80399C8
:106A100002460491284601310592039109F0B8F924
:106A2000DDE90313059A38B9394900965B465246A9
:106A30003846FEF7BFFB64E7C0799042E9D11F46B4
:106A40006300B9F1000F31D01A1942445678013E63
:106A50007A1C234414BF2946002108EB030208F8DE
:106A600003107B1C53700AACFF23937039462246F7
:106A70002846FAF703FF08AA31462846FAF7FEFE31
:106A8000B74216D1234808AB5A465146FCF7C4FA20
:106A900037E721493046F9F717FE20B11F49009624
:106AA0005B465246C4E74FF0FF37C9E74FF0FF3669
:106AB000CEE71B48009408AB5A465146FCF7ACFAA7
:106AC0001FE704EB4404174B0093A044024698F8D8
:106AD000011001232846FAF7F5F912E7E71908082B
:106AE00012240808E5230808462508085F25080839
:106AF0006625080887250808782508087B1E0808E9
:106B00008D250808A4250808A7280808CD25080809
:106B1000D025080822260808AA210808FC2508080C
:106B200040260808F12F0108209E0708381708089A
:106B30006C400020B82508082DE9F04F89B00746C1
:106B400005AA08469C4958F0A8FE054630B90146FA
:106B50004120FDF79DFB09B0BDE8F08F9749F9F79B
:106B6000B3FD044600283CD19548964D964EDFF87B
:106B70009882FCF79DFA14204FF0CEFF95F906009D
:106B800006F064FE2968AA8801F13F4101F57E0103
:106B9000B2FA82F2890A03464131C2F11F0230463D
:106BA000FDF7FAFBE97911B14046FDF7F5FB013439
:106BB000FCF71AFA502C05F10805DFD17E4905AA29
:106BC000002058F06AFE8149F9F77EFD0028C2D105
:106BD00038467A49FFF724FE78493846FFF74AFCE1
:106BE000B9E7DFF8FC91002419F9340006F02EFE15
:106BF000804601462846F9F767FD40B10134272C4D
:106C0000F2D173492A463846FEF7D4FAA3E76A4917
:106C100005AA58F042FE064690B3FAF779FF0546FA
:106C20006C4B03EBC4034FEAC40A93F8EA314BBB45
:106C3000002D29DC09EB0A03588893F8049093F897
:106C400005A04CF093FDEBB2D0F808B0009303FB25
:106C500009AA002E00F09A803378002B00F096806D
:106C600006A93046FAF72EFF002800F08C809DF828
:106C7000185005BB0BF80A505748FCF719FA6AE799
:106C80000546CDE7002D05DD012B1A4638BF012250
:106C9000954208DD012B514938BF012301223846B6
:106CA000FEF7B2FB57E7444905AA002058F0F5FD6E
:106CB000013D0646BEE72846F3F79AFC81460028C8
:106CC0005DD02B09403302930BF80A5005F00F03F7
:106CD000434F03934FF00008BB79012B38BF0123CA
:106CE00001930026788897F804B097F805A04CF037
:106CF0003DFD06FB0BA38268D15CA94222D144452D
:106D000004D10099B1421DD00021D154DDE9021215
:106D100034485FFA86FB5FFA88FAFDF73DFB594677
:106D20005046FDF79FFF444509D12F48FDF734FB3E
:106D300050465946FDF796FF2C48FDF72DFB2C4891
:106D4000FCF7B6F9019B0136B342CBDC08F1010830
:106D5000B8F1270F07F10807BED1D9F80010B9F82C
:106D60000420244801F13F4101F57E01B2FA82F28C
:106D7000890AC2F11F024131FCF74EF9EBE63846B1
:106D8000FEF72EFAE7E61C4932463CE71BF80A30CC
:106D9000013573B11A09194903F00F03403206A8EF
:106DA000FAF7E4FC06AB16482A464146FCF734F9EC
:106DB000D1E6144BF7E700BF7B1E0808E52308085F
:106DC00066260808AC1A0020A4260808AF26080882
:106DD000B3260808B4230708D5260808CF260808D4
:106DE00098250708E7260808511708080B27080800
:106DF000252E08081527080831270808A1160808B5
:106E00004D270808EC120808F634080820B100786D
:106E1000B0FA80F040097047012070472DE9F74F24
:106E200081460846FFF7F2FF0E46054670B1002482
:106E300001A920464FF0A6FF013401464846FFF75E
:106E4000EDFF122CF4D103B0BDE8F08F0846FAF73D
:106E50005FFEC4B2112C71D8701C3D4D3D4EF9F748
:106E600064FF05EB4408670098F8F4A38346B8B9BB
:106E7000AAF102014B424B413D4495F8F423B25C28
:106E8000002B54D095F8F533192040F2EE2100FB89
:106E900003133148214603B0BDE8F04FFCF7BCB8FE
:106EA0000178304658F02DFD78B1032C94BF0022B4
:106EB00001222A4902EB4202831B0A4452FA83F35D
:106EC00093F8C8A6BAF1030F05D1484603B0BDE850
:106ED000F04FFEF785B95846F9F727FFF0B1BAF140
:106EE000020FF2D1FAF714FE40F6CA0380B29842BC
:106EF000A8BF184640F2EE239842B8BF1846A0F249
:106F0000EE201923B0FBF3F088F8F503AAF1020292
:106F100053425341EA1982F8F4A3ADE7BAF1020FE4
:106F2000F4D1484603B0BDE8F04FFEF795B90C48E0
:106F3000214603B0BDE8F04FFCF76EB809491123B4
:106F40002A46484603B0BDE8F04FFEF75DBA00BFE1
:106F5000DCEC00203CAF070861270808B4230708D1
:106F6000712708087E2708082DE9F041054686B0FC
:106F70000846FFF74BFF0F46064640B100235C4929
:106F80001A46012006B0BDE8F041FCF7CBBA08462E
:106F9000FAF7BEFD1328044600F3A18006254543F9
:106FA000781C8DF81760F9F7C0FE524E074660B1A5
:106FB000FAF7AEFDC0B212F04BFD30B17319027991
:106FC00083F81C2601238DF817303846F9F7ADFEFB
:106FD000074668B1FAF79CFD0D2809D8062303FB84
:106FE000046383F81D069DF8173001338DF81730C0
:106FF000DFF8FC80A91C0DF1170241443846FAF76E
:107000008BFDF9F792FE074668B1FAF781FD01287A
:1070100009D89DF81730062202FB0462013382F87A
:1070200020068DF817303846F9F77FFE80B1FAF761
:107030006FFDC0B212F00CFD50B19DF81730017910
:10704000062202FB0462013382F821168DF8173004
:107050009DF81720042A4FF006032FD103FB046389
:107060000022A3F82026062505FB046521F084FAFA
:1070700095F81C0612F0D0FC95F81F1695F81E76B0
:1070800019234FF46172804695F8210613FB0126FF
:1070900013FB072712F0C0FC437998F805200393EF
:1070A00095F820360097CDE90163134895F81D3611
:1070B0002146FBF7B1FF06B0BDE8F081052A05D1F6
:1070C00003FB0463002283F82126CCE7062ACAD0FA
:1070D00008EB0502002348F805309380C3E7074911
:1070E00013233246284606B0BDE8F041FEF78CB9BE
:1070F00000E20020E4DB0020F4140808CF26080892
:107100002DE9F04780468CB00846FFF77FFE054624
:1071100040B1002359491A4601200CB0BDE8F047A0
:10712000FCF77CBACDE909000B90079107A85449F8
:1071300058F086FB06464FF003FD431C04460ED173
:107140002B460A2208A93046FAF742FC089B1B7816
:107150002BB9C4B2132C96BF333444B264B2204668
:107160000AF084FC054628B94046FEF739F80CB011
:10717000BDE8F08742498DF8284007A858F060FB29
:10718000B0B300230A221946FAF722FC022609901E
:10719000DFF8EC90DFF8F0A00027494607A858F088
:1071A0004FFBF8B1FAF7B4FC364A002352F8041B3F
:1071B00088421FD1DBB20AEB8302D2F8A4219042AD
:1071C00010D1022F20D0032F23D05A1E012FD2B26C
:1071D00015D00B2A03D88DF829300136F6B20137C5
:1071E000042FDAD1052E1AD84046FEF735F8BEE74F
:1071F0000126CDE70133102BD8D10023DBE7052A88
:10720000EDD88DF82A30E8E7092BE8D88DF82C3036
:10721000E3E79A1E0D2AE2D88DF82B30DDE709ABA3
:1072200003CB286018686960A86020464FF094FD81
:10723000154A9DF82B1002EB81010346D1F8A411E9
:1072400004919DF82C1002EB8101D1F8A411039157
:107250009DF82A1002EB8101D1F8A41102919DF84A
:10726000291002EB81020021D2F8A4210192099A8F
:1072700000920846054AFBF7BBFE78E7DCE00020F9
:107280007B1E080858250708B42307080D150808B1
:107290002DE9F04F0346A1B00846FFF7B7FD0546BC
:1072A00028B1184621B0BDE8F04FFDF7D5BFDFF893
:1072B000C4920B90FF238DF82830D9F8AC33ADF889
:1072C0003000CDE9050093F838200D908DF8382076
:1072D0000F90ADF840001193099107464FF0FF3829
:1072E000934909A858F0ACFA044618BB914F0146DF
:1072F0000AAC0B0190481A57002310F9016BB242F7
:1073000040F0D28010464E1C4FF026FD314602461A
:107310003846FBF781FE022E4FF00101E9D19DF9BD
:1073200038A09DF92830534540F0C5808348FBF7CD
:1073300073FE4DE02378002BD2D0032FD4BF00265C
:107340000126062F00F2A980DFE807F004475091DC
:1073500004475000042F10D079492046FAF720FB4B
:1073600058B14FF480600DF041F9002800F0B5816C
:1073700090F90400012306930AE072492046F9F7C8
:10738000A3F970B9D9F8AC3393F93800042F22D09F
:10739000119B119320AB03EB061606F8580C01372E
:1073A0009EE720464FF0CCFB0028EFDA01230A22AB
:1073B00012A92046FAF70CFB40B2002803DB129B0F
:1073C0001B78002BE2D060482246711CFBF724FE9C
:1073D00021B0BDE8F08F0023DBE72046FAF798FBE9
:1073E00020AB03EB061646F8540CD8E75749204665
:1073F000FAF7D6FA5649B0F1000A204618BF4FF006
:10740000010AFAF7CDFA08B14AF0020A3301DFF8AF
:1074100068C1079320AB03EB0616BCE80F0006F823
:1074200050AC12AE0FC6BCE80F000FC6BCE80F0090
:107430000FC69CE8030086E8030000260DF1480A09
:10744000B346DAF80010204658F0B2FA10B19AF8B4
:1074500004301E430BF1010BBBF1070F0AF1080AC0
:10746000EFD1079B80336B4403F84F6C97E73949A2
:107470002046F9F729F9A0B137492046F9F724F950
:1074800000288CD02046FAF743FB0328804686D993
:1074900001463248FBF7C0FD9AE7314822460821F1
:1074A00094E7012305937AE70133092B7FF425AF95
:1074B0002C4801318AE70B9B1BB9AAF114025542F3
:1074C000554100235F1CE368002B62D194F900B0A2
:1074D00058460AF00DFBD4F8049018B10668002E47
:1074E00040F08B80B9F1000F237A14BF4E464FF461
:1074F0006146666023B91C48FBF78EFD03232372A7
:10750000627A2AB1194807923946FBF785FD079A36
:107510000292237ACDE9006300231A4619465846A1
:107520000DF0E8F8E06048BB11483946B2E700BF0B
:107530007B1E0808022808089F1107081F28080852
:10754000A1270808AC270808B0270808CB27080897
:10755000A42C0808441E0808AA210808CE270808F9
:10756000E62708080D2808083828080853280808BE
:107570006E280808DCEC0020842A07085849594A7C
:107580005948B9F1000F18BF0A4633463946FCF78F
:1075900003FF022F04F110044FF0010392D1119E5A
:1075A0000D9F4DB15148FBF783FD33681B6A1BB13A
:1075B0004F493A4630469847059B002B50D04D49DD
:1075C000474BBAF1140F18BF19464B48FBF724FD7F
:1075D000BAF1140F09D1059B002B43D03368DB6946
:1075E0001BB14649002230469847069B002B43D1E9
:1075F0000022314638464FF0BBFAE660B9F1000F81
:107600002CD04946304601F06BFE3D4AB3683D48F8
:107610003946FBF701FD94F80890B9F1000F0CD042
:107620003279914509D038484B463946FBF7F4FC8E
:10763000336849469B6930469847637A23B172792B
:1076400032483946FBF7E8FCF36A002BA1D03048FA
:107650003946FBF7E1FC0023F3629AE7204AD5E7BD
:107660001F49B2E7B8F1000FBFDB3368DB69002BBD
:10767000BBD028494246B6E705F08AFE0520F2F75E
:10768000E9FEDFF89490DFF894A000254FF0030B9B
:107690009AF80030AB42ABD919F8014FC4B120467B
:1076A00008F09EFB804698B12046F2F7A1FFEBB2AE
:1076B000044610B180F806B0C37120460921F2F7E4
:1076C00071FF98F80630DB07204603D5F3F754F92D
:1076D0000135DDE7F3F756F9FAE74FF0FF3049E6F9
:1076E000A7280808862708088A28080840290808C3
:1076F000E19201089427080869290808450D010846
:107700008F270808A8280808CD280808F0280808A6
:1077100027290808D50A0108F3400020D05B002083
:107720002DE9F04380468BB00846FFF76FFB0F460C
:10773000044640B100235E491A4601200BB0BDE863
:10774000F043FBF7F1BF0846FAF7E2F91D280546BA
:1077500000F3A5800A264643781C8DF82740F9F7E8
:10776000E4FA10B101238DF82730F9F7DEFA514C15
:10777000074668B1FAF7CCF90D2809D80A2303FBAC
:10778000054383F818049DF8273001338DF827301E
:10779000DFF81C91711C0DF1270249443846FAF7B5
:1077A000BBF9F9F7C2FA074668B1FAF7B1F923282D
:1077B00009D89DF827300A2202FB0542013382F8DE
:1077C0001B048DF827303846F9F7AFFA074668B141
:1077D000FAF79EF90D2809D89DF827300A2202FBF6
:1077E0000542013382F81C048DF827309DF82730BC
:1077F000062B0CD009EB06020023404649F8063060
:10780000536013810BB0BDE8F043FDF725BD0A2698
:1078100006FB054600233846A6F81E34A6F8203499
:10782000F9F783FA074618B1FAF772F9A6F81E04B9
:107830003846F9F77AFA30B1FAF76AF90A2303FB06
:107840000543A3F820041C4B4FF0FF325A600A2373
:1078500003FB05424FF46170B2F820340693B2F88E
:107860001E34059392F81C34049392F81B3403934E
:1078700092F81A14192313FB0101029192F81914BA
:1078800013FB0103019392F81834009300210B4A73
:107890002B460846FBF7ACFB0BB0BDE8F08308496C
:1078A0001D23224640460BB0BDE8F043FDF7ACBDBA
:1078B000F4F00020DCEC0020A80400202A150808C1
:1078C000CF2608082DE9F14FDFF894B106460D46A2
:1078D0002846FFF79BFA074640B1002359491A464C
:1078E000012001B0BDE8F04FFBF782BF56490522E9
:1078F0002846FAF731F860B9524B00221A601A6133
:107900001A621A631A641A651A661A6701B0BDE82A
:10791000F08F042259462846FAF71EF804462846F6
:10792000002C42D1F9F701FA07460028EED055F0B5
:1079300083F8DFF830A15FFA80F85AF8049BB9F1B8
:10794000000F07D141492A46304601B0BDE8F04F4B
:10795000FDF730BC424649463846F9F7FDFF013491
:1079600084460028E9D1374A0346154600210133F1
:10797000082B42F8101BFAD1354B03EBC4025768B1
:107980002FB93448344D4946FBF746FBA0E713F8BE
:1079900034E0F445F5DA07EB0C130FCB05EB0C14D0
:1079A00084E80F000CF1010CF3E7FAF7B1F80728AF
:1079B00004463DD82846F9F7B8F9074658B3F8F712
:1079C00025FF204B03EB041383ED000A0125384605
:1079D000F9F7ABF9074638B1F8F718FF194B03EB85
:1079E000041383ED010A01353846F9F79EF907467D
:1079F00038B1F8F70BFF134B03EB041383ED020AC6
:107A000001353846F9F791F938B9304601B0BDE88B
:107A1000F04FFDF721BC0546D9E7F8F7F7FE094B13
:107A2000032D03EB041383ED030A3FF456AFECE799
:107A30000A4907233A46304601B0BDE8F04FFDF74A
:107A4000E3BC00BF545D0020441E08084F1E080818
:107A5000A8110708601E0808A7280808CF260808EC
:107A60004A1E0808982907082DE9F34105460846EB
:107A7000FFF7CCF90C46074640B1002333491A46BC
:107A8000012002B0BDE8F041FBF74EBF304920466F
:107A9000F8F71AFE70B92D4B04224FF47A704FF4A8
:107AA000FA61013A1880598003F10403F9D102B058
:107AB000BDE8F0812046FAF72BF80328064641D8A6
:107AC0002046F9F732F9074698B1FAF721F84FF056
:107AD000010804463846F9F728F920B1FAF718F8F2
:107AE000B8F1000F09D1284602B0BDE8F041FDF71A
:107AF000B3BB40F2EE248046ECE7A4F2EE2240F263
:107B0000DC539A4203D8A0F2EE229A420AD91149D4
:107B100040F6CA0340F2EE22284602B0BDE8F0412A
:107B2000FDF772BC0C4B0D4A03EB86030021A3F852
:107B30004445A3F84605CDE9004033460846FBF727
:107B400057FAB4E7064903233A46E5E720F2002056
:107B5000441E08088C290808DCEC00206115080880
:107B60007E270808F0B5074689B00846FFF74EF9AA
:107B70000E46054640B100231A491A46012009B0B5
:107B8000BDE8F040FBF714BF0846F9F7C1FF1F2816
:107B900004461DD83046F9F7C8F8014620463DF0A6
:107BA0008DF978B10F4803AE314600EB84004FF0F9
:107BB00081F80D4A0096234629462846FBF718FA15
:107BC00009B0F0BD384609B0BDE8F040FDF708BB8C
:107BD00006491F232A46384609B0BDE8F040FDF7A4
:107BE00013BC00BF30F2002072150808CF26080829
:107BF000F0B5074685B00846FFF708F90E4605467A
:107C000040B100231D491A46012005B0BDE8F040EF
:107C1000FBF716BF0846F9F77BFF0F28044623DC65
:107C20003046F9F782F8014620463DF02DFAA8B11A
:107C3000134B04F1200203EB8203294693F85725E6
:107C4000029293F856250192B3F8543500930D4AE9
:107C500023462846FBF7CCF905B0F0BD384605B001
:107C6000BDE8F040FDF7BCBA07490F232A46384665
:107C700005B0BDE8F040FDF7C7BB00BFB0F2002083
:107C8000DCEC00207C150808CF260808F0B5054676
:107C900085B00846FFF7BAF80B46044640B100230A
:107CA0001B491A46012005B0BDE8F040FBF710BFA4
:107CB0001849184F6A46184657F0EFFD01AE88B1D3
:107CC000032C04D12846FDF7C7FA05B0F0BDF9F73B
:107CD0001FFF6A4646F8040B39460020013457F06E
:107CE000DCFDECE7032CEDD1DDE90146039F3146D5
:107CF0003A46E0B23DF004FA18B92846FDF770FAAA
:107D0000E3E705483B4632462146FBF785F9DCE7C9
:107D100030F200207B1E08088E150808F0B50646D4
:107D20008BB00846FFF772F80D46044628B30023CF
:107D30003E491A4601200BB0BDE8F040FBF766BF94
:107D40002D2903D0A1F13003092B49D8052C05DDDD
:107D500030460BB0BDE8F040FDF77EBA2846F9F793
:107D6000D7FE0AAB621C03EB440424F80C0C15F894
:107D7000013F303B092BFAD9144629780029DFD17D
:107D8000062CE5D1BDF81C20BDF91C30072ADFD830
:107D9000BDF91E50A5F5FA7292B2B2F5FA6F18D875
:107DA000BDF92070A7F5FA7292B2B2F5FA6F10D849
:107DB000BDF922C065450CDC67450ADBBDF924E04E
:107DC0000EF1640292B2C82A03D8BDF92640112CE4
:107DD00011DD174930460BB0BDE8F040FDF7EAB9B8
:107DE000202902D101352246C6E730460BB0BDE856
:107DF000F040FDF7F5B90F4A0C2000FB032264B2F6
:107E0000A2F82C53A2F82E73A2F830C382F832E302
:107E100082F833430846CDE903E4CDE9017C064A04
:107E20000095FBF7E5F80BB0F0BD00BF04F00020B3
:107E3000831E0808DCEC0020A21508082DE9F04F8D
:107E4000074689B00846FEF7E1FF8B46054640B17C
:107E500000234D491A46012009B0BDE8F04FFBF759
:107E6000F9BF4A4B084693F8B8A693F8B99693F829
:107E7000A287F9F74DFE092804467BDC0626464317
:107E80000BF101008DF81F50F8F74FFF3E4D834670
:107E900038B1F9F73DFE0D2803D80123A8558DF818
:107EA0001F305846F8F741FF834660B1F9F730FEBE
:107EB000504508D8062303FB045358709DF81F3023
:107EC00001338DF81F305846F8F72FFF824660B116
:107ED000F9F71EFE484508D8062303FB04539870A3
:107EE0009DF81F3001338DF81F305046F8F71DFF05
:107EF000814660B1F9F70CFE804508D3062303FBE9
:107F00000453D8709DF81F3001338DF81F30311D98
:107F10000DF11F0229444846F9F7FEFD9DF81F3078
:107F2000062B09D0AA1900233846AB51938009B01B
:107F3000BDE8F04FFDF790B96343EA184FF461765E
:107F40005079192111FB00600590107911FB006137
:107F50000491D17803919178029152780192EB5C6F
:107F6000009300210A4A23460846FBF741F809B06E
:107F7000BDE8F08F074909232A46384609B0BDE815
:107F8000F04FFDF741BA00BFC4620020E4DB0020DF
:107F9000EC150808CF2608082DE9F74F05460846D6
:107FA000FEF734FF0B46044618B9334A92F844767C
:107FB0002FB9284603B0BDE8F04FFDF711B92F499E
:107FC000DFF8C890DFF8C8A001AA184657F065FC92
:107FD000264610B905F0E8F908E056B90122014635
:107FE0002846FEF701F8421C04461AD103B0BDE84A
:107FF000F08FF9F78DFD2F28834636D80FB105F0A5
:10800000C7F9BBF1060F13D01D49012309785FFAA8
:108010008BF2E0B204F062FE59464846FAF7FCFFE4
:108020000027164901AA0020013657F036FCD0E798
:10803000DAF800301B0114D5FF2C0ED0E1B228462F
:10804000FDF7FCFFE8E72846FDF7F8FF013798F851
:108050000020F9B28A42F6D8DEE7DFF82480002754
:10806000F5E70848FBF724F8D6E707492F2228460A
:10807000FDF7A0F8D5E700BFDCEC00207B1E080868
:10808000D05B0020BA210808AB2908089A29080803
:10809000085700202DE9F74307460846FEF7B6FECD
:1080A0000B46044628B1384603B0BDE8F043FDF75F
:1080B000D3B82F49DFF8B89001AA184657F0EDFB66
:1080C00026460546A04665B92A4B3246D3F8AC038E
:1080D000A1B254F0BEF968BB27493846FDF76AF8EB
:1080E00028E0B8F1000F06D0B8F1010F25D03846CE
:1080F000FDF7B2F81EE0284654F09EFC1F490646E4
:1081000002462846F9F728FC50B31D493246284656
:10811000F9F722FC30B31B4932462846F9F71CFC1C
:1081200010B3194932462846F9F716FCF0B1384623
:10813000FDF756F803B0BDE8F083B31E5A425A412A
:1081400029463846FDF750FF421C0446F2D001AAEA
:108150004946002057F0A1FB08F101080546B2E7A7
:108160004646F4E70126F2E70226F0E70426EEE7AA
:108170007B1E0808DCEC0020D7290808CB2908085A
:10818000CE290808D1290808D42908082DE9F74381
:1081900080460846FEF73AFE0B46054628B14046A3
:1081A000FDF75AF803B0BDE8F0832D49DFF8B09031
:1081B00001AA184657F071FB2F4604462E467CB99B
:1081C000022DECD1A7F57A73B3F57A7F21D9254931
:1081D0004FF4FA634FF47A724046FDF715F9E1E780
:1081E0004DB1012D10D001AA4946002057F055FB92
:1081F00001350446E3E7012221464046FDF7F4FE3F
:10820000431C0646EFD1CDE72046F9F781FC07462F
:10821000E9E7154B1B68B8B25B689847FF2EBCEEC8
:10822000C00A124B0BD1124AF8EE407A1278A242E1
:1082300012DC10EE101A0F48FAF7EEFEB2E7F8EE75
:10824000407A03EB860310EE102A0B48C3ED007A48
:108250003146FAF7E1FEA5E7E3EC017A0134E6E7FF
:108260007B1E0808E52A08088867002024F3002000
:10827000D05B0020022A0808F5290808F8B507464F
:108280000846FEF7C3FDD0B1204BD3F89860013605
:10829000304609F0DDFB34460546F0B90134182CB0
:1082A000A8BF0024204609F0D3FB0546A8B9B44274
:1082B000F4D138461649BDE8F840FCF77BBF0846C4
:1082C000F9F726FC044609F0C3FB054628B9214608
:1082D0001048BDE8F840FAF79FBE0C4BC3F8984031
:1082E0000CF08AFA0C482A462146FAF795FE172C1C
:1082F00009D80A4B0C2202FB043393F80807BDE8A7
:10830000F8400CF0B3BA0020F9E700BFA804002041
:10831000112A0808252A08083B2A0808B423070858
:1083200038B5124D04460846FEF770FD60B1104B9B
:10833000104893F900104B1C0ABF0F4BC9B21978B3
:10834000BDE83840FAF768BE0846F9F7E1FB0328B4
:1083500004D8C0B2FAF7A4FA2946E4E72046074950
:10836000BDE838400322FCF725BF00BFA728080856
:10837000A8040020542A0808F4560020642A08089B
:10838000F0B5032985B005460C46164614D80B4FA8
:108390003970FAF729FE0A492846FFF7C1FF094953
:1083A000224601A8F9F7E2F901AB32460821284636
:1083B000FCF77EFEFF233B7005B0F0BDA804002053
:1083C000A7280808542A080838B5124D044608465C
:1083D000FEF71CFD60B1104B104893F901104B1CC7
:1083E0000ABF0F4BC9B25978BDE83840FAF714BE3E
:1083F0000846F9F78DFB032804D8C0B213F0C8F87B
:108400002946E4E720460749BDE838400322FCF747
:10841000D1BE00BFA7280808A8040020502A0808D9
:10842000F45600205F2A0808F0B5032985B00546F8
:108430000C46164614D80B4F7970FAF7D5FD0A4949
:108440002846FFF7C1FF094922466846F9F78EF929
:108450006B46324610212846FCF72AFEFF237B702C
:1084600005B0F0BDA8040020A7280808502A080875
:108470002DE9F74F444BDFF82C911A785B7889F897
:108480000130424B00911B7889F8002005460BB95A
:1084900004F060FA4BF0A4F900263D4CB0460D23E1
:1084A0003B4A0099734352F803A05046F9F778FA13
:1084B000002841D0B8F1000F01DDFAF795FD3548ED
:1084C0005146FBF769FF002221462846FCF764FE6F
:1084D000FAF78AFD237903F01803082B46D0102BF6
:1084E00049D02046FBF765FF294B0D2202FB0633DE
:1084F000B3F809004BF03AF98346D8B12046F8F7B3
:10850000B5FADBE902210746024401442046F8F7A8
:1085100045FA78B9019051461F48FBF73DFFDBF85B
:108520000810019A28461346CA192146FCF7D6FCC2
:10853000FAF75AFD08F10108013640F27B239E420A
:1085400004F10D04ABD10020F8F76FFAFF2389F88E
:10855000003089F80130B8F1000F11D1009A0F49AD
:10856000284603B0BDE8F04FFCF724BE0C4928466E
:10857000FFF7D6FEB5E70A492846FFF725FFB0E723
:1085800003B0BDE8F08F00BFF4560020E4DB00200C
:10859000C4320708851D08087F2A08084F1E0808EE
:1085A000A7280808A80400202DE9F74F80460846B0
:1085B0000F4654F041FA044620B1012825D13B78FA
:1085C0002A2B22D1A948AA4EAA4FFAF771FD0025FD
:1085D000B1464FF00D0A04F001040AFB05F33846DA
:1085E00059F80310FBF7D8FE314622464046FCF707
:1085F000D3FD0135FAF7F8FC40F27B239D4206F1EA
:108600000D06EAD103B0BDE8F08F3D21384657F0A2
:1086100078F9002800F0238103469A4613F8012DCB
:10862000202AFAD0AAEB070A0130054610F8013BD0
:10863000202BFAD0DFF838B25FFA8AFA4FF000093F
:108640000D2303FB09F352465BF8031000913846F3
:108650000BEB0304F9F780F9064670BB0099084656
:1086600054F0EAF9824528D1277907F0E001402942
:1086700000F0898012D871B366797F4A02EBC60692
:10868000002796F820230092BA463B46009ABA4249
:1086900002D9BAF1000F62D02BB12DE06029ECD0E5
:1086A000802900F0A48040467449FCF783FD2046F1
:1086B00003B0BDE8F04FFBF77CBE09F1010940F2C1
:1086C0007B239945BCD16E493A46404603B0BDE88C
:1086D000F04FFCF76FBD07F00703042B1CD10B46CE
:1086E0000A222846F9F774F9D4F805308342014686
:1086F000D9D32046F8F7D6FA0D2303FB09F96148D0
:108700005BF80910FBF748FE00222146404603B003
:10871000BDE8F04FFCF740BD052B0DD101230A2227
:108720002846F9F755F9D4F8053083420146BADBFB
:108730005B428342B7DCDCE72846F9F7E9F917F03A
:10874000050F0BBFB4F80520B4F90520B4F80730C5
:10875000B4F9073090420146A5DB9842EAE7D6F823
:108760001C1351F8270060B129460193F7F7ACFFBD
:10877000019B30B9394620464FF0010AF8F792FACA
:108780005346013782E76379009307F00707013FFB
:10879000009BB342B0DDAA4615F8013B202BFAD06E
:1087A0002046F8F76BFA0546042F04D8DFE807F0F7
:1087B000030E0E141D005046F9F7AAF9A8552C21F6
:1087C000504657F09EF80136451CE1E75046F9F750
:1087D0009FF925F81600F2E700230A2200215046EF
:1087E000F9F7F6F845F82600E9E70123F5E728460A
:1087F00054F022F9E37994F805A0A779DB0706463F
:108800000AD52046F8F73AFA0378014623B13246F2
:10881000284657F09CF8E0B9DEB1B74219D320469C
:10882000F8F72CFA3A46002157F054F8B2453FF6D3
:1088300063AF15493246284657F089F800283FF4BF
:108840005BAF2046F8F71AFA3246294656F0EAFF9F
:1088500052E70E493A464046FCF7ACFC23E739465E
:10886000404603B0BDE8F04F02E600BF8F2A08087B
:10887000C4320708851D0808B4230708DD2A080844
:108880004F1E0808D22A08080E2F0808A22A080836
:1088900070B5044608460E4654F0CEF831460546FB
:1088A00002462046F9F758F868B9635D1846F9F7AB
:1088B0003DF800B933B901352C4420460134037822
:1088C000202BFAD070BD0020FCE708B5044609480B
:1088D000FAF782FBFAF764FB074BD3F8AC030BF013
:1088E000F1FE04F0F1FC012C01D150F03FFCF5F752
:1088F00075FC00BFEB2A0808DCEC002010B504462C
:1089000008460B46FEF782FA28B9094903221846A1
:10891000F9F722F828B90748FAF724FC0120FFF7F5
:10892000D4FF20460449BDE81040FCF743BC00BF1B
:10893000F72A0808FB2A0808B82308082DE9F74F8A
:10894000064601AA08462E49DFF8C480DFF8C49025
:10895000DFF8ACA056F0A1FF4FF0000B04465D46D7
:10896000012714BBBBF1000F27D1264C002D43D0AB
:1089700025482946FAF750FB23780BB903F0EAFFA4
:108980004AF02EFF002384F84D30FAF7DFFA15B1D4
:108990002846F8F74AF89FB13046FDF731FD78B127
:1089A000FAF740F90020FFF790FFBBF1000F0AD063
:1089B0002046F9F7ADF885B2C5B93046FCF710FC92
:1089C00003B0BDE8F08F41462046F8F7E9FF80B9D3
:1089D00049462046F8F7E4FF0028EED05F4601AA9A
:1089E0005146002056F059FF0446BAE74FF0000BFD
:1089F000F5E74FF0010BF2E70448FAF7B3FBBFE7E6
:108A00007B1E0808E4DB0020262B0808492B0808F9
:108A10001D2B0808052C080810B50C46FDF7F0FCC6
:108A200078B1084B0122DA73FAF7FCF80648FAF736
:108A300099FB06492046F7F747FE10B10020FFF7E3
:108A400044FF10BDF45600205F2B0808A814080846
:108A50002DE9F04F93B00E460290A04930461746DC
:108A6000FFF716FF0546002840F021819C4930465B
:108A7000FFF70EFF0546002840F01B81994930465C
:108A8000FFF706FF0546002840F01581964930465D
:108A9000FFF7FEFE0546002840F00F81934930465F
:108AA000FFF7F6FE002805460ABF012408243546D4
:108AB0007F4207F010078E4928463C43FFF7E8FE47
:108AC000002800F0FC8044F020048A4B1B780BB98E
:108AD00003F040FF4AF084FE14F0090F00F05083C9
:108AE0008548FAF73FFB0020FCF71AF814F480736E
:108AF000059340F0EE808148FAF734FB8048FAF79E
:108B0000D7FA04F01803182B05D17E48FAF72AFB90
:108B10007D48FAF7CDFA01230493FAF765FA7B4909
:108B20007B48FAF779FA7B497B48FAF775FA04F43F
:108B30008473082B07D179490298FAF77CFA7749B0
:108B40000298FDF74FF814F0800307930ED1744B91
:108B500093F86826002A734A03F5CD6306BF012106
:108B600013460021704A2046FAF742FA6F49204620
:108B7000FBF78EFB6E492046FAF718FC6D4920463C
:108B8000FAF709FB6C4BD3F800A06C4B14F01006FD
:108B90001D6840F0A0806A48FAF7E4FA0396694B32
:108BA000069399466AEA05034FF00008099359F8BD
:108BB00004BBBBF1000F21D0099B039A012707FAE0
:108BC00008F73B400CBF0121002120460893FAF72B
:108BD000D5FA65EA0A033B4214BF012100215A4A33
:108BE00003905B462046FAF785FC0899564A0039FF
:108BF0005B4618BF01212046FAF7FAF908F101088F
:108C0000B8F11D0FD3D165EA0A03DFF85491089338
:108C10004FF00008069B53F804BB0693BBF1000F0E
:108C200024D0012707FA08F73D420AD06AEA050373
:108C30003B424A465B4614BF012100212046FAF719
:108C400059FC1AEA070F11D0089B039A1F400CBF6A
:108C5000012100212046FAF791FA391E03905B4664
:108C60004A4618BF01212046FAF7C2F908F1010867
:108C7000B8F11D0FCED12A4D344B354A05F5DA61D6
:108C80002046FAF7CBFC079B002B6BD0134B0298C6
:108C900022461821FCF70CFA049B002B00F0D4812B
:108CA0002C48FAF75FFA2C48FAF702FACCE10124D3
:108CB000FEE60224FCE60424FAE68124F8E62749CD
:108CC0002846FFF7E5FD00283FF4FFAE44F480742A
:108CD000FBE6002320E71A4B039360E7852B080887
:108CE0008C2B0808942B08089A2B0808AF26080834
:108CF000402B0808E4DB0020A82B0808B02B08084C
:108D0000C82B0808D42B0808FC2B0808161B0808D9
:108D1000BA2008081E1B0808D8200808A728080839
:108D2000DCEC00200E2F08080C2C0808192C080871
:108D3000232C080811180808BC690020E0660020F0
:108D4000662B0808082A0708292C0808402C080860
:108D5000DCE00020042D08081A2D0808A32B0808C1
:108D6000352C0808DFF8C0A3DFF8C0B39AF800205C
:108D70009BF80030BC4F9A4214BF01210021BB4A2E
:108D800020460CBF4FF001094FF00009FAF7F6F941
:108D90009BF80030B64A07EB83038046D3F8E035F2
:108DA00049462046FAF7A6FB9AF80030B04A07EB8E
:108DB00083074946D7F8E035AE4F2046FAF718F951
:108DC000D7ED007AAC4AF5EE407AF1EE10FA0CBF1E
:108DD000012100212046FAF70BF9A84943463A46FB
:108DE0002046FAF705FDA64B05F54A7205F5E86140
:108DF0002046FAF70BFF26B195F9BA32002B00F0A6
:108E00002981A048FAF7AEF99F48FAF751F90023F3
:108E10009E4A9F4F9F4D02F59D612046FAF79EFFA7
:108E20009D4B9E4A019300923A6829682046FBF7C1
:108E3000D9F940F202229A4B01930092BA68A968CC
:108E40002046FBF7CFF9002E40F006819548FAF74F
:108E500089F93246944F9548DFF8D4C201250021A4
:108E600017F8013B10F8018B03F1480EEE440EF8A1
:108E7000208C1CF801EB0EF14809E94409F8108C2C
:108E8000002D00F0EB80A3EB0E056B426B4101312E
:108E900008291D46E4D183F00101002720468DF802
:108EA0003070FAF76BF9824A8DF840700EAB2946A4
:108EB0002046FAF71FFB7E4A0AAB29462046FAF7FE
:108EC00097F87C4A7C4B02F52F712046FAF770FD2B
:108ED0007A4A7B4B02F52F712046FAF7B1FD754AAD
:108EE000784B02F52F712046FAF7F2FD764B774A60
:108EF00077492046FAF716FB764A774B02F5AC61C4
:108F00002046FAF711FC754A754B02F5AC61204614
:108F1000FAF70AFD734B744A74492046FAF7FAFFD0
:108F2000734B744A74492046FAF794FF002E40F0C0
:108F300097807248FAF716F9B346714DDFF8F4815D
:108F4000A5F2DC77002639460222284656F046FD77
:108F500000285A4614BF01210021204695F800A0A0
:108F60000CBF4FF001094FF00009FAF707F9BAF109
:108F7000020F834640F0E0807B784FF0190A40F200
:108F8000EE221AFB032301933B785E4A18F8033064
:108F90000093494633462046FAF7ACFA6B7840F224
:108FA000EE221AFB032301932B78564A18F803305C
:108FB0000093494633462046FAF71AF80136122E36
:108FC00005F1020507F10207BDD100214E4B0298C1
:108FD0002246FCF76DF8210740F1C6800025E9B272
:108FE000029822460135FFF7CBF9042DF7D1474F00
:108FF000474D3B782B70059B33B94648FAF7B2F8DA
:1090000045490298FFF78CF9FF232B700026F1B237
:10901000029822460136FFF707FA042EF7D17B7833
:109020006B70059B002B40F09C803C48FAF79AF847
:1090300039490298FFF7C8F93948FAF793F83948DF
:10904000F9F7CAFFFF236B70002013B0BDE8F04FA3
:10905000F7F7EBBC0B4BDBE6124AFBE62B4616E7B9
:10906000DFF898B069E700BFB4230708742B08083D
:10907000472C0808545D0020502C0808CC670020BD
:109080007D1E08086E2B08085F2C080894EF00204E
:1090900034620020586A00206C2C0808FFFF7F0013
:1090A000732C08087A2B08086C6800202CAD070880
:1090B000241E080830F2002076210808B0F20020B3
:1090C0007F2C08087A2C0808852C080800E200206C
:1090D000DCF50020F4F00020892C080820F20020A4
:1090E000922C08089A2C08089CE2002090F7002097
:1090F000A32C0808C4620020C86800207E2B080842
:10910000ACF8002061270808852B0808B06800200B
:10911000A8040020A72C0808A7280808CA2C0808BB
:10912000F12C0808072C08087C6A0020BC5B002092
:109130000C5700203CAF07083B781B4A18F8033057
:109140000093494633462046FAF7D4F92B78164A5D
:1091500018F803300093494633462046F9F748FF94
:109160002CE7FF236B7097E5104D02982978224673
:10917000FFF706F9697802982246FFF755F98BE563
:10918000A20706D5094B029819782246FFF7F8F88E
:109190005AE763077FF558AF044B02985978224687
:1091A000FFF742F950E700BF71270808B0680020B8
:1091B000224BB0F5FA6F1A680346A8BF4FF4FA6362
:1091C000B3F57A7FB8BF4FF47A73D20416D540F264
:1091D000DC52904215D007EE903A40F2DB529042BA
:1091E000F8EE677A1FD8DFED166A9FED167A9FEDCD
:1091F000160A77EEE67AA7EE870A7047B0F57A7F0F
:1092000002D89FED120A704707EE903ADFED106A20
:109210009FED107A9FED100AF8EE677A77EEE67A06
:10922000A7EE870A7047DFED0D6A9FED0D7A9FED7F
:109230000D0A77EEE67AA7EE870A704708570020F6
:1092400000007A44D62000C000E082440000000004
:1092500000407A44661000400000404200A0BB4439
:10926000D620004000008344704700BF704700BF15
:109270000020704701207047704700BF704700BF53
:10928000704700BF704700BF9FED010A704700BFE5
:109290000000000000207047064B1B78834206D96F
:1092A000054B00EB400003EBC003586970470020FA
:1092B000704700BFA9230020AC230020034B00EB24
:1092C000400003EBC003587C704700BFAC23002074
:1092D000024B1878003818BF01207047A9230020DE
:1092E00003681B6903B11847704700BF70B5094C8C
:1092F000236873B10546002606E099681A681E7354
:1093000021609047236823B15A68AA1A002A184698
:10931000F3DA70BDFCFE00200022FFF799BB0122AA
:10932000FFF796BB2DE9F84F00261F4DDFF8809020
:10933000DFF880A007460C46B0462046FDF766FDE4
:10934000D5F800B048B921465846F8F729FB20B9AE
:1093500068682146F8F724FB80B15846F9F73CFECF
:10936000696811B15046FBF717F8A96811B1484672
:10937000FBF712F8F9F738FE4FF0010801363A2EE4
:1093800005F11005D9D12046FDF740FD48B9B8F1E7
:10939000000F06D1224638460449BDE8F84FFBF7D6
:1093A00009BFBDE8F88F00BF045307085E2D080809
:1093B000582D0808522D0808F8B5354C2368002BA5
:1093C00053D00A2801D00D284DD1324D2B790BB145
:1093D000F9F70AFE304E2321304656F092FA08B1D2
:1093E000801B2060236800226BB902B12360F9F76B
:1093F000C7FD2B79EBB1BDE8F8402848F9F7ECBD83
:1094000001220B46F0E7591E705C2028F8D08AB97B
:109410000022234C204FF2543B26013E0CD1314612
:10942000204B9C4211D2E368206898476B79002B4F
:10943000DDD1F8BD2360EBE721683846FFF728FA55
:1094400001460028ECD11034E7E72B7923B1164907
:109450001648FBF729FDCAE71548F9F7BDFD0E4888
:10946000F9F726FEC3E7FF2BE3D8A0F120025E2A1E
:10947000DFD80BB92028DCD05A1C2260064AD05411
:10948000044B1B79002BD4D0BDE8F840FAF728B87C
:1094900010E50020FCFE002010E40020A3140808C2
:1094A00004530708A4560708722D08088E2D0808D3
:1094B000942D080808B5254B1B68DB040AD5B5EECA
:1094C000400AF1EE10FA12D19FED210A55F04EF943
:1094D00080B208BDDFED1F7AB4EEE70AF1EE10FAB4
:1094E0001CDA9FED1D0A55F041F980B208BDDFED91
:1094F000197AB4EEE70AF1EE10FAE5D49FED177A87
:10950000B4EEC70AF1EE10FA14D870EE677A9FED48
:10951000147A9FED140AA7EE870AE4E770EE677AE3
:109520009FED117A9FED110AA7EE870A55F01EF9FB
:1095300080B208BDDFED0E7A9FED0E7A70EE677A8D
:109540009FED0D0AA7EE870ACDE700BF0857002060
:109550000080BB440000404200007A4400E08244A6
:1095600066BEFFBE0060BB4438DFFF3E00407A4469
:109570000000834466BEFF3E00A0BB442DE9F843D3
:10958000CF4B1E6816F004072DED048B40F01F81B1
:109590009FEDCC8ACC4C16F0200605D094F8846060
:1095A00016F0020640F0AB8094F8C530DFEDC78AB4
:1095B00094F8C42013F0010340F0B780002A40F073
:1095C0009980D4ED327A9FEDC27ADFEDC26A67EE00
:1095D000877A94ED347AE8EE267A38EE477AC4ED4D
:1095E000327A84ED337A66B1012284F8C62094F889
:1095F000D820D4F88830C4F8D430012A18BFC4F871
:10960000CC30B54B93F80080B8F10D0F0BD1D4EDF1
:10961000227A9FEDB27AB24B67EE877AFDEEE77A57
:1096200017EE902A9A809FEDA77AAE4DB0EE489A39
:109630000023D4ED397AD4ED3A6A94ED388A37EEC6
:10964000677AE6EE877A37EEC87AC4ED397AA6EE05
:10965000878A85ED008A84ED388A0BB184ED338AE0
:1096600094ED3B7AD4ED3D7ADFED9F5AD4ED3E6A1E
:1096700094ED3C0A84ED3B8A38EE477AB0EE676A97
:1096800097EE256AE6EE867A37EEC07AC4ED3D7A2B
:10969000A6EE870A84ED3C0A84ED3F0A55F066F891
:1096A00002B282EAE273A3EBE2739BB2092B40F2AF
:1096B000FC80002AACBF0A380A3005B2B8F10D0FA1
:1096C000A4F8005100F0CF80B8F1240F00F0E28040
:1096D000B8F1380F05D1B0EE480A55F047F8804B85
:1096E0009880BDEC048B002E18BF374684F80271B9
:1096F000BDE8F88384F8C63084F8C43061E7D4ED5F
:10970000257AB4F89830F8EEE77AC4ED227A002B87
:109710007DD1DFED6E8A94F8C53094F8C42013F043
:1097200001034FF001063FF449AF002A67D0D4EDA2
:10973000349A694B94F8C69093F8008038EE699A91
:10974000002E49D0B9F1000F73D094ED220AD4ED68
:10975000357A644D30EE670AB8F10D0F85ED000AD9
:1097600007D1DFED627A20EE270A54F0FFFF5C4B51
:10977000988094F8D830002B40F0998095ED007ACD
:10978000002F3AD094F8D9309FED596A77EE487A95
:1097900006EE903A77EEA97AF8EEE66AF0EEE77A0E
:1097A00067EEA67A3B46F4EEC67AF1EE10FAC4BF35
:1097B00028EE866AC6EE278AF7EE007A77EEE87A18
:1097C00067EE897AE8EE877AB0EE677A31E73E4C49
:1097D000012794ED1E8ADEE6B8F10D0F37D0414D1A
:1097E000DFED388AB9F1000FC3D1002F64D094F8AF
:1097F000D830002B5ED1B0EE497A012319E7D4EDC1
:10980000329A0123C4ED349A84F8C43091E707EE0C
:10981000903ADFED356A9FED377AF8EEE77AC6EEDB
:10982000A78AF4EEC78AF1EE10FA88BFF0EE478AF5
:1098300071E7002F60D094ED220A70EE487A012380
:1098400077EEA97A84F8C630C4ED357A81E7254DE4
:10985000DFED267A95ED000A20EE270A54F086FF08
:109860001F4B9880BCE7DFED207A9FED200ADFF8E0
:10987000708068EEA77A29EE000AFDEEE77A17EE0F
:10988000903AA8F8003054F071FFA8F80650A8F8F4
:10989000020026E7DFED157A94ED330A20EE270A61
:1098A00054F064FF0E4B58801BE7002506E7022B9F
:1098B00002D00FB1012B9ED095ED007A0123B8E6BE
:1098C00048E5002000000000FCFE00209A99993E27
:1098D000CDCC4C3FCDCC4C3E263A00200AD7233C81
:1098E000283A0020B46700200000C842CDCCCC3D0F
:1098F00000401C466666663FB8F10D0F064DDBD191
:10990000DFED067A95ED000A20EE270A54F02EFFCF
:10991000034B9880D0E700BFB4670020CDCCCC3D8E
:10992000283A00204E4B1B681B0600D47047F0B548
:109930004C4C2DED048BD4F8103185B013B104F5E7
:10994000827098470023CDE90033CDE90233D4F883
:109950001421454869469047009BD4F82C21BDF955
:109960000460A4F818619D1A03D105B0BDEC048B06
:10997000F0BD94F834219DED039A94ED4E7A9DED5F
:10998000020A002A394A67EE498A92ED008AB4F841
:109990003621E0EE088AF7EE007A29EE088AFFEE1B
:1099A000006A18BFF0EE667AA0EE078A68EEA78A12
:1099B0001AB394ED507AD4ED537A94ED516AD4ED04
:1099C000546A78EEC78A38EE678AA6EE287AE6EE01
:1099D000887AD4ED4F8A94ED528A84ED507A37EE2E
:1099E000685A77EEC85AE6EE058AA6EEA58AC4ED57
